:100000000C9470110C94A1110C94A1110C94A111D9
:100010000C94A1110C94A1110C94A1110C94A11198
:100020000C94A1110C94A1110C94A1110C94A11188
:100030000C94A1110C9438B40C94A1110C94A1113E
:100040000C94A1110C943A630C94A1110C94A1117D
:100050000C94A1110C94A1110C94E2730C9426AE93
:100060000C94A1110C9462150C94A1110C94A11183
:100070000C94A1110C94A1110C94A1110C94A11138
:100080000C94A1110C94A1110C94A1110C94A11128
:100090000C94A1110C94A1110C94A1110C94A11118
:1000A0000C94A1110C94A1110C94A1110C94A11108
:1000B0000C94A1110C94A1110C94A1110C94A111F8
:1000C0000C94A1110C94A1110C94A1110C94A111E8
:1000D0000C94A1110C94A1110C94A1110C94A111D8
:1000E0000C94A1115974687484749374AD74BC74C5
:1000F000D674DA74ABA7C8A7CAA7D6A7DCA7DFA7B0
:10010000E9A75CAF61AF66AF70AF7AAFF3AF84AF12
:100110008CAF94AF9EAFA8AFB2AFC1AFCBAFF3AFD0
:10012000D5AFDFAFE9AF15B018B007B00BB011B065
:100130004FB01CB020B026B02AB02EB034B038B0CA
:100140003CB04FB042B046B04AB0084AD73B3BCE75
:10015000016E84BCBFFDC12F3D6C74319ABD5683C6
:100160003DDA3D00C77F11BED9E4BB4C3E916BAA7E
:10017000AABE000000803F05A84CCDB2D44EB938CD
:1001800036A9020C50B9918688083CA6AAAA2ABEB4
:10019000000000803F0048617264636F6465642002
:1001A00044656661756C742053657474696E677319
:1001B000204C6F616465640053746F7265642073D2
:1001C000657474696E6773207265747269657665AB
:1001D000640053657474696E67732053746F72653D
:1001E00064006563686F3A004B494C4C45442E20CF
:1001F000005072696E7465722068616C7465642E5B
:10020000206B696C6C28292063616C6C656421002B
:100210006F6B00526573656E643A20002200556E64
:100220006B6E6F776E20636F6D6D616E643A202226
:1002300000486F74656E64206F6666736574733A08
:10024000007A5F6D696E3A2000795F6D696E3A20C1
:1002500000785F6D696E3A20005A3A00593A0020E2
:10026000436F756E7420583A00453A005A3A005967
:100270003A00583A004649524D574152455F4E4167
:100280004D453A4D54312E355F33445072696E748A
:1002900065725F50524F4752414D20564552534967
:1002A0004F4E3A312E393920455854525544455213
:1002B0005F434F554E543A32204D414348494E45D5
:1002C0005F545950453A526570526170202057650D
:1002D00062736974653A687474703A2F2F77777710
:1002E0002E6D756C746F6F2E636F6D200A00426502
:1002F0006420646F6E652E0020423A002054313A2B
:100300000054303A004265642048656174696E6744
:100310002E0048656174696E6720646F6E652E00FB
:1003200020573A002054313A0054303A0048656171
:1003300074696E672E2E2E002042403A0020403A0B
:1003400000202F0020423A00202F002054313A0094
:10035000202F006F6B2054303A002569206D696EA4
:100360002C2025692073656300456E642066696CE6
:1003700065206C69737400426567696E2066696CFC
:1003800065206C697374004E6F206D6F76652E006A
:100390005072696E74696E67202E2E2E0057616947
:1003A0007420666F7220757365722E2E2E004D308C
:1003B0003500536C6565702E2E2E0046696E69738C
:1003C0006865642E00446F6E65207072696E746992
:1003D0006E672066696C6500473332310053544FB5
:1003E000505045442E20005072696E74657220731F
:1003F000746F707065642064756520746F20657219
:10040000726F72732E204669782074686520657259
:10041000726F7220616E6420757365204D393939B1
:1004200020746F20726573746172742E2028546575
:100430006D70657261747572652069732072657381
:1004400065742E205365742069742061667465722A
:100450002072657374617274696E6729006F6B0036
:100460004E6F204C696E65204E756D626572207707
:1004700069746820636865636B73756D2C204C61CB
:100480007374204C696E653A20004E6F2043686596
:10049000636B73756D2077697468206C696E652075
:1004A0006E756D6265722C204C617374204C696EA0
:1004B000653A2000636865636B73756D206D6973C1
:1004C0006D617463682C204C617374204C696E6597
:1004D0003A20004C696E65204E756D626572206928
:1004E00073206E6F74204C617374204C696E6520AC
:1004F0004E756D6265722B312C204C617374204CEB
:10050000696E653A20004D31313000446F6E6520D0
:10051000736176696E672066696C652E006F6B008B
:100520004D3239002020506C616E6E6572427566E6
:1005300066657242797465733A200020467265657B
:10054000204D656D6F72793A20004A756E20313901
:10055000203230313700436F6D70696C65643A202A
:10056000004D554C544F4F00207C20417574686FEE
:10057000723A20004A756E203139203230313720EE
:1005800031353A33313A323100204C6173742055A1
:100590007064617465643A20004D54312E3500203A
:1005A000536F6674776172652052657365740020BD
:1005B0005761746368646F672052657365740020C7
:1005C00042726F776E206F75742052657365740088
:1005D0002045787465726E616C2052657365740095
:1005E000506F7765725570007374617274002200E9
:1005F000656E717565696E672022002200656E71F7
:100600007565696E67202200FFFFFF0000A04000B3
:1006100000A0400000803F0000000000000000003B
:100620000000006563686F3A004572726F723A00AD
:100630007C3C3E5E2B3D3F2F5B5D3B2C2A225C00C9
:100640004D383420582059205A2045004D3234006E
:100650004D3233202573006175746F25692E670054
:100660006572726F722077726974696E6720746F39
:100670002066696C65004E6F742053442070726967
:100680006E74696E67002F005344207072696E7437
:10069000696E67206279746520002E0044656C6580
:1006A00074696F6E206661696C65642C2046696CA4
:1006B000653A200046696C652064656C6574656404
:1006C0003A002E006F70656E206661696C65642C5F
:1006D0002046696C653A200057726974696E67201C
:1006E000746F2066696C653A20002E006F70656E2D
:1006F000206661696C65642C2046696C653A20004F
:100700002E006F70656E206661696C65642C2046F2
:10071000696C653A200046696C652073656C656399
:10072000746564002053697A653A200046696C65F7
:10073000206F70656E65643A20002E006F70656EE4
:10074000206661696C65642C2046696C653A2000FE
:1007500053442063617264206F6B006F70656E524A
:100760006F6F74206661696C656400766F6C756D7F
:10077000652E696E6974206661696C656400534416
:1007800020696E6974206661696C006563686F3A00
:10079000004572726F723A0020746F6F206C6F6E3A
:1007A0006720657874727573696F6E2070726576F4
:1007B000656E7465640020636F6C64206578747284
:1007C0007573696F6E2070726576656E746564000E
:1007D0006563686F3A00656E6473746F7073206848
:1007E00069743A205A00205A3A00656E6473746F37
:1007F0007073206869743A20590020593A00656E78
:100800006473746F7073206869743A2058002058BC
:100810003A00656E6473746F7073206869743A206F
:100820000024F4D43050C38E20C2A24017828B70B3
:1008300011127A910D816CD90AA861E108C7586636
:1008400007615143061E4B5D05C145A7041A4111BE
:1008500004093D9803713931034036DB0265339159
:1008600002D4305402802E1D02632CEE01752AC57D
:1008700001B028A001102781018F2564012B244B92
:1008800001E0223401AC211F018D200D01801FFCED
:1008900000841EED00971DDF00B81CD200E61BC6C9
:1008A00000201BBC00641AB200B219A8000A19A0EB
:1008B000006A189900D117910040178B00B5168473
:1008C0000031167E00B31579003A157300C7146F16
:1008D0000058146A00EE1366008813630025135E47
:1008E00000C7125B006C12570015125400C1115161
:1008F0000070114F0021114B00D61049008D104798
:10090000004610440002104200C00F4000800F3E1D
:1009100000420F3C00060F3B00CB0E3800930E3711
:10092000005C0E3500270E3400F30D3200C10D318E
:1009300000900D3000600D2E00320D2D00050D2CA5
:1009400000D90C2B00AE0C2900850C29005C0C276B
:1009500000350C27000E0C2600E80B2400C40B24E5
:1009600000A00B23007D0B23005A0B2100390B2123
:1009700000180B2000F80A1F00D90A1E00BB0A1E2F
:10098000009D0A1D00800A1D00630A1C00470A1B07
:10099000002C0A1B00110A1A00F7091A00DD0919B8
:1009A00000C4091900AB091900920917007B091846
:1009B00000630917004C09160036091600200916B5
:1009C000000A091500F5081500E0081400CC081409
:1009D00000B8081400A4081400900813007D081241
:1009E000006B081300580812004608120034081162
:1009F00000230811001208110001081100F007106F
:100A000000E0071000D0071000C0071000B0070F6B
:100A100000A107100091070E0083070F0074070F55
:100A20000065070E0057070E0049070E003B070D33
:100A3000002E070E0020070D0013070D0006070DFE
:100A400000F9060C00ED060D00E0060C00D4060CC3
:100A500000C8060C00BC060C00B0060C00A4060B77
:100A60000099060C008D060B0082060B0077060B22
:100A7000006C060B0061060A0057060B004C060AC4
:100A80000042060A0038060A002E060A0024060A5A
:100A9000001A060A001006090007060A00FD0509EB
:100AA00000F4050900EB050900E2050900D9050974
:100AB00000D0050900C7050900BE050900B50508F5
:100AC00000AD050800A50509009C0508009405086F
:100AD000008C050800840508007C050800740508E2
:100AE000006C050700650508005D05070056050850
:100AF000004E0507004705070040050800380507B8
:100B000000310507002A050700230507001C05061C
:100B100000160507000F0507000805060002050777
:100B200000FB040600F5040700EE040600E80406D6
:100B300000E2040700DB040600D5040600CF04062B
:100B400000C9040600C3040600BD040600B704067D
:100B500000B1040500AC040600A6040600A00405CC
:100B6000009B04060095040500900406008A040515
:100B70000085040500800406007A0405007504055C
:100B800000700405006B040500660405006104059F
:100B9000005C04050057040500520405004D0405DF
:100BA0000048040500430405003E0404003A04051F
:100BB0000035040500300404002C0405002704045B
:100BC00000230405001E0404001A04040016040592
:100BD00000110404000D04040009040500040404C9
:100BE0000000040400FC030400F8030400F4030400
:100BF00000F0030400EC030400E8030400E4030431
:100C000000E0030400DC030400D8030400D4030460
:100C100000D0030400CC030400C8030300C5030391
:100C20000024F404D9201BC40C5C0E9804C4095F92
:100C30000265077101F405F900FB04B3004804875D
:100C400000C10369005803550003034500BE023A82
:100C5000008402310053022A0029022500040220E8
:100C600000E4011C00C8011900AF0117009801142D
:100C70000084011300710110006101100051010E88
:100C80000043010D0036010B002B010B0020010B6E
:100C900000150109000C01090003010800FB000810
:100CA00000F3000800EB000700E4000600DE000689
:100CB00000D8000600D2000600CC000500C70005E1
:100CC00000C2000500BD000400B9000400B5000426
:100CD00000B1000400AD000400A9000400A5000359
:100CE00000A20003009F0004009B00030098000383
:100CF000009500020093000300900003008D0002A5
:100D0000008B0003008800020086000200840003BC
:100D100000810002007F0002007D0002007B0002D3
:100D200000790002007700010076000200740002E2
:100D30000072000100710002006F0002006D0001EE
:100D4000006C0002006A00010069000200670001F7
:100D500000660001006500010064000200620001FD
:100D60000061000100600001005F0002005D000101
:100D7000005C0001005B0001005A00010059000105
:100D80000058000100570001005600010055000105
:100D90000054000100530000005300010052000104
:100DA0000051000100500001004F0001004E000002
:100DB000004E0001004D0001004C0001004B0000FE
:100DC000004B0001004A00010049000100480000FA
:100DD00000480001004700010046000000460001F5
:100DE00000450000004500010044000100430000F0
:100DF00000430001004200000042000100410000E9
:100E00000041000100400001003F0000003F0001E0
:100E1000003E0000003E0001003D0000003D0001DA
:100E2000003C0000003C0000003C0001003B0000D2
:100E3000003B0001003A0000003A000100390000C8
:100E400000390001003800000038000000380001BF
:100E500000370000003700010036000000360000B7
:100E600000360001003500000035000000350001AB
:100E700000340000003400000034000100330000A2
:100E80000033000000330001003200000032000097
:100E9000003200010031000000310000003100018B
:100EA000003000000030000000300001002F000082
:100EB000002F0000002F0000002F0001002E000076
:100EC000002E0000002E0001002D0000002D00006B
:100ED000002D0000002D0001002C0000002C00005F
:100EE000002C0000002C0001002B0000002B000053
:100EF000002B0000002B0001002A0000002A000047
:100F0000002A0000002A000100290000002900003A
:100F1000002900000029000000290001002800002D
:100F20000028000000280000002800000028000120
:100F30000027000000270000002700000027000015
:100F40000027000100260000002600000026000007
:100F500000260000002600010025000000250000FA
:100F600000250000002500000025000000250001EC
:100F700000240000002400000024000000240000E1
:100F800000240001002300000023000000230000D3
:100F900000230000002300000023000000230001C4
:100FA00000220000002200000022000000220000B9
:100FB00000220000002200010021000000210000AA
:100FC000002100000021000000210000002100009D
:100FD000002100010020000000200000002000008F
:100FE0000020000000200000002000000020000081
:100FF00000200001001F0000001F0000001F000073
:10100000001F0000001F0000001F0000001F000163
:10101000001E0000001E0000001E0000001E000058
:10102000006563686F3A00202D20496E76616C6917
:1010300064206578747275646572206E756D626582
:1010400072202100504944204175746F74756E659B
:101050002066696E6973686564202120506C616345
:101060006520746865204B702C204B6920616E648C
:10107000204B6420636F6E7374616E747320696EAD
:101080002074686520636F6E666967757261746944
:101090006F6E2E6800504944204175746F74756EF0
:1010A00065206661696C6564212074696D656F7582
:1010B000740020403A006F6B20543A006F6B20425E
:1010C0003A00504944204175746F74756E6520660E
:1010D00061696C6564212054656D70657261747519
:1010E000726520746F206869676800204B643A203D
:1010F00000204B693A2000204B703A200020436CBE
:10110000617369632050494420002054753A2000DF
:10111000204B753A2000206D61783A2000206D69DF
:101120006E3A200020643A200020626961733A2000
:10113000004572726F723A00A0007201B0006D013A
:10114000B0006801C0006301D0005E01D000590109
:10115000E0005401F0004F0100014A011001450177
:101160002001400130013B014001360160013101A5
:1011700070012C0190012701B0012201C0011D0165
:10118000F00118011002130130020E016002090182
:1011900090020401C002FF000003FA004003F500C2
:1011A0008003F000D003EB002004E6007004E100AF
:1011B000E004DC004005D700C005D2004006CD00A9
:1011C000D006C8008007C3003008BE00F008B90090
:1011D000C009B400B00AAF00B00BAA00D00CA50043
:1011E000000EA000500F9B00C010960050129100FE
:1011F00000148C00C0158700B0178200B0197D0064
:10120000D01B7800001E730040206E009022690001
:10121000F024640040275F0090295A00E02B55001D
:10122000102E500020304B0010324600E0334100B9
:1012300090353C001037370070383200A0392D004F
:10124000B03A2800A03B2300603C1E00103D19006E
:10125000903D1400103E0F00703E0A00C03E050095
:10126000003F0000436172642072656D6F766564B3
:10127000004361726420696E736572746564004D29
:101280003234004D3233202573004D303500257344
:1012900000257300517569740051756974004E65BD
:1012A00078742050616765005072652050616765F1
:1012B000004D61696E005061757365642E004D616B
:1012C00074657269616C206973206F75742E002DCE
:1012D0002D3A2D2D004D38340046494E49534800D3
:1012E0004241434B004E45585400466C6F770046D0
:1012F0006C6F770046616E207370656564004661AF
:101300006E207370656564004E6F7A7A6C6532008A
:101310004E6F7A7A6C6532004E6F7A7A6C65004E49
:101320006F7A7A6C65004D6F7665004D6F7665005B
:101330004D61696E0053746F7265206D656D6F72DB
:1013400079004E6F7A7A6C65004E6F7A7A6C650020
:1013500046616E2073706565640046616E2073702F
:1013600065656400507265706172650053746F72D8
:1013700065206D656D6F7279004E6F7A7A6C6500CD
:101380004E6F7A7A6C650046616E20737065656495
:101390000046616E2073706565640050726570610F
:1013A000726500436F6E6669726D2053657474696F
:1013B0006E677300536574205A00536574205A0099
:1013C0005365742059005365742059005365742087
:1013D0005800536574205800507265706172650042
:1013E00041626F7574207573005265736574204493
:1013F000656661756C740053697A65205365747411
:10140000696E67730050726568656174204142536C
:1014100020436F6E66005072656865617420504CA1
:101420004120436F6E660046616E2073706565648F
:101430000046616E207370656564004C617365726F
:1014400020456E67726176696E67204D6F64650036
:10145000436F6F6C646F776E00507265686561747E
:1014600020414253005072656865617420504C41C0
:10147000004D6F76652041786973004732382059F6
:1014800000486F6D65205900473238205800486F7A
:101490006D65205800473238205A00486F6D65202E
:1014A0005A004D38340044697361626C652053748E
:1014B000657070657273004D61696E004732380067
:1014C000526573756D65205072696E7400473332D2
:1014D000320046696E69736865642E004D383400C9
:1014E0004D383420582059205A2045004D6F7665DC
:1014F00020302E316D6D004D6F766520316D6D00A1
:101500004D6F76652031306D6D005072657061727F
:10151000650058005900457874727564657200451D
:10152000787472756465720045787472756465725A
:1015300020310045787472756465722030004D6FFB
:101540007665205A004D6F76652059004D6F76659F
:101550002058004D6F76652041786973005A004D20
:101560003035004D30330041626F75742075730063
:10157000536176652064697374616E636500466FBC
:1015800063616C2064697374616E636500466F63A8
:10159000616C2064697374616E6365005475726E6A
:1015A000206F6666204C61736572005475726E2000
:1015B0006F6E204C61736572004D6F7665205A0026
:1015C000473238205A3000486F6D65205A004D610F
:1015D000696E204D656E75004E6F20436172640028
:1015E000456E67726176652066726F6D2053442088
:1015F000636172640053746F7020456E6772617628
:10160000696E6700526573756D6520456E6772611E
:1016100076696E6700506175736520456E6772610B
:1016200076696E670047313031005365742062611E
:10163000736520706F696E74004F626A6563742011
:10164000686569676874004F626A656374206865DD
:101650006967687400466F63616C205365747469D0
:101660006E6773004D6F7665004D6F7665004E6F47
:101670002043617264005072696E742066726F6DEF
:1016800020534420636172640053746F7020507261
:10169000696E7400526573756D65205072696E7461
:1016A000005061757365205072696E7400506C61F2
:1016B0007465204C6576656C696E6700473238004A
:1016C000486F6D6520616C6C005072657061726569
:1016D000004F6666004F6E20004F6666004F6E201A
:1016E00000456E61626C652046570054756E65005A
:1016F0005374617475732073637265656E00000BBB
:101700001000000D000000003039000D000D000930
:101710000D1A0B0000FF80FF80C180C180C180C115
:1017200080C180C180C180C180C180FF80FF8004F2
:101730000D0D060000F0F0303030303030303030F9
:101740003030090D1A0A0000FF80FF8001800180FF
:101750000180FF80FF80C000C000C000C000FF808B
:10176000FF80090D1A0B0000FF80FF8001800180BF
:101770000180FF80FF800180018001800180FF8067
:10178000FF800B0D1A0D00000180038007800D8083
:10179000198031806180FFE0FFE0018001800180DD
:1017A0000180090D1A0A0000FF80FF80C000C00000
:1017B000C000FF80FF800180018001800180FF80E8
:1017C000FF80090D1A0A0000FF80FF80C000C000E2
:1017D000C000FF80FF80C180C180C180C180FF80C8
:1017E000FF80090D1A0A0000FF80FF800180018040
:1017F00001800180018001800180018001800180E1
:101800000180090D1A0B0000FF80FF80C180C1809C
:10181000C180FF80FF80C180C180C180C180FF8006
:10182000FF80090D1A0B0000FF80FF80C180C1807E
:10183000C180FF80FF800180018001800180FF80E6
:10184000FF8000060900000701850308207FFE07CE
:10185000FE07FE00000005000001070702000080EF
:10186000808080800080030202040005A0A006079B
:1018700007060000C0D8242020241805070706000A
:10188000002078A07028F02007070708000042A475
:101890004810244A8406050507000210387C10F021
:1018A000FF030707040000204080808040200307DA
:1018B0000704000080402020204080050505060028
:1018C00000A870F870A80505050600002020F82083
:1018D000200203030300FF404080030101040002D3
:1018E000E0010202020000808005070706000008F0
:1018F000081020408080050707060000F8888888C7
:101900008888F8020707030000C04040404040407C
:10191000050707060000F80808F88080F8050707A3
:10192000060000F80808F80808F80607070700008E
:1019300008182848FC0808050707060000F88080FA
:10194000F80808F8050707060000F88080F888887E
:10195000F8050707060000F8080808080808050742
:1019600007060000F88888F88888F8050707060049
:1019700000F88888F80808F8010505020000808052
:101980000080800205050300FF40004040800505FF
:10199000050600001860806018040303050001F0CC
:1019A00000F0050505060000C0300830C005070737
:1019B00007010070880810200020080707090000B0
:1019C0003C4299A999423C0507070600002050882F
:1019D000F8888888050707060000F08888F088885E
:1019E000F005070706000070888080808870050772
:1019F00007060000F08888888888F004070705003B
:101A000000F08080F08080F0040707050000F0807F
:101A100080F0808080050707060000708880B88805
:101A20008870050707060000888888F8888888017C
:101A300007070200008080808080808005070706FD
:101A400000000808080808887005070706000088D5
:101A500090A0C0A0908804070705000080808080C7
:101A60008080F007070708000082C6AA928282825F
:101A70000507070600008888C8A898888805070712
:101A800006000070888888888870050707060000AF
:101A9000F08888F08080800508080600FF7088883C
:101AA0008888887008050707060000F08888F08895
:101AB0008888050707060000708880700888700510
:101AC0000707060000F82020202020200507070631
:101AD00000008888888888887005070706000088C5
:101AE0008888888850200707070800008292929211
:101AF00092926C050707060000888850205088885D
:101B000005070706000088885020202020050707C9
:101B1000060000F80810204080F8020707030000C4
:101B2000C08080808080C00507070701008080405A
:101B300020100808020707030000C0404040404052
:101B4000C0FF050101060000F8FF050505060000BD
:101B500070087888780507070600008080F088887C
:101B600088F0050505060000708880887005070765
:101B700006000008087888888878050505060000B2
:101B80007088F88078030707030000608080C080B9
:101B900080800507070600FE788888887808300569
:101BA00007070600008080F0888888880107070200
:101BB0000000800080808080800209090300FE40D0
:101BC00000404040404040800507070600008890E4
:101BD000A0C0A0908801070702000080808080805C
:101BE0008080070505080000EC9292929205050599
:101BF000060000F0888888880505050600007088C2
:101C00008888700507070600FEF0888888F08080C5
:101C10000507070600FE7888888878080804050507
:101C2000050000B0C08080800505050600007880B2
:101C30007008F00307070400004040E040404040C7
:101C400005050506000088888888780505050600D2
:101C5000008888885020070505080000929292921B
:101C60006C0505050600008850205088050707060A
:101C700000FE88888888780830050505060000F889
:101C8000102040F803070704000020404080404037
:101C90002001070702000080808080808080030789
:101CA0000704000080404020404080FFFF0000000B
:101CB0000000000000000000000000000000000024
:101CC0000000000000000000000000000000000014
:101CD0000000000000000000000000000000000004
:101CE00000000000000000000000000000000000F4
:101CF00000000000000000000000000000000000E4
:101D000000000000000000000000000000000000D3
:101D100000000000000000000000000000000000C3
:101D200000000000000000000000000000000000B3
:101D300000000000000000000000000000000000A3
:101D40000000000000000000000000000000000093
:101D5000000000000000000000000000000000F093
:101D600000000000E00000000000000000000198FA
:101D70000000000720000000000000000000030C2D
:101D80000000001C20000000000000000000020510
:101D9000C0000070200000000001F70000000205F4
:101DA000300001C020000090000014800000030DEE
:101DB0000C000700200D92B98C001440000001991E
:101DC00003001C00201252925201F440000000F166
:101DD00000C0700020125292520014400000000116
:101DE0000031C00020125292520014800000000105
:101DF000000E000020124E998C01F700000003FD38
:101E00000004001020000000000000000000020597
:101E100080040030200000000000000000000204E8
:101E2000600400D020000000000000000000020458
:101E3000180403102000000000000000000002044D
:101E400006040C1020000000000000000000020446
:101E50000184301020000000000000000000020497
:101E60000064C01020000000000000000000020418
:101E7000001F00102010023FF883E0000000020461
:101E80000004001020180601008200000000020477
:101E90000000001020140A0100820000000002046B
:101EA0000000001020121201008200000000020455
:101EB00000000010201122010083E0000000020455
:101EC000000000102010C201008020000000020469
:101ED0000000001020100201008020000000020419
:101EE00000000010201002010090200000000204F9
:101EF00000000010201002010093E0000000020426
:101F0000000000102000000000000000000002049B
:101F1000000000102000000000000000000002048B
:101F2000000000102000000000000000000002047B
:101F3000000000102000000000000000000002046B
:101F4000000000102000000000000000000002045B
:101F5000000000102000000000000000000002044B
:101F60000000001020000000000000000000010838
:101F700000000010200000000000000000000090A1
:101F80000000001FE00000000000000000000060F2
:101F90000000000000000000000000000000000041
:101FA0000000000000000000000000000000000031
:101FB0000000000000000000000000000000000021
:101FC0000000000000000000000000000000000011
:101FD0000000000000000000000000000000000001
:101FE00000000000000000000000000000000000F1
:101FF00000000000000000000000000000000000E1
:1020000000000000000000000000000000000000D0
:1020100000000000000000000000000000000000C0
:1020200000000000000000000000000000000000B0
:1020300000000000000000000000000000000000A0
:102040000000000000000000000000000000000090
:102050000000000000000000000000000000000080
:102060000000000000000000000000000000000070
:102070000000000000000000000000000000000060
:102080000000000000000000000000000000000050
:102090000000000000000000000000000000000040
:1020A0000000000000000000000000000000000030
:1020B0000002010000040080000800400010002021
:1020C000002000100040000800FFFFFC00804804D2
:1020D00000804804008048040080480400804804D0
:1020E0000080480400FFCFFC00000000000000005A
:1020F0000000000000000000000000000000300CA4
:10210000000060060000C0030001800180030000A1
:10211000C0060000600C00003018000018300000FD
:102120000C600000067FFFFFFE7FFFFFFE600FF0E8
:1021300006600C3006600C3006600C3006600C3017
:1021400006600C3006600C30067FFC3FFE3FF81F37
:10215000FC00000000000000000000000000000083
:1021600000000000000000000000000000FFE0FF91
:10217000D11000FFFEFFD0FFE0FFC1FFD140A0C89B
:10218000A6A22FF800238127AC00AFFF64A5FF644F
:10219000FF64A4FFD0FFFE00000A0B02090C0D0E25
:1021A0000807030401000000000000000000000018
:1021B000000000000000000000000000000000001F
:1021C00000000012111000000000000000000000DC
:1021D00000000000000000000000000000010210EC
:1021E0002020080810204010204080020102010831
:1021F00004020101020408102040808040201008E1
:102200000402018004020180402010080402010839
:102210000402010102040810204080010204081099
:102220002040800505050507050808080802020288
:10223000020A0A0808040404040101010101010161
:10224000010303030303030303040707070C0C0C38
:102250000C0C0C0C0C020202020606060606060610
:10226000060B0B0B0B0B0B0B0B00002200250028A1
:10227000002B002E0031003400020100000501088F
:10228000010B0100002100240027002A002D00304E
:1022900000330001010000040107010A01024E4160
:1022A0004E494E495459494E46CDCCCC3D0AD723D0
:1022B0003C17B7D13877CC2B329595E6241FB14F18
:1022C0000A000020410000C84200401C4620BCBE5D
:1022D0004CCA1B0E5AAEC59D74001E37F8A5223796
:1022E00011241FBECFEFD1E2DEBFCDBF00E00CBF97
:1022F00015E0A0E0B2E0ECECF0E801E00BBF02C0BA
:1023000007900D92A037B107D9F723E1A0E7B5E018
:1023100001C01D92A93AB207E1F712E2CEEDD2E276
:1023200000E006C022970109FE010BBF0E94A5B97B
:10233000CA3DD10780E00807A9F70E9498B40C9421
:1023400055C00C940000EF92FF920F931F93CF9310
:10235000DF931F92CDB7DEB78C017B01460FF701EB
:1023600061917F01F8018081918149830E949EBF24
:10237000F8018081918101969183808349814E117A
:10238000EECF0F90DF91CF911F910F91FF90EF90C3
:102390000895EF92FF920F931F93CF93DF931F92B5
:1023A000CDB7DEB78C017B01460FF80180819181AA
:1023B00049830E9496BFF70181937F01F8018081D4
:1023C000918101969183808349814E11EECF0F90C8
:1023D000DF91CF911F910F91FF90EF9008950F9390
:1023E0001F93CF93DF93CDB7DEB72A970FB6F8943C
:1023F000DEBF0FBECDBF80E390E3A0E3B0E08D83EE
:102400009E83AF83B88704E610E01A87098744E00B
:10241000BE016B5F7F4FCE01099695DF40E165E518
:1024200071E1CE0109968FDF40E165E671E1CE01F1
:10243000099689DF40E165E471E1CE01099683DF09
:1024400044E06DE371E1CE0109967DDF44E069E38C
:1024500071E1CE01099677DF44E061E471E1CE01DC
:10246000099671DF44E069E271E1CE0109966BDF04
:1024700044E065E771E1CE01099665DF44E065E37C
:1024800071E1CE0109965FDF44E061E371E1CE01C5
:10249000099659DF44E06DE271E1CE01099653DF00
:1024A0004CE06EEC78E0CE0109964DDF42E06AE048
:1024B00079E0CE01099647DF41E06BEF78E0CE018D
:1024C000099641DF42E06CEF78E0CE0109963BDFF0
:1024D00042E06EEF78E0CE01099635DF42E060E041
:1024E00079E0CE0109962FDF42E06DEE72E1CE0178
:1024F000099629DF42E06BEE72E1CE01099623DFF7
:1025000042E069EE72E1CE0109961DDF42E067EE1E
:1025100072E1CE01099617DF42E065EE72E1CE016D
:10252000099611DF42E063EE72E1CE0109960BDFFE
:1025300044E069E672E0CE01099605DF44E065E615
:1025400072E0CE010996FFDE44E061E672E0CE0162
:102550000996F9DE86E590E3A7E3B0E089839A83E4
:10256000AB83BC831A87098744E0BE016F5F7F4F4E
:10257000CE010996E8DEE2EEF1E08491882341F095
:102580009091C00095FFFCCF8093C6003196F5CFA7
:10259000E2EDF1E08491882341F09091C00095FF35
:1025A000FCCF8093C6003196F5CF8091C00085FFA7
:1025B000FCCF8AE08093C6002A960FB6F894DEBF5F
:1025C0000FBECDBFDF91CF911F910F910895AF92B4
:1025D000BF92CF92DF92EF92FF920F931F93CF9310
:1025E000DF93CDB7DEB7E0970FB6F894DEBF0FBE2E
:1025F000CDBF80E1E9E9F2E0DE01919601900D9214
:102600008A95E1F780E1E9EAF2E0DE015196019076
:102610000D928A95E1F780E1E9EBF2E0DE01119697
:1026200001900D928A95E1F76E0181E2C80ED11CEE
:1026300085E5E82E81E1F82E8E010F5E1F4F65E6DD
:1026400071E1AE014F5F5F4F95E4A92E91E1B92E84
:1026500020E030E0F60181919191A191B1916F015B
:10266000F70181939193A193B1937F01F801819137
:102670009191A191B1918F01FB0181939193A193CC
:10268000B193BF01FA0181919191A191B191AF01F3
:10269000F50181939193A193B1935F012F5F3F4F18
:1026A00024303105B9F60E94476280E090E0AAEF3D
:1026B000B4E480933D1190933E11A0933F11B093E9
:1026C000401180E090E8ABE3B5E48093391190933A
:1026D0003A11A0933B11B0933C111092411110920A
:1026E0004211109243111092441180E29EE4A0E046
:1026F000B0E08093751190937611A0937711B09309
:10270000781180E090E0A0EAB1E4809329119093E1
:102710002A11A0932B11B0932C1180E090E0A0E23D
:10272000B1E48093351190933611A0933711B09393
:1027300038118DEC9CECACECBEE38093311190939E
:102740003211A0933311B093341180E090E0A0EAED
:10275000B0E480932D1190932E11A0932F11B0937C
:1027600030111092D6081092D7081092D808109203
:10277000D9081092D2081092D3081092D40810925F
:10278000D5081092CE081092CF081092D00810925F
:10279000D1088EE590E090930B0980930A0910927E
:1027A000F60881E08093FB0880E991E09093FD08B2
:1027B0008093FC089093FF088093FE089093010992
:1027C0008093000988EC90E09093EE128093ED12D4
:1027D0008CE390E09093EC128093EB128DE790E005
:1027E0009093EA128093E91220EF30E03093E812E0
:1027F0002093E7122AE530E03093E6122093E512A9
:102800009093E4128093E3128AE999E9A1EBB1E491
:102810008093690290936A02A0936B02B0936C025A
:1028200061E77DE38AE89FE30E947D75609365021E
:1028300070936602809367029093680260E070E094
:1028400084EE92E40E948975609361027093620243
:1028500080936302909364020E94736C80E090E026
:10286000A0E8BFE380935D0290935E02A0935F02B5
:10287000B0936002B4DDE2EEF1E08491882341F090
:102880009091C00095FFFCCF8093C6003196F5CFA4
:10289000E6E9F1E08491882341F09091C00095FF32
:1028A000FCCF8093C6003196F5CF8091C00085FFA4
:1028B000FCCF8AE08093C600E0960FB6F894DEBFA6
:1028C0000FBECDBFDF91CF911F910F91FF90EF9081
:1028D000DF90CF90BF90AF900895CF93DF93CDB7A7
:1028E000DEB72A970FB6F894DEBF0FBECDBF84E6E1
:1028F00090E09A87898786E590E3A7E3B0E0898333
:102900009A83AB83BC8344E0BE016B5F7F4FCE01F3
:1029100009963FDD43E050E0BE016B5F7F4FCE0183
:1029200001960E94E5BC892B09F0C2C040E165E533
:1029300071E1CE0109962DDD40E165E671E1CE0140
:10294000099627DD40E165E471E1CE01099621DDBC
:102950000E94476244E06DE371E1CE01099619DD02
:1029600044E069E371E1CE01099613DD44E061E4DE
:1029700071E1CE0109960DDD44E069E271E1CE011D
:10298000099607DD44E065E771E1CE01099601DDB6
:1029900044E065E371E1CE010996FBDC44E061E3CC
:1029A00071E1CE010996F5DC44E06DE271E1CE0102
:1029B0000996EFDC4CE06EEC78E0CE010996E9DC9C
:1029C00042E06AE079E0CE010996E3DC41E06BEF9A
:1029D00078E0CE010996DDDC42E06CEF78E0CE01D4
:1029E0000996D7DC42E06EEF78E0CE010996D1DCA3
:1029F00042E060E079E0CE010996CBDC42E06DEE8A
:102A000072E1CE010996C5DC42E06BEE72E1CE01C7
:102A10000996BFDC42E069EE72E1CE010996B9DCAD
:102A200042E067EE72E1CE010996B3DC42E065EE6A
:102A300072E1CE010996ADDC42E063EE72E1CE01B7
:102A40000996A7DC44E069E672E0CE010996A1DCB4
:102A500044E065E672E0CE0109969BDC44E061E665
:102A600072E0CE01099695DC0E94736CE2EEF1E013
:102A70008491882341F09091C00095FFFCCF809312
:102A8000C6003196F5CFE8EBF1E08491882341F060
:102A90009091C00095FFFCCF8093C6003196F5CF92
:102AA0008091C00085FFFCCF8AE08093C60001C002
:102AB0008EDD2A960FB6F894DEBF0FBECDBFDF9134
:102AC000CF9108951F920F920FB60F9211240BB65B
:102AD0000F922F933F934F935F936F938F939F9397
:102AE000EF93FF936091C6002091F1053091F205BC
:102AF000C90101968F7799274091F3055091F4050C
:102B00008417950741F0F901EF58FA4F60839093CD
:102B1000F2058093F105FF91EF919F918F916F9155
:102B20005F914F913F912F910F900BBE0F900FBE71
:102B30000F901F9018959A01AB01211581EE38076F
:102B40004105510549F182E08093C00060E079E0E1
:102B50008DE390E00E9473B9215031094109510978
:102B6000CA01B90122E030E040E050E00E9473B9B0
:102B70003093C5002093C4008091C1008061809390
:102B8000C1008091C10088608093C1008091C10024
:102B900080688093C10008951092C00020E130E069
:102BA000E7CF2091F3053091F4058091F1059091E4
:102BB000F2058217930771F0F901EF58FA4F8081FF
:102BC0002F5F3F4F2F7733273093F4052093F30582
:102BD00090E008958FEF9FEF08958091F305909115
:102BE000F4059093F2058093F10508954F925F925A
:102BF0006F927F928F929F92AF92BF92CF92DF920D
:102C0000EF92FF920F931F93CF93DF93CDB7DEB771
:102C1000A0970FB6F894DEBF0FBECDBF5C01411583
:102C2000510561057105E9F420E030E040E350E032
:102C300060E070E0A0960FB6F894DEBF0FBECDBF87
:102C4000DF91CF911F910F91FF90EF90DF90CF9088
:102C5000BF90AF909F908F907F906F905F904F90BC
:102C60005BC08E010F5F1F4FC12CD12C7601480134
:102C7000422E512C612C712C8FEFC81AD80AE80A09
:102C8000F80ACB01BA01A30192010E9451B9CA010D
:102C9000F80161938F01A901BC014115510561053E
:102CA000710551F7F1E0CF1AD108E108F108F401FC
:102CB000EC0DFD1D80818A3010F440E301C047E334
:102CC000480F552747FD5095652F752F20E030E0C0
:102CD000C50122D081E0C81AD108E108F108EFEF60
:102CE000CE16DE06EE06FE0611F7A0960FB6F89495
:102CF000DEBF0FBECDBFDF91CF911F910F91FF902F
:102D0000EF90DF90CF90BF90AF909F908F907F908B
:102D10006F905F904F9008952115310539F480919F
:102D2000C00085FFFCCF4093C60008952A303105CE
:102D300009F41CC05BCFCF93DF93EC0120E030E0BF
:102D40004DE050E060E070E0E7DF20E030E04AE096
:102D500050E060E070E0CE01DF91CF91DDCF9A01CD
:102D6000AB01662757FD6095762FD6CFCF92DF92C5
:102D7000EF92FF92CF93DF93EC016A017B0177FF23
:102D80000FC020E030E04DE250E060E070E0C4DFD2
:102D9000F094E094D094C094C11CD11CE11CF11CAF
:102DA0002AE0B701A601CE01DF91CF91FF90EF900D
:102DB000DF90CF901BCF2115310539F48091C000F1
:102DC00085FFFCCF4093C600089510CF9A01462F8F
:102DD00050E060E070E0EFCFCF93DF93EC019A0119
:102DE000AB0160E070E0E7DFCE01DF91CF91A3CFD0
:102DF0008F929F92AF92BF92CF92DF92EF92FF920B
:102E00001F93CF93DF93EC016A017B01122F20E027
:102E100030E0A901C701B6010E9480B587FF0CC050
:102E200020E030E04DE250E060E070E0CE0174DF81
:102E3000F7FAF094F7F8F094B12C60E070E080E0DD
:102E40009FE3B11641F020E030E040E251E40E94FF
:102E500087B5B394F6CF9B01AC01C701B6010E94C0
:102E6000A7B46B017C010E94F4B54B015C010E9488
:102E700020B69B01AC01C701B6010E94A6B46B014C
:102E80007C012AE0B501A401CE01B0DE112361F07E
:102E9000E9E4F4E08191882339F09091C00095FF36
:102EA000FCCF8093C600F6CF112319F120E030E06B
:102EB00040E251E4C701B6010E9455B86B017C01A4
:102EC0000E94EFB54B01AA2497FCA094BA2CB5013F
:102ED000A401CE014BDFC501B4010E9422B69B01C3
:102EE000AC01C701B6010E94A6B46B017C01115070
:102EF000DBCFDF91CF911F91FF90EF90DF90CF90CC
:102F0000BF90AF909F908F90089572CF4F925F9235
:102F10006F927F92AF92BF92CF92DF92EF92FF9229
:102F20000F931F93CF93DF935C01FC01EE0FFF1F04
:102F3000EE0FFF1FE652F74F1082118212821382AA
:102F400026EE38E042EE58E06EED78E08AED98E04B
:102F50000E947C61E501C85FD94FFE0154903501A4
:102F6000660C771C660C771C83010557174FF3011D
:102F7000EA54F74F20E030E040EC5FE3608171817C
:102F8000828193810E9455B86B017C01652D772762
:102F900067FD7095872F972F0E9422B69B01AC0189
:102FA000C701B6010E9455B8F8016083718382831E
:102FB0009383F301E15DFD4F608171818281938193
:102FC00060930A0270930B0280930C0290930D029F
:102FD00020E030E040E752E40E9487B52DE9C22EA0
:102FE00028E0D22E7B018C0127E938E043E958E044
:102FF0006FE878E08BE898E00E94E5570E94616AEC
:10300000F301E652F74F108211821282138226EEEC
:1030100038E042EE58E06EED78E08AED98E00E94EC
:103020007C61C301855F994F3C01FC01C590D5903F
:10303000E590F490FE0164918501000F111F000FCF
:10304000111F0557174FF7FAF094F7F8F094772708
:1030500067FD7095872F972F0E9422B69B01AC01C8
:10306000C701B6010E9455B8F8016083718382835D
:10307000938320E030E040E752E460910A027091CF
:103080000B0280910C0290910D020E9487B54DE9D0
:10309000C42E48E0D42E7B018C0127E938E043E9B7
:1030A00058E06FE878E08BE898E00E94E5570E94CE
:1030B000616AF3016591759185919491FE01749017
:1030C000E501CC0FDD1FCC0FDD1F8E010557174F1B
:1030D0009B01AC010E94A7B46B017C01672D77278F
:1030E00067FD7095872F972F0E9422B69B01AC0138
:1030F000C701B6010E9455B8F801608371838283CD
:103100009383FE01E15DFD4F20E030E040E05FE3AE
:1031100060817181828193810E9455B860930A0217
:1031200070930B0280930C0290930D0220E030E02C
:1031300040E752E40E9487B5EDE9CE2EE8E0DE2EAE
:103140007B018C0127E938E043E958E06FE878E03B
:103150008BE898E00E94E5570E94616AFE01E25305
:10316000F74FC080D180E280F380FE01E655F74F33
:103170002081318142815381C701B6010E94A7B4E9
:103180002B013C01FE01E652F74F6083718382837D
:103190009383C95ED94FFE01659175918591949194
:1031A000E501CC0FDD1FCC0FDD1F8E010E53174F35
:1031B000A70196010E94A7B4F801608371838283FE
:1031C00093838E01015E1D4FFE01E256F74FA7016A
:1031D000960160817181828193810E94A7B4F80178
:1031E0006083718382839383C557D74F4882598206
:1031F0006A827B8210920A0210920B0210920C02D9
:1032000010920D02DF91CF911F910F91FF90EF90DF
:10321000DF90CF90BF90AF907F906F905F904F9076
:103220000C942A63FC012491222341F03091C000C8
:1032300035FFFCCF2093C6000196F4CF22E030E0AA
:1032400080E795E062CECF93DF931F921F92CDB7B8
:10325000DEB78091A3139091A4139E012F5F3F4F7F
:10326000009719F4295A334102C0281B390B3A83BD
:10327000298389819A810F900F90DF91CF910895D2
:103280002091E0063091E106243031050CF06AC04F
:103290004091E2065091E30660E6649F9001659FCD
:1032A000300D1124BC01C9018651994F0E94DEBC2A
:1032B000E3E2F6E08491882341F09091C00095FF0D
:1032C000FCCF8093C6003196F5CFEDEFF5E0849109
:1032D000882341F09091C00095FFFCCF8093C600F9
:1032E0003196F5CF8091E2069091E30620E6289F83
:1032F000F001299FF00D1124E651F94F81918823A7
:1033000039F09091C00095FFFCCF8093C600F6CFB6
:10331000EBEFF5E08491882341F09091C00095FF98
:10332000FCCF8093C6003196F5CF8091C00085FF19
:10333000FCCF8AE08093C6008091E2069091E3067C
:10334000019664E070E00E943EB99093E30680939A
:10335000E2068091E0069091E10601969093E106E5
:103360008093E00608952091E0063091E106243034
:1033700031050CF06AC04091E2065091E30660E628
:10338000649F9001659F300D1124BC01C9018651D5
:10339000994F0E9461BCE3E2F6E08491882341F0FA
:1033A0009091C00095FFFCCF8093C6003196F5CF79
:1033B000E0EFF5E08491882341F09091C00095FF03
:1033C000FCCF8093C6003196F5CF8091E2069091B4
:1033D000E30620E6289FF001299FF00D1124E65115
:1033E000F94F8191882339F09091C00095FFFCCF6F
:1033F0008093C600F6CFEEEEF5E08491882341F08D
:103400009091C00095FFFCCF8093C6003196F5CF18
:103410008091C00085FFFCCF8AE08093C600809138
:10342000E2069091E306019664E070E00E943EB9E6
:103430009093E3068093E2068091E0069091E10686
:1034400001969093E1068093E00608958F929F92F3
:10345000AF92BF92CF92DF92EF92FF926091FC0801
:103460007091FD08882777FD8095982F0E9422B6DD
:103470004B015C0160931F02709320028093210234
:10348000909322026091FE087091FF08882777FDD3
:103490008095982F0E9422B66B017C0160932302D5
:1034A0007093240280932502909326026091000974
:1034B00070910109882777FD8095982F0E9422B688
:1034C00060932702709328028093290290932A0226
:1034D0008092B6089092B708A092B808B092B90846
:1034E000C092BA08D092BB08E092BC08F092BD0826
:1034F0006093BE087093BF088093C0089093C10882
:103500001092AA081092AB081092AC081092AD0865
:103510001092AE081092AF081092B0081092B10845
:103520001092B2081092B3081092B4081092B50825
:1035300080929E0890929F08A092A008B092A10845
:10354000C092A208D092A308E092A408F092A50825
:103550006093A6087093A7088093A8089093A90881
:10356000FF90EF90DF90CF90BF90AF909F908F90A3
:10357000089560E080E40E9450B09FB7F894E8E0BE
:10358000F1E08081846080839FBF0895269A2E9801
:103590000895EFDFFBDF40E950ED63E070E080E786
:1035A00095E0C9DAE8EEF5E08491882341F0909146
:1035B000C00095FFFCCF8093C6003196F5CF809177
:1035C000C00085FFFCCF8AE08093C60084B780FFEF
:1035D00014C0E0EEF5E09491992341F02091C000F1
:1035E00025FFFCCF9093C6003196F5CF9091C00097
:1035F00095FFFCCF9AE09093C60081FF14C0E0EDE8
:10360000F5E09491992341F02091C00025FFFCCF73
:103610009093C6003196F5CF9091C00095FFFCCFF6
:103620009AE09093C60082FF14C0EFEBF5E094910E
:10363000992341F02091C00025FFFCCF9093C60054
:103640003196F5CF9091C00095FFFCCF9AE0909312
:10365000C60083FF14C0EFEAF5E09491992341F08E
:103660002091C00025FFFCCF9093C6003196F5CF86
:103670009091C00095FFFCCF9AE09093C60085FF23
:1036800014C0EFE9F5E08491882341F09091C000E7
:1036900095FFFCCF8093C6003196F5CF8091C00096
:1036A00085FFFCCF8AE08093C60014BEE9E9F5E00F
:1036B0008491882341F09091C00095FFFCCF8093C6
:1036C000C6003196F5CF8091C00085FFFCCF8AE01F
:1036D0008093C600E9E8F5E08491882341F0909159
:1036E000C00095FFFCCF8093C6003196F5CFE4E78C
:1036F000F5E08491882341F09091C00095FFFCCFC4
:103700008093C6003196F5CFE8E6F5E084918823F2
:1037100041F09091C00095FFFCCF8093C600319698
:10372000F5CFE1E6F5E08491882341F09091C00067
:1037300095FFFCCF8093C6003196F5CF8091C000F5
:1037400085FFFCCF8AE08093C600E6E5F5E0849132
:10375000882341F09091C00095FFFCCF8093C60074
:103760003196F5CFEAE4F5E08491882341F0909119
:10377000C00095FFFCCF8093C6003196F5CF8091B5
:10378000C00085FFFCCF8AE08093C600EBE3F5E044
:103790008491882341F09091C00095FFFCCF8093E5
:1037A000C6003196F5CF4FDD4AE050E0BC0180E71E
:1037B00095E0D5DAE4E2F5E08491882341F0909138
:1037C000C00095FFFCCF8093C6003196F5CF4AE04C
:1037D00050E060ED74E080E795E0C1DA8091C000D0
:1037E00085FFFCCF8AE08093C6001092E606109217
:1037F000E7061092E8061092E9061092F608109279
:10380000F0081092F7081092F30881E18093F40811
:103810001092F80881E08093F9088093FB0880E912
:1038200091E09093FD088093FC089093FF088093AB
:10383000FE0890930109809300091092F5084DD875
:1038400005DE0E94A76E0E947F560E94D4690E94E6
:10385000F686109208098BE080930C0910920709F4
:103860001092060908958091DA069091DB0660E0D7
:1038700070E001960C94B8B98091DA069091DB065D
:103880004AE050E060E070E001960C9420BB682FA5
:10389000772767FD70952091E4063091E50640E6B4
:1038A000429FC001439F900D11248651994F0E9461
:1038B000D3BC9093DB068093DA0621E0892B09F4D0
:1038C00020E0822F08950E9470AE6093D606709318
:1038D000D7068093D8069093D906E091E406F0913C
:1038E000E506EA51F94F8081811114C0E0E1F2E070
:1038F0008491882341F09091C00095FFFCCF809384
:10390000C6003196F5CF8091C00085FFFCCF8AE0DC
:103910008093C600089580E795E05FD9E3E1F2E087
:103920008491882341F09091C00095FFFCCF809353
:10393000C6003196F5CF40916F08509170086091A4
:103940007108709172084F5F5F4F6F4F7F4F2AE091
:1039500030E080E795E0E0D98091C00085FFFCCFA2
:103960008AE08093C600AFCF4F925F926F927F92B2
:103970009F92AF92BF92CF92DF92EF92FF920F93FE
:103980001F93CF93DF9330E6B32EC4E0D0E007EE71
:1039900013E04AE0A42E5DE5E52E54E0F52E9924CF
:1039A00093948091F1059091F2052091F305309167
:1039B000F405821B930B8F779927892B09F424C276
:1039C0008091E0069091E10604970CF01DC280E71B
:1039D00095E0E7D88093DF061092F6082091DD0687
:1039E0003091DE068A3061F08D3051F08A3321F457
:1039F0009091DC06992321F02F3531050CF427C175
:103A00002115310509F441C18091E2069091E30648
:103A1000B89E6001B99ED00C1124F601E20FF31F8D
:103A2000E651F94F10822091DC0621110BC1FC01F7
:103A3000EA51F94F1082C6018651994F3C016EE45C
:103A400070E00E94D3BC0097F1F19093DB06809365
:103A5000DA06861997098C0D9D1D4AE050E060E05A
:103A600070E08551994F0E9420BB6093730870935A
:103A70007408809375089093760840906F08509072
:103A800070086090710870907208EFEF4E1A5E0A2D
:103A90006E0A7E0AC090E206D090E30664157505B2
:103AA0008605970509F4F4C0BC9CC001BD9C900D2F
:103AB000112466E075E08651994F0E9498BC892BCD
:103AC00009F0E6C074C16AE270E0C3010E94D3BC91
:103AD000892B09F443C0E9E2F6E08491882341F0A0
:103AE0009091C00095FFFCCF8093C6003196F5CF32
:103AF000E0E6F4E08491882341F09091C00095FFC6
:103B0000FCCF8093C6003196F5CF40916F0850915D
:103B1000700860917108709172082AE030E080E7C7
:103B200095E0FAD88091C00085FFFCCF8AE08093B1
:103B3000C6001092DE061092DD067CC280917308EA
:103B400090917408A0917508B091760880936F08E1
:103B500090937008A0937108B09372088091E20668
:103B60009091E306B89E6001B99ED00C1124C60165
:103B70008651994F3C0167E470E00E94D3BC0097E6
:103B800009F44BC09093DB068093DA0686199709F7
:103B90008C0D9D1D60E070E08551994F0E94B8B971
:103BA0000E94EFB56430710508F037C08091F505CB
:103BB00081111AC080910F0981112FC0F7018491E2
:103BC000EDE5F4E0882349F09091C00095FFFCCF2B
:103BD0008093C60031968491F5CF8091C00085FF17
:103BE000FCCFA092C60019C0F8018491E7EEF3E083
:103BF000882349F09091C00095FFFCCF8093C600C8
:103C000031968491F5CF8091C00085FFFCCFA092C2
:103C1000C6008DED93E00E940F868091E2069091A0
:103C2000E3060196BE010E943EB99093E30680939D
:103C3000E2068091E0069091E10601969093E106FC
:103C40008093E0061092DE061092DD06AACE8B333A
:103C500011F49092DC069091DC069111A2CE409175
:103C6000E2065091E306B9016F5F7F4F7093DE0665
:103C70006093DD06B49EF001B59EF00D1124E20FB5
:103C8000F31FE651F94F80838CCE1092DC06D2C12F
:103C9000BC9C3001BD9C700C1124C3018651994F0E
:103CA0002C016AE270E00E94D3BC009781F5E9E242
:103CB000F6E08491882341F09091C00095FFFCCFFD
:103CC0008093C6003196F5CFEAE8F4E0849188232A
:103CD00041F09091C00095FFFCCF8093C6003196D3
:103CE000F5CF40916F085091700860917108709104
:103CF00072082AE030E080E795E00ED88091C0009D
:103D000085FFFCCF8AE08093C60005DE12CF20E05D
:103D1000D12CF301E20FF11DE651F94F30813A3217
:103D200019F02F5FD326F5CF9093DB068093DA0648
:103D300084199509860D971D60E070E08551994FB3
:103D40000E94B8B90E94EFB52D2D30E02617370735
:103D500009F4F4CEE9E2F6E08491882341F09091F1
:103D6000C00095FFFCCF8093C6003196F5CFE4EB01
:103D7000F4E08491882341F09091C00095FFFCCF3E
:103D80008093C6003196F5CF40916F08509170082E
:103D900060917108709172082AE030E080E795E048
:103DA0000E948C168091C00085FFFCCFABCFE9E26A
:103DB000F6E08491882341F09091C00095FFFCCFFC
:103DC0008093C6003196F5CFE3EDF4E0849188232B
:103DD00041F09091C00095FFFCCF8093C6003196D2
:103DE000F5CF40916F085091700860917108709103
:103DF00072082AE030E080E795E00E948C168091FE
:103E0000C00085FFFCCF7ECF80911109882389F007
:103E10008091DD069091DE06892B59F490E6E92E1B
:103E2000FF24F394C4E0D0E005EC13E02AE0D22EA6
:103E3000AFC08091F608882309F4FCC08091F70890
:103E400087FDF8C080688093F70888ED93E0DF91E4
:103E5000CF911F910F91FF90EF90DF90CF90BF9087
:103E6000AF909F907F906F905F904F907CCA8091B1
:103E7000E0069091E10604970CF0DCC08091EB091C
:103E80009091EC09A091ED09B091EE098093060A9A
:103E90009093070AA093080AB093090A83EE99E069
:103EA0000E94F13B482F8093DF068A3019F04D3095
:103EB00009F085C04091060A5091070A6091080AEE
:103EC0007091090A8091FE099091FF09A091000A62
:103ED000B091010A481759076A077B0738F1F801C2
:103EE0008491E5ECF3E081117EC08091C00085FFF4
:103EF000FCCFD092C6008BEB93E00E940F86F0922D
:103F0000F0081092F3080E9470AE6093CA06709396
:103F1000CB068093CC069093CD068FE099E00E946B
:103F20007F4F61E08FE099E00E94C04D2091DD0657
:103F30003091DE062115310509F4A7CE8091E20605
:103F40009091E306E89EF001E99EF00D1124E20F46
:103F5000F31FE651F94F1082FC01EA51F94FF0824C
:103F60002091E0063091E1062F5F3F4F3093E1064C
:103F70002093E0060196BE010E943EB99093E306AD
:103F80008093E2061092DC061092DE061092DD06A7
:103F90004091060A5091070A6091080A7091090A37
:103FA0008091FE099091FF09A091000AB091010A49
:103FB000481759076A077B0708F03CC058CF4A33B7
:103FC00029F42091DC06222309F474CF2091DD0628
:103FD0003091DE062F3531050CF06CCF8F3FFFEFAF
:103FE0009F0751F467CF9091C00095FFFCCF80935D
:103FF000C6003196849177CF4B3311F4F092DC06F2
:104000004091DC064111C4CF4091E2065091E30695
:10401000B9016F5F7F4F7093DE066093DD06E49E0B
:10402000F001E59EF00D1124E20FF31FE651F94F68
:104030008083AECFDF91CF911F910F91FF90EF90D2
:10404000DF90CF90BF90AF909F907F906F905F90E8
:104050004F9008958F929F92AF92BF92CF92DF922E
:10406000EF92FF920F931F93CF93DF9369ECE62EAD
:1040700063E0F62E0AED18E0CBE8D8E07CEEC72E20
:1040800078E0D72EF70181917F0101DC882311F1BF
:10409000EADB4B015C01F6018081811103C0609174
:1040A0006A0801C061E070E080E090E00E9422B602
:1040B000F80120813181428153810E9455B89B01D2
:1040C000AC01C501B4010E94A7B4688379838A83D7
:1040D0009B8309C0F80180819181A281B38188838B
:1040E0009983AA83BB830C5F1F4F2496FFEFCF1ADF
:1040F000DF0A8DECE81683E0F80621F686E4C7DBDC
:104100008823D1F0B0DB6B017C0160937B08709356
:104110007C0880937D0890937E0820E030E0A90120
:104120000E9483B7181644F4C0920A02D0920B0280
:10413000E0920C02F0920D02DF91CF911F910F914E
:10414000FF90EF90DF90CF90BF90AF909F908F90B7
:10415000089580DF89E49BDB882351F084DB609342
:104160007F0870938008809381089093820808C02C
:1041700010927F0810928008109281081092820895
:104180008AE485DB882351F06EDB609383087093AB
:104190008408809385089093860808951092830878
:1041A0001092840810928508109286080895CF9284
:1041B000DF92EF92FF92CF93DF93EC01C090C208A1
:1041C000D090C308E090C408F090C508A7019601FC
:1041D000688179818A819B810E9480B587FF04C0B4
:1041E000C882D982EA82FB82C090C608D090C708F4
:1041F000E090C808F090C908A70196016C817D8104
:104200008E819F810E9480B587FF04C0CC82DD82B1
:10421000EE82FF82C090CA08D090CB08E090CC0814
:10422000F090CD08A7019601688579858A859B85E0
:104230000E9480B587FF04C0C886D986EA86FB86BF
:10424000C0901F02D0902002E0902102F090220244
:10425000A7019601688179818A819B810E9483B739
:10426000181624F4C882D982EA82FB82C090230205
:10427000D0902402E0902502F0902602A70196013A
:104280006C817D818E819F810E9483B7181624F4F2
:10429000CC82DD82EE82FF82C0902702D09028027D
:1042A000E0902902F0902A02A7019601688579859D
:1042B0008A859B850E9483B7181624F4C886D98600
:1042C000EA86FB86DF91CF91FF90EF90DF90CF9051
:1042D0000895CF92DF92EF92FF920F931F938BE896
:1042E00098E065DF0E9470AE6093D6067093D706A3
:1042F0008093D8069093D90620918B0830918C0832
:1043000040918D0850918E086091DA087091DB0819
:104310008091DC089091DD080E9480B5811179C000
:1043200020918F0830919008409191085091920807
:104330006091DE087091DF088091E0089091E108BB
:104340000E9480B5811165C020E030E040E752E472
:1043500060910A0270910B0280910C0290910D0203
:104360000E9487B5EDE9CE2EE8E0DE2E7B018C01C0
:1043700027E938E043E958E06FE878E08BE898E017
:104380000E94E55780918B0890918C08A0918D0830
:10439000B0918E088093DA089093DB08A093DC0834
:1043A000B093DD0880918F0890919008A0919108BA
:1043B000B09192088093DE089093DF08A093E00804
:1043C000B093E1088091930890919408A09195088A
:1043D000B09196088093E2089093E308A093E408D4
:1043E000B093E5088091970890919808A09199085A
:1043F000B0919A088093E6089093E708A093E808A4
:10440000B093E9081F910F91FF90EF90DF90CF904C
:10441000089560912D0270912E02882777FD809576
:10442000982F0E9422B620910A0230910B024091EF
:104430000C0250910D020E9455B820E030E040E798
:1044400052E40E9487B520E030E048EC52E488CF87
:10445000AF92BF92CF92DF92EF92FF920F931F9392
:10446000CF93DF93D82F2091830830918408409117
:1044700085085091860860917F087091800880912E
:104480008108909182080E9490B7C62F172F082F9D
:10449000F92E60912D0270912E02882777FD80956C
:1044A000982F0E9422B620910A0230910B0240916F
:1044B0000C0250910D020E9455B820E030E040E718
:1044C00052E40E9487B520E030E048EC52E40E94BC
:1044D00087B520919D082F93DF93FF920F931F9331
:1044E000CF935B016C01F2E0EF2E01E020E04FE79B
:1044F00058E06BE878E08AED98E00E94B64F809132
:104500008B0890918C08A0918D08B0918E088093B3
:10451000DA089093DB08A093DC08B093DD08809163
:104520008F0890919008A0919108B0919208809383
:10453000DE089093DF08A093E008B093E108809133
:10454000930890919408A0919508B0919608809353
:10455000E2089093E308A093E408B093E508809103
:10456000970890919808A0919908B0919A08809323
:10457000E6089093E708A093E808B093E9080E9442
:1045800070AE6093D6067093D7068093D80690934A
:10459000D9060F900F900F900F900F900F90DF9112
:1045A000CF911F910F91FF90EF90DF90CF90BF9030
:1045B000AF9008952091F408223111F41092F6087A
:1045C0008091F0088D30E1F480910D0990910E09F1
:1045D000843F31E0930709F42C98813D974020F007
:1045E00010920E0910920D0980910D0990910E09FB
:1045F000009709F42C9A019690930E0980930D0967
:104600008091F0088D7F813031F4223121F4809146
:10461000090981112C988091F608882331F1809145
:104620001109882321F12CB12295217030910301C9
:104630008091F50883709091F708813039F08330CC
:1046400081F4211105C030FD03C00BC0222349F0C5
:1046500091609093F7088091F008823041F40C94B7
:10466000838690789093F70808951092F70808953C
:10467000F8940E948E6F5F9A8A9A9FB7F8948091FF
:1046800008018160809308019FBF129A479A60E0F9
:104690008CE00E9450B0E9E2F6E08491882341F07A
:1046A0009091C00095FFFCCF8093C6003196F5CF66
:1046B000E1EFF1E08491882341F09091C00095FFF3
:1046C000FCCF8093C6003196F5CF8091C00085FF66
:1046D000FCCF8AE08093C60088EE91E00E94948629
:1046E000FFCFCF92DF92EF92FF920F931F930E9422
:1046F00070AE0091D2061091D3062091D40630916D
:10470000D506C090D606D090D706E090D806F09097
:10471000D9066C197D098E099F0906171707280706
:10472000390728F4012B022B032B09F0A1DF80911C
:10473000060290910702A0910802B0910902892B0C
:104740008A2B8B2BC9F18091F0088730D1F40E941D
:1047500070AE0091D6061091D7062091D806309100
:10476000D906601B710B820B930B653C7940810568
:10477000910510F19091230C8091220C98131CC08C
:1047800027C00E9470AE0091D6061091D7062091E6
:10479000D8063091D906601B710B820B930B0091E8
:1047A00006021091070220910802309109020617B3
:1047B00017072807390780F08091060182FFB6CFDE
:1047C0001F910F91FF90EF90DF90CF900C94C857FE
:1047D00081E08093C906F0CF9091230C8091220C48
:1047E0009813EACF5F9A8A9A9FB7F894809108014C
:1047F0008160809308019FBF129A479ADDCFCF93C3
:10480000DF93EC0180919D088093F60584E53FD805
:10481000811102C080E064C026D80E94F4B5609384
:10482000F6056230B8F3E3E2F6E08491882341F0C4
:104830009091C00095FFFCCF8093C6003196F5CFD4
:10484000C936D10599F034F4C836D105C9F5EEE082
:10485000F3E015C0CD36D10531F0CA3DD10581F563
:10486000E9ECF2E02AC0E0EEF2E01DC0E7EFF2E092
:1048700010C09091C00095FFFCCF8093C60081913D
:104880008111F7CF1DC09091C00095FFFCCF8093A0
:10489000C60081918111F7CF13C09091C00095FFA0
:1048A000FCCF8093C60081918111F7CF09C0909110
:1048B000C00095FFFCCF8093C60081918111F7CF96
:1048C00040E050E06091F60580E795E00E94E61632
:1048D0008091C00085FFFCCF8AE08093C60081E014
:1048E000DF91CF9108953F924F925F926F927F92A6
:1048F0008F929F92AF92BF92CF92DF92EF92FF92F0
:104900000F931F93CF93DF93CDB7DEB7A2970FB668
:10491000F894DEBF0FBECDBF87E40E94471C8823FA
:1049200009F49CC30E94331C0E94EFB56A357105DF
:1049300009F4A2C2ACF46230710509F4B8C024F4E1
:1049400077FFADC00C94E2346430710509F4BFC048
:104950000CF4B4C06C31710509F400C10C94E2345C
:104960006636710509F43DC30CF051C06C35710514
:1049700009F48BC20CF484C26536710511F00C94F5
:10498000E2348EEA93E00E94B319609106097091B7
:10499000070980910A0990910B09680F791F6253EA
:1049A0007109882777FD8095982F0E9422B6609321
:1049B000E2087093E3088093E4089093E508198275
:1049C00020E030E040EA50E4609137027091380214
:1049D0008091390290913A020E9487B5FE0131968A
:1049E0006F017B018C0126EE38E042EE58E06EED5F
:1049F00078E08AED98E00E94E5570E94616A8DE0B8
:104A00008093F0088EE080930C090C94E2346234B9
:104A100021E0720709F4EAC2683E33E0730709F443
:104A20007FC26134714011F00C94E23420E030E038
:104A300040E251E46091E2087091E3088091E4085B
:104A40009091E5080E94A7B46093E2087093E30890
:104A50008093E4089093E508198220E030E040EA72
:104A600050E4609137027091380280913902909140
:104A70003A020E9487B59E012F5F3F4F69017B017B
:104A80008C0126EE38E042EE58E06EED78E08AEDDB
:104A900098E00E94E5570E94616A0C94E23480918C
:104AA000F505811104C0D6DA14DC0C9476368091B9
:104AB000F505811103C04DDB81E006C08091F5054D
:104AC000811105C046DB80E0C3DC0C94763682EBB6
:104AD00093E00E940F8680E50E94471C882339F0EE
:104AE0000E94331C0E94F4B54B015C0103C0812C71
:104AF000912C540183E50E94471C882361F00E9499
:104B0000331C20E030E04AE754E40E9455B80E948C
:104B1000F4B54B015C010E94616A0E9470AE6B01AA
:104B20007C01C80CD91CEA1CFB1C0E9470AE60936F
:104B3000D6067093D7068093D8069093D9060E9424
:104B400070AE6C157D058E059F0510F00C94E23457
:104B50000E949D6CC6DD0E941C87F1CF80910A02E5
:104B600090910B02A0910C02B0910D0280937708F6
:104B700090937808A0937908B0937A0880912D02D9
:104B800090912E029093EB088093EA0884E690E0DF
:104B900090932E0280932D020E9470AE6093D606F1
:104BA0007093D7068093D8069093D90681E00E942F
:104BB00031638091DA089091DB08A091DC08B09114
:104BC000DD0880938B0890938C08A0938D08B09398
:104BD0008E088091DE089091DF08A091E008B091E6
:104BE000E10880938F0890939008A0939108B09368
:104BF00092088091E2089091E308A091E408B091B6
:104C0000E5088093930890939408A0939508B09337
:104C100096088091E6089091E708A091E808B09185
:104C2000E9088093970890939808A0939908B09307
:104C30009A0810920A0210920B0210920C02109223
:104C40000D0288E50E94471C882311F090E00AC0FD
:104C500089E50E94471C8111F9CF8AE50E94471C13
:104C600091E0982790930E02992309F44BC020E01D
:104C700030E0A9016091DA087091DB088091DC08CE
:104C80009091DD080E9480B581113CC080E090E0E9
:104C9000A0EAB0E48093DA089093DB08A093DC08E4
:104CA000B093DD0860912F02709130028091310243
:104CB0009091320260930A0270930B0280930C026F
:104CC00090930D0220E030E040E752E40E9487B567
:104CD0000DE9C02E08E0D02E7B018C0126EE38E0D5
:104CE00042EE58E06EED78E08AED98E00E94E557DC
:104CF0000E94616A1092DA081092DB081092DC08B8
:104D00001092DD0880910E0281110C94E53489E542
:104D10000E94471C81110C94E53480910E02811190
:104D20000C94EB3488E50E94471C81110C94EB3401
:104D300080910E0281110C94F1348AE50E94471C87
:104D400081110C94F13488E50E94471C8823D1F02E
:104D50000E943C1C672B682B692BA1F00E94331C1E
:104D60002091CE083091CF084091D0085091D108C1
:104D70000E94A7B46093DA087093DB088093DC0884
:104D80009093DD0889E50E94471C8823D1F00E949A
:104D90003C1C672B682B692BA1F00E94331C2091CF
:104DA000D2083091D3084091D4085091D5080E9480
:104DB000A7B46093DE087093DF088093E0089093B7
:104DC000E1088AE50E94471C8823D1F00E943C1C20
:104DD000672B682B692BA1F00E94331C2091D60809
:104DE0003091D7084091D8085091D9080E94A7B4B3
:104DF0006093E2087093E3088093E4089093E508D9
:104E000026EE38E042EE58E06EED78E08AED98E06C
:104E10000E947C6180E00E943163809177089091CC
:104E20007808A0917908B0917A0880930A0290934B
:104E30000B02A0930C02B0930D028091EA089091AE
:104E4000EB0890932E0280932D020E9470AE609327
:104E5000D6067093D7068093D8069093D9060E9401
:104E60002A638091F008853011F00C94E23486E0DA
:104E70008093F0080C94E23410926A080C94E234A7
:104E800081E080936A080C94E23485E40E94471C18
:104E9000811102C00E94616AB9ECCB2EB3E0DB2E17
:104EA0001EECE12E18E0F12E0AED18E0B12CD6012F
:104EB0008D916D010E94471C882339F1B3E0BB122C
:104EC0000CC00E94331CF80160837183828393833A
:104ED00086EE98E00E94216218C00E94331CD70120
:104EE0002D913D914D915C910E94A7B4F801608392
:104EF00071838283938326EE38E042EE58E06EEDB4
:104F000078E08AED98E00E947C61B394F4E0EF0EC3
:104F1000F11C0C5F1F4F24E0B212C9CF0C94E23495
:104F20008FE080930C091092DA081092DB0810923F
:104F3000DC081092DD0826EE38E042EE58E06EED17
:104F400078E08AED98E00E947C611092DE08109271
:104F5000DF081092E0081092E10826EE38E042EEF9
:104F600058E06EED78E08AED98E00E947C616091F7
:104F700006097091070980910A0990910B09680F41
:104F8000791F882777FD8095982F0E9422B660931D
:104F9000E2087093E3088093E4089093E50819828F
:104FA00020E030E040EA50E460913702709138022E
:104FB0008091390290913A020E9487B5DE011196E4
:104FC0006D017B018C0126EE38E042EE58E06EED7B
:104FD00078E08AED98E00E94E5570E94616A0C949F
:104FE000E23481E0809308090C94E23420E030E060
:104FF00040E251E46091E2087091E3088091E40896
:105000009091E5080E94A6B46093E2087093E308CB
:105010008093E4089093E508198220E030E040EAAC
:1050200050E460913702709138028091390290917A
:105030003A020E9487B5DE0111966D017B018C0159
:1050400026EE38E042EE58E06EED78E08AED98E02A
:105050000E94E5570E94616A0C94E2348DE40E943C
:10506000471C882311F40C948C330E94331C0E943B
:10507000EFB56A36710509F4D9C50CF0A1C06B31E2
:10508000710509F417C20CF051C06431710509F4BF
:10509000B1C1FCF46330710509F492C134F462309B
:1050A000710508F433C10C94E2346131710509F4DF
:1050B0008FC16231710509F4F9C56530710511F0D0
:1050C0000C94E2340E94616A2C98109209090C94A5
:1050D000E2346731710509F4C1C17CF465317105B1
:1050E00009F4B6C16631710511F00C94E2348FE019
:1050F00099E00E94CA490C94E2346931710509F4BF
:10510000C5C10CF0C9C18FE099E00E94CE490E9450
:1051100070AE6093CE067093CF068093D0069093C6
:10512000D10682E08093F0080C94E2346235710578
:1051300009F4B5C5DCF46F31710509F468C254F4A3
:105140006C31710509F4BCC16E31710509F4EDC112
:105150000C94E2346035710509F49BC50CF09CC5D4
:105160006A32710509F4DAC20C94E23465357105CE
:1051700009F4D1C554F46335710509F493C5643558
:10518000710509F493C50C94E2346836710509F48D
:10519000F0C20CF01CC36C35710511F00C94E234B4
:1051A00029EC33E038A32F8F05E511E135E6832E96
:1051B00031E1932E49E1A42E41E1B42E312C22C6D7
:1051C0006D3C710511F40C94FF300CF045C068374C
:1051D000710509F434C7FCF46237710509F450C64F
:1051E00054F46B36710509F44FC56D36710509F439
:1051F000DCC30C94E2346537710509F420C66737C7
:10520000710509F480C06337710511F00C94E23424
:10521000E5E7F2E010C66E3B710509F445C454F4AD
:105220006937710509F40FC76C38710509F4BEC2FE
:105230000C94E2346B3C710509F4A5C70CF0BFC7B0
:10524000693C710511F00C94E23409EC13E025E49B
:10525000E22E21E1F22E7DC76E32B1E07B0711F420
:105260000C94263314F56C3D710511F40C94143232
:1052700064F46E3C710511F40C945D316A3D710566
:1052800011F40C9479310C94E2346C32F1E07F0724
:1052900011F40C94323214F00C9460326D3D7105AF
:1052A00011F40C9423320C94E234653F31E073071F
:1052B00011F40C9472339CF4603991E0790711F485
:1052C0000C946C33643FA1E07A0711F40C946F33B3
:1052D0006F32714011F00C94E2340C943433603A24
:1052E000E3E07E0709F45FC1673EF3E07F0711F456
:1052F0000C947533663F714011F00C94E2340E94B7
:10530000E7120C94E234E4E3F3E0A7C68DE993E0FE
:105310000E940F8680E50E94471C882339F00E9476
:10532000331C0E94F4B56B017C0103C0C12CD12C4D
:10533000760183E50E94471C882361F00E94331C9C
:1053400020E030E04AE754E40E9455B80E94F4B5EA
:105350006B017C010E94616A0E9470AE6093D60668
:105360007093D7068093D8069093D906C114D104C0
:10537000E104F104A9F00E9470AE4B015C018C0CB9
:105380009D1CAE1CBF1C0E9470AE681579058A0575
:105390009B0580F40E94228881110CC00C94F73484
:1053A0000E942288811106C00E949D6C9AD90E9499
:1053B0001C87F6CF80E993E00E940F860C94E234BC
:1053C0000E94616A2C9A81E0809309090C94E2346E
:1053D00087E893E00E940F865F988A989FB7F894B9
:1053E000809108018E7F809308019FBF1298479893
:1053F0000C94E234E7E7F3E08491882341F0909144
:10540000C00095FFFCCF8093C6003196F5CF809108
:10541000C00085FFFCCF8AE08093C6008FE099E052
:105420000E94B048E9E6F3E08491882341F090912E
:10543000C00095FFFCCF8093C6003196F5CF8091D8
:10544000C00085FFFCCF8AE08093C6000C94E23454
:105450008FE099E00E9407490C94E2340091DA064B
:105460001091DB060C5F1F4F6AE270E0C8010E94DA
:10547000D3BC009719F0FC013197108241E0B801CC
:105480008FE099E00E94DA490C94E2348FE099E0D1
:105490000E94D5490C94E23480911209882311F4BA
:1054A0000C94E23483E50E94471C81110C94FF3474
:1054B0000C94E2348FE099E00E94FB4C0C94E234AF
:1054C0008091DA069091DB066AE270E004960E9411
:1054D000D3BC8C010097E1F02091E4063091E50601
:1054E00040E6429FC001439F900D11246EE470E09E
:1054F0008651994F0E94D3BC60E270E00E94D3BCF9
:1055000001969093DB068093DA06F80131971082BA
:105510006091DA067091DB066C5F7F4F40E08FE0B0
:1055200099E00E94DA490C94E234809112098823B0
:1055300011F40C94E2348FE099E00E94B44E809113
:10554000DA069091DB066AE270E004960E94D3BC12
:105550008C010097E1F02091E4063091E50640E6E9
:10556000429FC001439F900D11246EE470E086516C
:10557000994F0E94D3BC60E270E00E94D3BC0196B8
:105580009093DB068093DA06F801319710826091E0
:10559000DA067091DB066C5F7F4F8FE099E00E9426
:1055A000C24B0C94E2348091DA069091DB066AE2F9
:1055B00070E005960E94D3BC8C010097E1F0209129
:1055C000E4063091E50640E6429FC001439F900DFE
:1055D00011246EE470E08651994F0E94D3BC60E2C2
:1055E00070E00E94D3BC01969093DB068093DA06AC
:1055F000F801319710826091DA067091DB066B5FDB
:105600007F4F8FE099E00E94BD4B0C94E2340E94E2
:1056100070AE6093CA067093CB068093CC069093CD
:10562000CD060091CE061091CF062091D006309184
:10563000D106601B710B820B930B28EE33E040E028
:1056400050E00E9451B9CA01B9012CE330E040E0BA
:1056500050E00E9451B97F936F933F932F938AE557
:1056600093E09F938F93CE0101969F938F930E9417
:105670007ABDE3E2F6E084910FB6F894DEBF0FBE88
:10568000CDBF882349F09091C00095FFFCCF809357
:10569000C60031968491F5CFFE0131968191882321
:1056A00039F09091C00095FFFCCF8093C600F6CFF3
:1056B0008091C00085FFFCCF8AE08093C600CE01B8
:1056C00001960E9400868091F410882311F40C94B6
:1056D000E2341092F41000919D0810E0000F111FA9
:1056E000045C1D4EF80160817181882777FD8095EB
:1056F000982F0E9422B62091470230914802409193
:10570000490250914A020E9483B7181614F00C9473
:10571000E234D8011D921C920C94E23483E50E947D
:10572000471C882311F40C94E2340E94331C6B0153
:105730007C0180E50E94471C882351F0C701B60117
:105740000E94EFB56F3F710509F010F40C940F350E
:105750006DE070E020E0E22FEE0FFF0BE757FC4F0B
:10576000808191818617970711F40C94E2342F5FA2
:10577000F2CF88E690E043D881110C94E23483E5BF
:105780000E94471C882371F00091F6050E94331C8B
:1057900010E0000F111F045C1D4E0E94EFB5F801D0
:1057A000718360830E948D6F0C94E23483E50E94C4
:1057B000471C882311F40C94E2340E94331C0E948D
:1057C000EFB570933B1260933A120C94E23489E681
:1057D00090E015D881110C94E234E3E5F3E0849174
:1057E000882341F09091C00095FFFCCF8093C600C4
:1057F0003196F5CF40912E1250912F1260913012B8
:105800007091311221E030E080E795E00E94851729
:10581000E0E5F3E08491882341F09091C00095FF8A
:10582000FCCF8093C6003196F5CF60913C12709109
:105830003D12882777FD8095982F0E9422B6AB01F4
:10584000BC0121E030E080E795E00E948517EBE4A1
:10585000F3E08491882341F09091C00095FFFCCF44
:105860008093C6003196F5CF409132125091331299
:10587000609134127091351221E030E080E795E0BC
:105880000E948517E8E4F3E08491882341F0909129
:10589000C00095FFFCCF8093C6003196F5CF609194
:1058A0003E1270913F12882777FD8095982F0E94B5
:1058B00022B6AB01BC0121E030E080E795E00E9418
:1058C0008517E4E4F3E08491882341F09091C000CF
:1058D00095FFFCCF8093C6003196F5CF40912812FA
:1058E0005091291260912A1270912B1221E030E020
:1058F00080E795E00E948517E1E4F3E08491882336
:1059000041F09091C00095FFFCCF8093C600319686
:10591000F5CF60913A1270913B12882777FD809500
:10592000982F0E9422B6AB01BC0121E030E080E755
:1059300095E00E948517EDE3F3E08491882341F020
:105940009091C00095FFFCCF8093C6003196F5CFB3
:105950008091F60590E00E94926C4AE050E0BC0114
:1059600080E795E00E94AF16E8E3F3E08491882396
:1059700041F09091C00095FFFCCF8093C600319616
:10598000F5CF8FEF9FEF0E94926C4AE050E0BC0190
:1059900080E795E00E94AF168091C00085FFFCCFA4
:1059A0008AE08093C6000C9476368DE690E00E94E3
:1059B000FF2381110C94E2348DE293E00E940F8664
:1059C0001092F41083E50E94471C882371F0009127
:1059D000F6050E94331C10E0000F111F045C1D4EE1
:1059E0000E94EFB5D8016D937C9383E50E94471C1C
:1059F000882351F00E94331C609347027093480241
:105A00008093490290934A0282E40E94471C8823B3
:105A100051F00E94331C60934B0270934C028093B0
:105A20004D0290934E0286E40E94471C882369F041
:105A30000E94331C6093430270934402809345029A
:105A40009093460281E08093F4100E948D6F0E9433
:105A500070AE4B015C010091F60510E0F801EE0F0D
:105A6000FF1FE45CFD4E60817181882777FD809582
:105A7000982F0E9422B62B013C01F801EE0FFF1F68
:105A8000EE0FFF1FE25DFD4E80819181A281B38107
:105A90008F8F98A3A9A3BAA3CC24CA94DC2C760137
:105AA0006AE0362E0C947A358091F90881118AC704
:105AB00085E093E00E940F8683E50E94471C8823BF
:105AC00041F00E94331C0E94EFB570933B1260932B
:105AD0003A120E9470AE4B015C0101E013E05CEFF2
:105AE000E52E52E0F52E68EFC62E62E0D62E7AE063
:105AF000772E60913A1270913B12882777FD80953E
:105B0000982F0E9422B6209128123091291240919C
:105B10002A1250912B120E9483B718160CF077C0EE
:105B20000E9470AE681979098A099B09693E734021
:105B30008105910508F461C0F8018491E1E0F3E08A
:105B4000882349F09091C00095FFFCCF8093C60058
:105B500031968491F5CF40912E1250912F12609181
:105B600030127091311222E030E080E795E00E941F
:105B70008517F7018491ECEFF2E0882349F09091CA
:105B8000C00095FFFCCF8093C60031968491F5CF7D
:105B9000409132125091331260913412709135124B
:105BA00022E030E080E795E00E948517F6018491BD
:105BB000E8EFF2E0882349F09091C00095FFFCCF18
:105BC0008093C60031968491F5CF40912812509170
:105BD000291260912A1270912B1221E030E080E7A7
:105BE00095E00E9485178091C00085FFFCCF7092E0
:105BF000C6000E9470AE4B015C010E949D6C0E9429
:105C000071230E941C878091FB08811172CF8EEE58
:105C100092E00E940F860E9470AE6093D606709349
:105C2000D7068093D8069093D906CCC683E50E9408
:105C3000471C882311F10E94331C20E030E0A901A9
:105C40000E9480B587FD0FC00E94331C20E030E029
:105C50004FE753E40E9483B7181644F00E94331CA8
:105C60000E94EFB505C060E070E002C06FEF70E029
:105C700070939C0860939B08A5C68FEF90E090936B
:105C80009C0880939B089EC610929C0810929B08CB
:105C900099C6269A2E9896C6269A2E9A93C6109240
:105CA000EF0890C681E08093EF088CC683E50E94E0
:105CB000471C882399F00E94331C20E030E04AE71B
:105CC00054E40E9455B80E94F4B5609306027093A4
:105CD000070280930802909309021AC088E50E9487
:105CE000471C8111E1C789E50E94471C8111DCC76F
:105CF0008AE50E94471C8111D7C785E40E94471C92
:105D00008111D2C70E94616A129A479A0E94C96A99
:105D10001092F30857C683E50E94471C0E94331C6B
:105D200020E030E04AE754E40E9455B80E94F4B500
:105D30006093D2067093D3068093D4069093D506D1
:105D400041C6B3E03B1268C00E94331C6B017C016A
:105D500020E030E040EA51E40E9480B587FF3FC078
:105D6000A7019601F80160817181828193810E946F
:105D700087B52B013C019B01AC0160912D11709105
:105D80002E1180912F11909130110E9455B860937F
:105D90002D1170932E1180932F1190933011A30128
:105DA0009201D4016D917D918D919C910E9455B885
:105DB000F4016083718382839383D5016D917D911A
:105DC0008D919C910E9420B6A30192010E9455B82A
:105DD0000E94F4B5F5016083718382839383D801B7
:105DE000CD92DD92ED92FC92139733940C5F1F4F8E
:105DF000F4E08F0E911C24E0A20EB11C34E03316A7
:105E000009F4E0C5AF8DB8A18D91B8A3AF8F0E9402
:105E1000471C882351F395CF0E94331CF8016083FF
:105E2000718382839383E1CF9091C00095FFFCCF73
:105E30008093C600319684918111F6CFC3C500913D
:105E4000DA061091DB060B5F1F4F6AE270E0C801B3
:105E50000E94D3BC009719F0FC0131971082C80151
:105E60000E9400860E9470AE6093CE067093CF06AB
:105E70008093D0069093D10681E08093F308A2C569
:105E8000E2E7F2E08491882341F09091C00095FF11
:105E9000FCCF8093C6003196F5CF4091DA0850913F
:105EA000DB086091DC087091DD0822E030E080E7DB
:105EB00095E00E948517EFE6F2E08491882341F097
:105EC0009091C00095FFFCCF8093C6003196F5CF2E
:105ED0004091DE085091DF086091E0087091E10880
:105EE00022E030E080E795E00E948517ECE6F2E0E2
:105EF0008491882341F09091C00095FFFCCF80935E
:105F0000C6003196F5CF4091E2085091E3086091C8
:105F1000E4087091E50822E030E080E795E00E9417
:105F20008517E9E6F2E08491882341F09091C00062
:105F300095FFFCCF8093C6003196F5CF4091E608DF
:105F40005091E7086091E8087091E90822E030E09C
:105F500080E795E00E948517EFE5F2E084918823C1
:105F600041F09091C00095FFFCCF8093C600319620
:105F7000F5CF0E94BB6A0E9422B620915511309144
:105F8000561140915711509158110E9487B5AB019D
:105F9000BC0122E030E080E795E00E948517ECE547
:105FA000F2E08491882341F09091C00095FFFCCFEE
:105FB0008093C6003196F5CF81E00E94BB6A0E94B3
:105FC00022B62091591130915A1140915B11509194
:105FD0005C110E9487B5AB01BC0122E030E080E794
:105FE00095E00E948517E9E5F2E08491882341F06D
:105FF0009091C00095FFFCCF8093C6003196F5CFFD
:1060000082E00E94BB6A0E9422B620915D1130910D
:106010005E1140915F11509160110E9487B5AB01F4
:10602000BC0122E030E080E795E00E948517809176
:10603000C00085FFFCCF8AE08093C600C3C480E027
:106040000E943163BFC481E00E943163BBC4909160
:10605000C00095FFFCCF8093C60081918111F7CFDE
:106060008091C00085FFFCCF8AE08093C600E1E507
:10607000F2E08491882341F09091C00095FFFCCF1D
:106080008093C6003196F5CF659903C0E5E2F3E051
:1060900009C0EFE2F3E006C09091C00095FFFCCF8D
:1060A0008093C60081918111F7CF8091C00085FF58
:1060B000FCCF8AE08093C600E9E4F2E08491882373
:1060C00041F09091C00095FFFCCF8093C6003196BF
:1060D000F5CF8091030181FD03C0E5E2F3E009C043
:1060E000EFE2F3E006C09091C00095FFFCCF8093F3
:1060F000C60081918111F7CF8091C00085FFFCCF50
:106100008AE08093C600E1E4F2E08491882341F0C4
:106110009091C00095FFFCCF8093C6003196F5CFDB
:106120004B9903C0E5E2F3E009C0EFE2F3E006C0FB
:106130009091C00095FFFCCF8093C60081918111A2
:10614000F7CF8091C00085FFFCCF8AE08093C60026
:1061500039C4D8018D918D010E94471C882349F0D4
:106160000E94331C0E94F4B5F7016083718382831F
:106170009383F4E0EF0EF11C23E00D3C120749F786
:106180000E9447621FC409EC13E095E6E92E91E1F5
:10619000F92ED8018D918D010E94471C882339F07A
:1061A0000E94331CF7016083718382839383F4E040
:1061B000EF0EF11C23E00D3C120759F703C483E5F1
:1061C0000E94471C882351F00E94331C60933D11AC
:1061D00070933E1180933F119093401184E50E948B
:1061E000471C882309F4EEC30E94331C60933911C5
:1061F00070933A1180933B1190933C11E3C383E574
:106200000E94471C882351F00E94331C6093411167
:1062100070934211809343119093441184E50E943E
:10622000471C882351F00E94331C609329117093FE
:106230002A1180932B1190932C1182E40E94471C09
:10624000882361F00E94331C0E94F4B5609375119D
:1062500070937611809377119093781188E50E945E
:10626000471C882351F00E94331C609335117093B2
:10627000361180933711909338118AE50E94471C9C
:10628000882351F00E94331C6093311170933211B6
:10629000809333119093341185E40E94471C882326
:1062A00009F490C30E94331C60932D1170932E113A
:1062B00080932F119093301185C309EC13E08EEC7D
:1062C000E82E88E0F82ED8018D918D010E94471CA0
:1062D000882339F00E94331CF70160837183828325
:1062E0009383F4E0EF0EF11C23E00C3C120759F706
:1062F00069C38AED90E00E94FF23811163C388E5A2
:106300000E94471C882381F00091F60510E00E944E
:10631000331CF801EE0FFF1FEE0FFF1FE15FFD4F73
:10632000608371838283938389E50E94471C88235D
:1063300081F00091F60510E00E94331CF801EE0F89
:10634000FF1FEE0FFF1FE95EFD4F608371838283A5
:106350009383E3E2F6E08491882341F09091C000BA
:1063600095FFFCCF8093C6003196F5CFE1E3F2E0D4
:106370008491882341F09091C00095FFFCCF8093D9
:10638000C6003196F5CF1092F6058091F605823061
:1063900008F042C0EBEBF4E08191882339F0909152
:1063A000C00095FFFCCF8093C600F6CFE091F605C4
:1063B00034E0E39FF0011124E15FFD4F4081518102
:1063C0006281738122E030E080E795E00E948517CA
:1063D000EFE4F3E08191882339F09091C00095FFBC
:1063E000FCCF8093C600F6CFE091F60584E0E89FED
:1063F000F0011124E95EFD4F40815181628173817A
:1064000022E030E080E795E00E9485178091F60554
:106410008F5F8093F605B9CF8091C00085FFFCCFD8
:106420008AE08093C600CEC283E50E94471C882381
:1064300009F4C8C20E94331C0E94EFB570932E026B
:1064400060932D02BFC283E50E94471C882309F494
:10645000B9C20E94331C0E94EFB570932C02609366
:106460002B02B0C283E50E94471C882331F00E94B2
:10647000331C0E94EFB58B0102C000E911E080E5FA
:106480000E94471C882331F00E94331C0E94EFB504
:106490007B0104C058EEE52E53E0F52E20E030E0FD
:1064A000A901B80185E20E9404B1B701882777FDF0
:1064B0008095982F0E949FAE85E20E9425B482C2EB
:1064C00080E50E94471C882351F00E94331C609392
:1064D000690270936A0280936B0290936C0289E464
:1064E0000E94471C882361F00E94331C0E947D7526
:1064F00060936502709366028093670290936802CE
:1065000084E40E94471C882361F00E94331C0E948F
:106510008975609361027093620280936302909325
:10652000640283E40E94471C882351F00E94331CBC
:1065300060935D0270935E0280935F0290936002AD
:106540000E94736CE1E5F3E08191882339F090912A
:10655000C00095FFFCCF8093C600F6CFE4E5F3E0E2
:106560008191882339F09091C00095FFFCCF8093F2
:10657000C600F6CF4091690250916A0260916B02A9
:1065800070916C0222E030E080E795E00E94851770
:10659000E8E5F3E08191882339F09091C00095FF00
:1065A000FCCF8093C600F6CF6091650270916602C1
:1065B00080916702909168020E948375AB01BC01D3
:1065C00022E030E080E795E00E948517ECE5F3E0FB
:1065D0008191882339F09091C00095FFFCCF809382
:1065E000C600F6CF609161027091620280916302F1
:1065F000909164020E948F75AB01BC0122E030E0F3
:1066000080E795E00E948517E0E6F3E0819188231A
:1066100039F09091C00095FFFCCF8093C600F6CF73
:1066200040915D0250915E0260915F027091600244
:1066300022E030E080E795E00E9485178091C0005D
:1066400085FFFCCF8AE08093C600BCC183E50E9431
:10665000471C882319F00E94331C03C060E070E0DF
:10666000CB010E943E62AEC185E40E94471C882394
:1066700041F00E94331C0E94EFB58B0177FD0AC0E8
:1066800002C000E010E0C12CD12C46E1E42E43E42E
:10669000F42E06C0C12CD12C3CE8E32E32E4F32EBC
:1066A00083E50E94471C882321F00E94331C6B0164
:1066B0007C0183E40E94471C882331F00E94331C34
:1066C0000E94EFB59B0102C025E030E0A801C701A0
:1066D000B6010E94B46F76C10E94616A73C10E94C4
:1066E000EF1170C10E946D146DC11092F5050E94EA
:1066F0009A8680916B0890916C08A0916D08B0917A
:106700006E0880936F0890937008A0937108B093FF
:1067100072080E948B1C56C184E50E94471C882386
:1067200009F40CC10E94331C0E94F4B56093F60575
:106730006230A8F1E3E2F6E08491882341F0909181
:10674000C00095FFFCCF8093C6003196F5CFE4E6FC
:10675000F3E08191882339F09091C00095FFFCCF40
:106760008093C600F6CF40E050E06091F60580E7E8
:1067700095E00E94E616E6E6F3E08191882339F081
:106780009091C00095FFFCCF8093C600F6CF80911A
:10679000C00085FFFCCF8AE08093C60013C186E469
:1067A0000E94471C8823E1F00E94331C6B017C018E
:1067B00060937B0870937C0880937D0890937E089B
:1067C00020E030E0A9010E9483B718165CF4C09263
:1067D0000A02D0920B02E0920C02F0920D0202C06B
:1067E000D12C02C0DD24D394C090F605E0909D0822
:1067F000CE1409F479C080E1EAEDF8E0ABE8B8E046
:1068000001900D928A95E1F78091F308882309F4AD
:1068100057C0F12C0C2D10E0F701EE0FFF1FEE0F0B
:10682000FF1FE15FFD4F20813181428153816091E3
:10683000DA087091DB088091DC089091DD080E94F5
:10684000A6B4F801EE0FFF1FEE0FFF1FE15FFD4F33
:1068500020813181428153810E94A7B46093DA087C
:106860007093DB088093DC089093DD08F701EE0F4E
:10687000FF1FEE0FFF1FE95EFD4F20813181428136
:1068800053816091DE087091DF088091E00890915B
:10689000E1080E94A6B4F801EE0FFF1FEE0FFF1FE4
:1068A000E95EFD4F20813181428153810E94A7B46E
:1068B0006093DE087093DF088093E0089093E1080E
:1068C000C0929D0826EE38E042EE58E06EED78E08A
:1068D0008AED98E00E947C61DD2031F08091F50521
:1068E000811102C00E946921E3E2F6E084918823CD
:1068F00041F09091C00095FFFCCF8093C600319687
:10690000F5CFE7E7F3E08191882339F09091C0005B
:1069100095FFFCCF8093C600F6CF60919D0870E094
:106920004AE050E080E795E00E94AF168091C000F9
:1069300085FFFCCF8AE08093C60044C0E3E2F6E026
:106940008491882341F09091C00095FFFCCF809303
:10695000C6003196F5CFEEE1F2E08491882341F054
:106960009091C00095FFFCCF8093C6003196F5CF83
:106970008091E4069091E50620E6289FF001299F8A
:10698000F00D1124E651F94F8191882339F090914F
:10699000C00095FFFCCF8093C600F6CFECE1F2E09B
:1069A0008491882341F09091C00095FFFCCF8093A3
:1069B000C6003196F5CF8091C00085FFFCCF8AE0FC
:1069C0008093C6000E94631C91C181E090E00E9408
:1069D00086170C948D2680E090E00E9486170C9418
:1069E000982682E090E00E9486170C94A3260E94CD
:1069F0009D6C0E9471230E941C870C94C3290E94E5
:106A00003C1CAB01BC014093060A5093070A6093FB
:106A1000080A7093090A83EE99E0ACD7D3CF0E949D
:106A2000331C0E94EFB50C94AA2B0E9470AE8B0110
:106A30009C01C701B6016053784F8F4F9F4F601B79
:106A4000710B820B930B28EE33E040E050E00E9484
:106A500051B9BA01A9012AE030E080E795E00E942F
:106A6000DB168091C00085FFFCCF3092C6000E94EB
:106A700070AE4B015C010E949D6C0E9471230E94CC
:106A80001C87FFEFCF16DF06EF06FF0609F0ACC04C
:106A90002F8D38A149A15AA1C301B2010E9483B729
:106AA000E091F605F0E08F01000F111F000F111F9C
:106AB000025D1D4EEE0FFF1FE45CFD4E6081718193
:106AC00018160CF079C0882777FD8095982F0E94C2
:106AD00022B620E030E040EA50E40E94A6B49B01D8
:106AE000AC01D8016D917D918D919C910E9483B7ED
:106AF00087FFB6C00E9470AE681979098A099B09A0
:106B0000693E73408105910508F4B5CFE9E2F3E0F1
:106B10008491882341F09091C00095FFFCCF809331
:106B2000C6003196F5CF40912E1250912F126091F0
:106B300030127091311222E030E080E795E00E943F
:106B40008517E4E2F3E08491882341F09091C0003E
:106B500095FFFCCF8093C6003196F5CF409132125D
:106B600050913312609134127091351222E030E06E
:106B700080E795E00E948517E0E2F3E084918823A6
:106B800041F09091C00095FFFCCF8093C6003196F4
:106B9000F5CFF7FE4ACFEDE4F3E006C09091C000D8
:106BA00095FFFCCF8093C60081918111F7CF809132
:106BB000C00085FFFCCF59CF882777FD8095982F9F
:106BC0000E9422B620E030E040EA50E40E94A7B4E0
:106BD0009B01AC01F80160817181828193810E94E7
:106BE00080B51816ECF586CFF7FC2FC0E091F605BE
:106BF000F0E08F01000F111F000F111F025D1D4EED
:106C0000EE0FFF1FE45CFD4E60817181882777FDE8
:106C10008095982F0E9422B69B01AC01D8016D91FE
:106C20007D918D919C910E94A6B40E94EFB597FF33
:106C300007C090958095709561957F4F8F4F9F4FBE
:106C400067307105810591055CF4F7FC14C00E9462
:106C500070AE6C197D09603D774008F44BCF0BC0D6
:106C60000E9470AE6B017C019FEFC916D906E90640
:106C7000F90659F73FCF82E193E00E940F860E9408
:106C800070AE6093CE067093CF068093D00690933B
:106C9000D1060E9470AE6093D6067093D70680939B
:106CA000D8069093D9068ECE0E94616A88E50E942C
:106CB000471C81115F9A89E50E94471C81118A9ABD
:106CC0008AE50E94471C882341F09FB7F894809181
:106CD00008018160809308019FBF85E40E94471CE2
:106CE000882309F415C8129A479A12C8A2960FB6BB
:106CF000F894DEBF0FBECDBFDF91CF911F910F91F2
:106D0000FF90EF90DF90CF90BF90AF909F908F90CB
:106D10007F906F905F904F903F900895CF93DF9357
:106D20008091E0069091E106039714F40E94B41C50
:106D300060E08FE099E00E94C04D8091E006909164
:106D4000E106892B09F463C080910F098823E1F0E3
:106D50008091E4069091E50620E6289FE001299FB6
:106D6000D00D1124C651D94F60E275E0CE010E94CA
:106D700098BC892BF1F4BE018FE099E00E94504D40
:106D800080911009882319F00E9473242AC0EDE134
:106D9000F5E08491882341F09091C00095FFFCCFED
:106DA0008093C6003196F5CF8091C00085FFFCCF5F
:106DB00015C08FE099E00E94B44EEBE0F5E08491BD
:106DC000882341F09091C00095FFFCCF8093C600CE
:106DD0003196F5CF8091C00085FFFCCF8AE080938B
:106DE000C6008091E0069091E10601979093E1063C
:106DF0008093E0068091E4069091E506019664E0B8
:106E000070E00E943EB99093E5068093E4060E94EC
:106E10009D6C0E9471230E948F620E94DA22DF9192
:106E2000CF910C941C8721ED33E0FC01318320834A
:106E30002781222311F0049680C608958FE099E0FF
:106E40000C94CB468FED99E0EEDF8DE999E0EBDF16
:106E50008EE799E0E8DF8FE599E0E5DF8EE399E0E2
:106E6000E2CF8FEF8EBD0DB407FEFDCF8EB5089536
:106E70008EBD0DB407FEFDCF089561E0FC01808159
:106E80000C9489B0FC012281322F306A36953CBDCA
:106E900020FD06C031E0263009F430E0232F01C088
:106EA00020E02DBD60E0FC0180810C9489B0CF9280
:106EB000DF92EF92FF920F931F93CF93DF93EC013A
:106EC0008B017A010E9470AE6B01CBDF8B838F3F09
:106ED00049F40E9470AE6C197D096D327140A8F3BF
:106EE00081E103C08E3F31F08FE08983CE01C5DFA1
:106EF00080E024C0E114F104E1F081E0E81AF10837
:106F00008FEF8EBDF8012FEFCF01801B910B8E15F7
:106F10009F0538F40DB407FEFDCF8EB581932EBDCD
:106F2000F3CF0DB407FEFDCF8EB5F801EE0DFF1DBA
:106F3000808397DF96DFCE01A0DF81E0DF91CF91E4
:106F40001F910F91FF90EF90DF90CF9008950F93D6
:106F50001F93CF93DF93EB010E9470AE8B0181DF13
:106F60008F3F49F00E9470AE601B710B6C177D075C
:106F7000B0F380E001C081E0DF91CF911F910F91CC
:106F80000895CF92DF92FF920F931F93CF93DF93D9
:106F900000D01F92CDB7DEB76C01F62E29833A835D
:106FA0004B835C836FDF6CE271E0C601D0DF8F2D15
:106FB00080645EDF08E110E05C814B813A812981C9
:106FC000DA01C901002E04C0B695A795979587955B
:106FD0000A94D2F729833A834B835C8349DF0850B4
:106FE000110929813A814B815C81083F8FEF180795
:106FF00039F7FF2029F0E8E0FE1621F08FEF03C0FB
:1070000085E901C087E834DFFCE0FF1201C029DF19
:1070100010E027DFF601838387FF04C01F3F11F0D4
:107020001F5FF7CF0F900F900F900F90DF91CF91D0
:107030001F910F91FF90DF90CF900895BF92CF9254
:10704000DF92EF92FF920F931F93CF93DF93EC01A8
:10705000B62E1C82198248830E9470AE8B0161E0BB
:1070600088810E9450B0CE0108DF60E082E30E9478
:1070700050B061E083E30E9450B061E084E30E947D
:1070800050B061E085E30E9450B061E085E30E946A
:1070900089B085E08A8382E58CBD1DBC2AE0F22E92
:1070A0008FEFE6DEFA94E1F720E030E0A90160E03E
:1070B000CE0167DFF82E8B8381E0F81649F00E943D
:1070C00070AE601B710B613D774070F381E046C08C
:1070D0002AEA31E040E050E068E0CE0152DF82FF72
:1070E00002C0FC820CC094E0F92EBBDE8B83FA94C4
:1070F000E1F78A3A11F082E031C082E08C838C8122
:10710000823031F4C12CD12CE12C80E4F82E03C064
:10711000C12CD12C760120E030E0A90167E3CE013B
:1071200030DFA701960169E2CE012BDF8B83882334
:1071300049F00E9470AE601B710B613D774058F3BF
:107140008AE00CC08C818230B1F420E030E0A901EB
:107150006AE3CE0116DF882329F088E08983CE0117
:107160008CDE14C07EDE807C803C11F483E08C8356
:1071700078DE77DE76DECE0180DE86E08B1518F4D1
:1071800088E1898303C0BA8281E001C080E0DF9199
:10719000CF911F910F91FF90EF90DF90CF90BF9014
:1071A00008950F931F93CF93DF93EC0189018C8196
:1071B000833039F039E0440F551F661F771F3A9529
:1071C000D1F79A01AB0161E1CE01DBDE811109C08B
:1071D00040E052E0B801CE01DF91CF911F910F91B5
:1071E00066CE84E08983CE0148DE80E0DF91CF91D6
:1071F0001F910F910895CF93DF93EC016EBD20E0B6
:1072000030E00DB407FEFDCFFA01E20FF31F8081DD
:107210008EBD0DB407FEFDCF81818EBD2E5F3F4F29
:10722000211582E0380769F70DB407FEFDCF8FEF17
:107230001FDE8FEF1DDE15DE8B838F71853031F001
:1072400083E18983CE0119DE80E001C081E0DF9116
:10725000CF9108950F931F93CF93DF93EC01890192
:107260008C81833039F089E0440F551F661F771FEA
:107270008A95D1F79A01AB0168E1CE0182DE8823BD
:1072800011F086E01EC0A8016EEFCE01B4DF8823A6
:10729000C9F068E572E0CE015ADE182F811102C0F4
:1072A00087E10FC020E030E0A9016DE0CE0169DE8A
:1072B000811106C0D6DD811103C0CE01DEDD05C01F
:1072C00086E18983CE01D9DD10E0812FDF91CF9156
:1072D0001F910F910895CF93DF93EC019C012C5FD8
:1072E0003F4F41E050E060E070E0898D9A8D0E9450
:1072F0002744882399F04D895E896F89788D452BC5
:10730000462B472B59F44C815D816E817F814D8BDB
:107310005E8B6F8B788F998190689983DF91CF9185
:107320000895CF92DF92EF92FF920F931F93CF9326
:10733000DF93EC0189899A89AB89BC89803E9F4F94
:10734000AF41B10510F080E06AC0CE01C4DF8823F0
:10735000D1F30E943B42182F8823A9F3E98DFA8DBF
:10736000CC80DD80EE80FF8032E0C31AD108E108D6
:10737000F108058404C0CC0CDD1CEE1CFF1C0A9433
:10738000D2F786859785A089B189C80ED91EEA1ED5
:10739000FB1E81E08093170AC0921A0CD0921B0C3E
:1073A000E0921C0CF0921D0C80E092E0EAE1FAE021
:1073B000DF019C011D9221503040E1F701E0E98D91
:1073C000FA8D8481081788F42AE13AE0B701A60112
:1073D000400F511D611D711D8091180A9091190A6D
:1073E00039DF8823E1F00F5FEACFC12C82E0D82E8D
:1073F000E12CF12C058404C0CC0CDD1CEE1CFF1C20
:107400000A94D2F749895A896B897C894C0D5D1D94
:107410006E1D7F1D498B5A8B6B8B7C8B812FDF916F
:10742000CF911F910F91FF90EF90DF90CF90089533
:10743000CF93DF93EC0141E0611101C040E06C8526
:107440007D858E859F850E947B42882341F08889B7
:1074500020E2829FC0011124865E954F02C080E029
:1074600090E0DF91CF91089530E020E04EE2DC0122
:107470005C91503271F0383029F4FB01E20FF11DBC
:1074800040832F5FFB01E20FF11DDC015C91508313
:107490002F5F3F5F01963B3051F7FB01E20FF11D7B
:1074A00010820895CF93DF93EB01FC01238121111A
:1074B00002C080E00EC02250223020F48FE2888388
:1074C000198206C060E0B4DF009799F3BE01CCDFFB
:1074D00081E0DF91CF910895FB012BE030E2319301
:1074E0002150E9F7DC0190E027E03A2FEB2F8D9156
:1074F00081110AC0DA013C931196EC9381E0FB0103
:107500009081903239F525C08F32A1F38E3219F077
:10751000E0E3F6E008C02A30E1F098E02AE0E5CFA9
:1075200031963817B1F034913111FACF291788F01C
:107530003FED380F3E3568F431E0390FFB01E90FBC
:10754000F11D9FE9980F9A3108F480528083932FA0
:10755000CCCF80E008950F931F93CF93DF93EC017E
:107560008B018B81882311F080E042C0FB01878969
:10757000803139F18032C1F783E08B83F801428D8D
:10758000538D648D758D4D8B5E8B6F8B788F9E01C7
:107590002F5E3F4FC8010E943243882329F31A8F80
:1075A000098F81E089831C821D821E821F821886BA
:1075B00019861A861B861C861D861E861F86188ABB
:1075C00017C082E08B831D8A1E8A1F8A188EFB01DA
:1075D000408D518D60E070E095E0440F551F661FAF
:1075E000771F9A95D1F7498B5A8B6B8B7C8BD7CFB2
:1075F000DF91CF911F910F9108952F923F924F925B
:107600005F926F927F928F929F92AF92BF92CF9232
:10761000DF92EF92FF920F931F93CF93DF93EC01D2
:107620005B016A018B81811103C08FEF9FEFC6C0A0
:10763000898180FFFACF49895A896B897C8988853D
:107640009985AA85BB852601612C712C8A019B0135
:10765000081B190B2A0B3B0B4016510662067306DA
:1076600018F06A01C81AD90A76013E0124E0620EB8
:10767000711CE114F10409F476C0488559856A85C6
:107680007B854A0181E098222B811A012B01E9E0D8
:107690005694479437942794EA95D1F7898D9A8D1B
:1076A000FC01223049F4628D738D848D958D620DBD
:1076B000731D841D951D3CC014811150122181142D
:1076C0009104C1F4111116C0452B462B472B49F4E8
:1076D0008D899E89AF89B88D8C839D83AE83BF834E
:1076E00009C04C815D816E817F8193013CD78823E5
:1076F00009F49BCFE98DFA8D6C817D818E819F810C
:107700006250710981099109058404C0660F771FD1
:10771000881F991F0A94D2F7268537854089518999
:10772000620F731F841F951F610F711D811D911DB5
:1077300020E032E02819390987012E153F0508F4A9
:1077400089010115F2E01F0761F520911A0C3091B3
:107750001B0C40911C0C50911D0C62177307840781
:10776000950719F41EC0C60129C09501AB01BC01E3
:107770008091180A9091190A14DD882309F455CFD5
:10778000A00EB11E88859985AA85BB85800F911FA3
:10779000A11DB11D88879987AA87BB87E01AF10AC6
:1077A00068CF40E0A8D6882309F43FCFB401665ED5
:1077B000754FA801C5010E94BFBCE2CFDF91CF91F8
:1077C0001F910F91FF90EF90DF90CF90BF90AF90FF
:1077D0009F908F907F906F905F904F903F902F90F1
:1077E0000895CF93DF931F92CDB7DEB741E050E00D
:1077F000BE016F5F7F4F01DF019719F4898190E02F
:1078000002C08FEF9FEF0F90DF91CF910895CF923D
:10781000DF92EF92FF920F931F93CF93DF936C0150
:10782000EB017A01FC018381823060F000851185D3
:10783000228533850F71112722273327012B022B35
:10784000032B11F08FEF5CC04115510511F0F701CA
:1078500010821DE040E250E0BE01C601CEDE803263
:10786000910539F021E0892B09F420E0822F8195E0
:1078700047C028812223C1F0253E61F32E3251F307
:107880003B853F733F3061F4E114F10449F04A8DC8
:107890005B8D452B29F42F713FEF320F323030F0E2
:1078A0002B8523FDD7CF2CC080E02AC030E02150AB
:1078B0003109129FC001139F900D1124F701E80FA9
:1078C000F91F298120832B8121832D8122832F8100
:1078D0002383298524832E852583288926832A8945
:1078E00027832C8920872E892187288D22872C8D1C
:1078F00023872E8D2487288126FFD2CF1586D0CFCF
:10790000DF91CF911F910F91FF90EF90DF90CF907B
:1079100008951F93CF93DF93EC018B81823018F48D
:1079200080E090E023C0488559856A857B85A5E085
:107930007695679557954795AA95D1F7142F1F709F
:10794000CE014FDF97FDECCF488559856A857B8551
:10795000415E5F4F6F4F7F4F488759876A877B87AC
:1079600020E2129FC0011124865E954FDF91CF91D6
:107970001F9108954F925F926F927F92AF92BF9244
:10798000CF92DF92EF92FF920F931F93CF93DF93EB
:10799000EC016A017B012B81222349F089899A89B4
:1079A000AB89BC8984179507A607B70710F480E058
:1079B0006BC0223009F463C0C114D104E104F104A6
:1079C00049F41C821D821E821F82188619861A861F
:1079D0001B8659C088859985AA85BB85E98DFA8D56
:1079E000E585F0E03996AC01BD01415051096109CE
:1079F00071090E2E04C076956795579547950A94A0
:107A0000D2F797018601015011092109310904C0FB
:107A10003695279517950795EA95D2F70417150718
:107A20002607370720F0892B8A2B8B2B49F48D8969
:107A30009E89AF89B88D8C839D83AE83BF8304C03C
:107A4000041B150B260B370B280139015E0184E05E
:107A5000A80EB11C411451046104710481F04C81E1
:107A60005D816E817F819501898D9A8D7CD591E0B4
:107A7000491A5108610871088111ECCF05C0C88608
:107A8000D986EA86FB8681E0DF91CF911F910F9125
:107A9000FF90EF90DF90CF90BF90AF907F906F906E
:107AA0005F904F9008950F931F93CF93DF93EC0156
:107AB0008B818823D1F1898187FF32C061E0CE01BB
:107AC000B7DC8C01009789F1FC018081853E69F16A
:107AD0008B81823040F449895A896B897C89448F33
:107AE000558F668F778F4D895E896F89788DF80104
:107AF000538F428F758B648BE091110AF091120ABB
:107B0000309759F0B8016A5E7F4FC80148961995C1
:107B1000F801808D918D938B828B89818F778983FA
:107B2000DF91CF911F910F91A6C481E0888380E0FF
:107B3000DF91CF911F910F910895CF93DF93EC01C7
:107B4000B2DF1B82DF91CF910895FC0123812111C7
:107B5000F4CF08954F925F926F927F92AF92BF924F
:107B6000CF92DF92EF92FF920F931F93CF93DF9309
:107B700000D01F92CDB7DEB75C016A017B01FC012A
:107B800083818130E9F4818181FF1AC0F501818907
:107B90009289A389B48984179507A607B70780F04F
:107BA000892B8A2B8B2B09F472C0F50140845184F8
:107BB00062847384B701A601C501DCDE811102C0B5
:107BC00080E066C0F501818D928DC114D104E1047D
:107BD000F10469F4458956896789708D41D78823F6
:107BE00079F3F501158A168A178A108E37C0F501C8
:107BF00044815581668177819E012F5F3F4FB3D4C9
:107C00008823F1F249815A816B817C81F501818D54
:107C1000928DFC012789203139F4483FFFEF5F073F
:107C200061057105D8F407C0483F2FEF520762077E
:107C30002FE0720798F414D7882309F4C1CFF50117
:107C400044815581668177810FEF1FEF2FEF3FE071
:107C5000818D928D6DD5882309F4B2CFF501C18A4B
:107C6000D28AE38AF48A818180688183C5011BDF1F
:107C7000882309F4A5CFB701A6014C145D046E0456
:107C80007F0410F4B301A201C50174DE01C081E0DC
:107C90000F900F900F900F90DF91CF911F910F9148
:107CA000FF90EF90DF90CF90BF90AF907F906F905C
:107CB0005F904F900895FF920F931F93CF93DF93A0
:107CC000EC01F42E80E2689FF0011124E65EF54F8E
:107CD0008385817121F0842F827109F04EC08091DB
:107CE0001A0C90911B0CA0911C0CB0911D0C8C8750
:107CF0009D87AE87BF87688B4489558960E070E0B7
:107D0000BA0155274427028D138D20E030E0402B27
:107D1000512B622B732B4D8B5E8B6F8B788F8385F2
:107D2000887151F4048D158D268D378D098B1A8B32
:107D30002B8B3C8B81E00BC08031F9F49E012F5ED0
:107D40003F4F898D9A8D8ED48823B9F084E08B8340
:107D50008F2D8F7089831C821D821E821F82188640
:107D600019861A861B86F4FE0BC040E050E0BA016B
:107D7000CE01F0DE811104C011C01B8280E00EC074
:107D8000F5FE0BC049895A896B897C89CE01DF9148
:107D9000CF911F910F91FF90EDCD81E0DF91CF91B9
:107DA0001F910F91FF900895AF92BF92CF92DF92F3
:107DB000EF92FF920F931F93CF93DF937C01EB0120
:107DC0006A01B22E898D9A8DF701928F818F40E0E2
:107DD00050E0BA01CE01CEDDA12C088519852A8597
:107DE0003B8589899A89AB89BC89081719072A07B5
:107DF0003B07A0F585E036952795179507958A9559
:107E0000D1F70F70CE0185DD009709F481C0FC0128
:107E10002081222311F0253EB9F4A1100EC040911B
:107E20001A0C50911B0C60911C0C70911D0CF701E9
:107E30004487558766877787008BFC018081AA2459
:107E4000A3948111CACF0AC04BE050E0BC01C60127
:107E50000E94B2BC892B09F0C0CF58C08B2D827410
:107E6000823409F055C0AA2049F0F701008961E089
:107E7000C701DEDAEC01009769F44AC08B818230D9
:107E800009F446C0CE014DDA882309F441C0CAE1A5
:107E9000DAE000E080E2FE0111928A95E9F78BE0DA
:107EA000F601DE0101900D928A95E1F7E091110A49
:107EB000F091120A309739F0BE01625F7F4FCE0118
:107EC0004096199508C081E298E2998B888B80E0F2
:107ED00098E09F878E87888999899B8B8A8B998F59
:107EE000888F8E859F859F8B8E8BC5D2882381F04E
:107EF0004B2D602FC701DF91CF911F910F91FF9004
:107F0000EF90DF90CF90BF90AF90D5CEB7FEF0CF7F
:107F100080E0DF91CF911F910F91FF90EF90DF9064
:107F2000CF90BF90AF9008953F924F925F926F9223
:107F30007F928F929F92AF92BF92CF92DF92EF92F9
:107F4000FF920F931F93CF93DF93CDB7DEB7C35448
:107F5000D1090FB6F894DEBF0FBECDBF5C016B0137
:107F600024965FAF4EAF2497522E1C8E1F8E19821F
:107F70001C826115710511F410E073C0FC0183814E
:107F80008111FACF2496EEADFFAD249780818F3218
:107F900011F076011DC02496EEADFFAD24978081CF
:107FA0008F3231F431962496FFAFEEAF2497F3CFA2
:107FB000F60183818250823060F3F601618D728D0B
:107FC000CE010196C8DA8823B9F2CE0101967C0170
:107FD0008E01045E1F4F3801FE0131964F01402E85
:107FE000312E19C08823A9F121E0AE01495C5F4F11
:107FF000B701C801D9DE882309F4BECFEC14FD0413
:1080000011F0C7019ADD0615170501F1942D832D96
:108010007801092F182FAE014E5B5F4FBE01695CDE
:108020007F4F24968EAD9FAD249756DA882309F4AE
:10803000A3CF2496EEADFFAD249780818F3291F6C9
:1080400031962496FFAFEEAF2497F3CF982D892D6C
:10805000DFCF252DAE01495C5F4FB701C501A4DE1E
:10806000182FCE01019671DDCE014C966EDD812F69
:10807000CD5BDF4F0FB6F894DEBF0FBECDBFDF91F3
:10808000CF911F910F91FF90EF90DF90CF90BF9015
:10809000AF909F908F907F906F905F904F903F90A8
:1080A0000895CF93DF93EC0140E050E0BA0152DD38
:1080B000882361F061E0CE01BBD9009739F025EE4D
:1080C000FC0120831B82DF91CF91D5C180E0DF913D
:1080D000CF9108951F93CF93DF93CDB7DEB76B9702
:1080E0000FB6F894DEBF0FBECDBFAB0119821C8264
:1080F00022E0BC01CE01019617DF182F882321F062
:10810000CE010196CEDF182FCE0101961EDD812F04
:108110006B960FB6F894DEBF0FBECDBFDF91CF9147
:108120001F9108952F923F924F925F926F927F928C
:108130008F929F92AF92BF92CF92DF92EF92FF9277
:108140000F931F93CF93DF9300D01F921F92CDB751
:10815000DEB78C015B013A01DC0113968C91139719
:108160008130C1F411968C9181FF14C082FF18C038
:10817000F801418952896389748980859185A28536
:10818000B38584179507A607B70751F0C801F2DB3E
:10819000811106C081E0F80180838FEF9FEF37C126
:1081A000630183C0D80159968D919C915A97FC0127
:1081B000F481F1501A012B0169E0569447943794E9
:1081C00027946A95D1F7F221FD834A0121E092229A
:1081D000FF2309F476C080E092E0881999097601BE
:1081E0008C159D0508F47C01D8015996ED91FC9100
:1081F0005A9714962D903D904D905C901797B2E051
:108200002B1A310841085108058404C0220C331C84
:10821000441C551C0A94D2F786859785A089B1899C
:10822000280E391E4A1E5B1EED812E0E311C411C8C
:10823000511CE114F2E0FF0609F089C080911A0C8C
:1082400090911B0CA0911C0CB0911D0C82159305F4
:10825000A405B50569F41092170A8FEF9FEFDC01B2
:1082600080931A0C90931B0CA0931C0CB0931D0CC4
:108270009501B201A1018091180A9091190A0E94FA
:108280002A39882309F486CFF80180859185A28553
:10829000B3858E0D9F1DA11DB11D80879187A2877B
:1082A000B387AE0CBF1CCE18DF08D80118964D91CD
:1082B0005D916D917C911B97C114D10409F072CF2F
:1082C0007AC08114910409F086CF14964D915D9186
:1082D0006D917C911797411551056105710559F410
:1082E00055968D919D910D90BC91A02D0097A10563
:1082F000B10539F520C09E012F5F3F4F34D188234F
:1083000009F448CF89819A81AB81BC81F801218D24
:10831000328DF9012789203139F4883FFFEF9F071B
:10832000A105B10540F40DC0883F2FEF9207A207C9
:108330002FE0B20730F0C8010E946B3981114BCF9A
:1083400029CFF80184839583A683B78344CF811412
:10835000910411F5D80118964D915D916D917C9124
:108360001B9751968D919D910D90BC91A02D481712
:1083700059076A077B0780F07ED0882309F40ACF6B
:1083800081E08093170A20921A0C30921B0C4092C5
:108390001C0C50921D0C07C041E0C201B101ABD0D2
:1083A000882309F4F7CEA701B501C401865E954F75
:1083B0000E94BFBC69CF51968D919D910D90BC914B
:1083C000A02DF801218184179507A607B70738F477
:1083D000418B528B638B748B206821830CC08091FE
:1083E000110A9091120A892B31F06114710419F06D
:1083F0002068F8012183D80111968C9183FD02C079
:10840000C30105C0C8014FDB8111FACFC3CE0F9065
:108410000F900F900F900F90DF91CF911F910F91C0
:10842000FF90EF90DF90CF90BF90AF909F908F9094
:108430007F906F905F904F903F902F900895CF93D3
:10844000DF931F92CDB7DEB7698341E050E0BE01F4
:108450006F5F7F4F049666DE0F90DF91CF91089596
:10846000FB0101900020E9F7AF0141505109461B83
:10847000570B049657CECF938091170A8823B9F1F2
:1084800040911A0C50911B0C60911C0C70911D0CAA
:108490002AE13AE08091180A9091190A0E942A393B
:1084A000C82F811102C0C0E023C04091130A50912F
:1084B000140A6091150A7091160A4115510561055B
:1084C000710591F02AE13AE08091180A9091190A19
:1084D0000E942A39882339F31092130A1092140A41
:1084E0001092150A1092160A1092170A01C0C1E0E4
:1084F0008C2FCF910895CF92DF92EF92FF92CF937E
:108500006B017C01C42F80911A0C90911B0CA091DF
:108510001C0CB0911D0C8C159D05AE05BF05C9F056
:10852000AADF811102C080E018C02AE13AE0B70159
:10853000A6018091180A9091190A0E94D1388823C7
:1085400091F3C0921A0CD0921B0CE0921C0CF0928A
:108550001D0C81E0C1118093170ACF91FF90EF901D
:10856000DF90CF9008958F929F92AF92BF92CF925B
:10857000DF92EF92FF920F931F93CF93DF93EC0163
:108580006A017B01890189859A85AB85BC85019645
:10859000A11DB11D84179507A607B70710F480E049
:1085A00054C08F89803129F49927872F762F652F22
:1085B0000BC08032A1F7CB01BA0127E096958795D1
:1085C000779567952A95D1F78B889C88AD88BE886A
:1085D000680D791D8A1D9B1D80901A0C90901B0CB4
:1085E000A0901C0CB0901D0C681579058A059B05A0
:1085F00081F48F89803191F4DD24EE24FF24F6018B
:10860000EE0FFF1FE65EF54F80819181A0E0B0E0A4
:1086100016C040E070DF8111ECCFC1CFE894C7F8FD
:10862000DD24EE24FF24F601EE0FFF1FEE0FFF1FE7
:10863000E65EF54F80819181A281B381BF70F80120
:1086400080839183A283B38381E0DF91CF911F91D7
:108650000F91FF90EF90DF90CF90BF90AF909F90E1
:108660008F9008954F925F926F927F92AF92BF92D8
:10867000CF92DF92EF92FF920F931F93CF93DF93EE
:1086800000D01F92CDB7DEB78C0149835A836B832C
:108690007C835901C12CD12C7601412C42E0542E0F
:1086A000612C712C49815A816B817C819E012F5FE5
:1086B0003F4FC80158DF882341F1D301C201F801BF
:1086C000058404C0880F991FAA1FBB1F0A94D2F704
:1086D000C80ED91EEA1EFB1E49815A816B817C811E
:1086E0008789803139F481E0483F5F4F610571052A
:1086F00038F4D8CF81E0483F5F4F6F4F7F4090F212
:10870000F501C082D182E282F3820F900F900F9028
:108710000F90DF91CF911F910F91FF90EF90DF901D
:10872000CF90BF90AF907F906F905F904F900895E3
:108730004F925F926F927F928F929F92AF92BF9271
:10874000CF92DF92EF92FF920F931F93CF93DF931D
:10875000EC014A015B0128013901423051056105F4
:10876000710508F462C049855A856B857C854F5F29
:108770005F4F6F4F7F4F481559056A057B0508F419
:1087800054C08F89803129F4FF24EB2CDA2CC92CBA
:108790000CC0803209F049C07501640177E0F6949D
:1087A000E794D794C7947A95D1F74B895C896D8902
:1087B0007E89C40ED51EE61EF71E41E0C701B60134
:1087C0009ADE882391F19F89903159F49924AA2443
:1087D000BB24F401EE0FFF1FE65EF54F518240828D
:1087E00010C0E89487F89924AA24BB24F401EE0F62
:1087F000FF1FEE0FFF1FE65EF54F4082518262823F
:1088000073829A89923090F04D815E816F81788574
:108810004C0D5D1D6E1D7F1D4093130A5093140A6D
:108820006093150A7093160A01C080E0DF91CF9122
:108830001F910F91FF90EF90DF90CF90BF90AF907E
:108840009F908F907F906F905F904F9008952F92A0
:108850003F924F925F926F927F928F929F92AF92D0
:10886000BF92CF92DF92EF92FF920F931F93CF931D
:10887000DF93CDB7DEB72F970FB6F894DEBF0FBEEC
:10888000CDBF1C014C875D876E877F873B872A871A
:10889000DC0119960D911D912D913C911C970F5F54
:1088A0001F4F2F4F3F4F0D831E832F833887EA853D
:1088B000FB8580809180A280B38081149104A10403
:1088C000B10431F0FFEF8F1A9F0AAF0ABF0A10C040
:1088D000DC018D909D90AD90BC90B1E0B9870C8586
:1088E0001D852E853F85013011052105310509F0D3
:1088F000198675016401412C512C3201F1018185E9
:108900009285A385B485481659066A067B0608F049
:108910004EC00D811E812F8138850C151D052E0539
:108920003F0550F4F2E0CF2ED12CE12CF12CA2E047
:108930008A2E912CA12CB12C9E012F5F3F4FB701A5
:10894000A601C10110DE882391F149815A816B8112
:108950007C81D701C6010196A11DB11D452B462B77
:10896000472B19F04C015D010FC0AC01BD01481946
:1089700059096A097B090C851D852E853F8540179D
:1089800051076207730741F01FEF411A510A610A4C
:10899000710A6C017D01B2CF0FEF1FEF2FEF3FE0A7
:1089A000B701A601C101C4DE8D83811113C01D82F0
:1089B0003DC02601370121E0421A510861087108C3
:1089C00097018601B301A201C101B2DE882379F3C8
:1089D000730162018C149D04AE04BF0450F3AA8598
:1089E000BB854D915D916D917C914115510561055E
:1089F0007105A9F4EA85FB8580829182A282B38207
:108A0000F985FF2399F00FEF801A900AA00AB00AA7
:108A1000D1018D929D92AD92BC92139707C09501A2
:108A20008401C10185DE8111E5CFC1CF8D812F96F3
:108A30000FB6F894DEBF0FBECDBFDF91CF911F916F
:108A40000F91FF90EF90DF90CF90BF90AF909F90ED
:108A50008F907F906F905F904F903F902F900895F0
:108A6000AF92BF92CF92DF92EF92FF920F931F933C
:108A7000CF93DF9300D01F92CDB7DEB75C016A01C0
:108A80007B0182E090E0A0E0B0E0F501808391837B
:108A9000A283B3839E012F5F3F4FB701A601C5019B
:108AA00062DD811102C080E023C000E010E0980187
:108AB000B701A601C5013CDE8823A9F3C980DA808D
:108AC000EB80FC80F5018789803149F481E0F8EF83
:108AD000CF16FFEFDF06E104F10450F4DBCF81E0B5
:108AE00098EFC9169FEFD906E9069FE0F90690F2C4
:108AF0000F900F900F900F90DF91CF911F910F91DA
:108B0000FF90EF90DF90CF90BF90AF9008957F924D
:108B10008F929F92AF92BF92CF92DF92EF92FF928D
:108B20000F931F93CF93DF93EC01142F7093190AC7
:108B30006093180A1F8A82E090E0A0E0B0E088838A
:108B40009983AA83BB831092170A1092130A10927A
:108B5000140A1092150A1092160A8FEF9FEFDC018B
:108B600080931A0C90931B0CA0931C0CB0931D0CBB
:108B7000442349F1453008F0DEC040E060E070E099
:108B8000CB01B9DC882309F4D6C020E1129FF001A3
:108B90001124E853F44F80818F7709F0CCC084858D
:108BA0009585A685B78584369105A105B10508F49C
:108BB000C2C0C084D184E284F384C114D104E1042E
:108BC000F10421F4B8C0C12CD12C760140E0C701DA
:108BD000B60191DC782E882309F4ADC08091250A76
:108BE0009091260A8115924009F0A5C030912A0A79
:108BF000332309F4A0C08091280A9091290A892B77
:108C000009F499C02091270A222309F494C03A8BD1
:108C10002C831D8630E041E050E06D85062FCA01AF
:108C2000062E02C0880F991F0A94E2F72817390709
:108C300031F081E0860F8D87683078F37CC0209119
:108C4000300A3091310A2115310519F040E050E029
:108C500008C020913E0A30913F0A4091400A50914D
:108C6000410A2D833E834F8358878091280A909133
:108C7000290A46015701880E991EA11CB11C8B8A36
:108C80009C8AAD8ABE8AE0912B0AF0912C0AF98F5A
:108C9000E88FA0912A0AB0E00E9495B9680D791D6D
:108CA0008A1D9B1D6A8F7B8F8C8F9D8FB5E0EE0F89
:108CB000FF1FBA95E1F7E150FE4FEF2FFF27E69532
:108CC000DC01CB018E0F9F1FA11DB11D8E879F87D9
:108CD000A88BB98B80902D0A90902E0A8114910454
:108CE00019F0A12CB12C08C080903A0A90903B0A50
:108CF000A0903C0AB0903D0AA7019601281B390BB1
:108D00004A0B5B0BDA01C901880D991DAA1DBB1D19
:108D100004C0B695A795979587950A95D2F7898748
:108D20009A87AB87BC87853F3FE09307A105B105D4
:108D300020F48CE08F8B712C15C0853F9F4FA105CF
:108D4000B10510F480E10DC08091460A9091470A68
:108D5000A091480AB091490A8A8F9B8FAC8FBD8F32
:108D600080E28F8B872DDF91CF911F910F91FF9024
:108D7000EF90DF90CF90BF90AF909F908F907F90BB
:108D80000895FC01148217821382128281ED93E010
:108D90009183808308950F931F93CF93DF93EC010A
:108DA0008F96EFDFCE01805B9F4FEBDFCE018159C5
:108DB0009F4FE7DFCE0182579F4FE3DFFE01E35570
:108DC000FF4F89E1818314823596178ACE01805343
:108DD0009F4FD7DFFE01E151FF4F108211821282B7
:108DE0001382389610821182128213821A821B8299
:108DF000188219828E010D501F4FF80110821182C6
:108E000012821382389681E080831EA61DA60E94DE
:108E100070AE68577C4E8F4F9F4FF801608371830F
:108E200082839383DF91CF911F910F910895FC016D
:108E300020E03EE2DB014C91403241F0283011F459
:108E400030833196DB014C91408331962F5F6F5F09
:108E50007F4F2B3079F7108208953F924F925F92A7
:108E60006F927F928F929F92AF92BF92CF92DF923A
:108E7000EF92FF920F931F93CF93DF93CDB7DEB79F
:108E8000C758D1090FB6F894DEBF0FBECDBF8C0115
:108E90006B017A01312C84E0E80EF11C2801E1E13C
:108EA0004E0E511C5801FCEFAF0EB11C48018EEF65
:108EB000880E911C80E4682E712C6C0E7D1EE4E0FF
:108EC0006E0E711CA201BE016F5F7F4FC7010E9431
:108ED000073C18160CF02BC12C85322F387130311D
:108EE00009F09EC0F501808191810197029708F4F5
:108EF00097C0BE016F5F7F4FCE0187589F4F97DFAE
:108F0000A0961FAEA097F6018081811107C065ED84
:108F100073E0CE01815A9F4F0E94C8BCB601CE01BA
:108F2000815A9F4F0E94C8BCBE0167587F4FCE0137
:108F3000815A9F4F0E94C8BC65ED73E0CE01815AF3
:108F40009F4F0E94C8BCCE01805C9F4F1ADF21E07A
:108F5000AE0147585F4FB701C3010E94943F811192
:108F600039C0F50180819181892BA1F5EBE8F7E00B
:108F70008491882341F09091C00095FFFCCF8093AD
:108F8000C6003196F5CFE7EDF3E08191882339F003
:108F90009091C00095FFFCCF8093C600F6CF8091E2
:108FA000C00085FFFCCF8AE08093C600FE01E75831
:108FB000FF4F8191882339F09091C00095FFFCCF3D
:108FC0008093C600F6CF8091C00085FFFCCF8AE079
:108FD0008093C6008BE1FE01EC5BFF4FDE019596AE
:108FE00001900D928A95E1F724968EAD9FAD24975E
:108FF0009CA38BA381ED93E09AA389A3AE014F5D5F
:109000005F4FBE01615A7F4FC80127DFCE018196B5
:109010000E941337CE01805C9F4F0E94133752CFBE
:109020008981882309F483C0853E09F44BCF8E32B1
:1090300009F448CF8F3509F445CFF8018189882399
:1090400031F08E3209F43ECF8F3509F43BCF23FD4A
:1090500039CF81E0303109F080E0F80184A7811137
:1090600010C09091F4088985923121F48E3409F072
:1090700029CF03C0873409F025CF8A858E3709F4BC
:1090800021CF98012C5F3F4FBE016F5F7F4FC90119
:10909000CA57DF4F2883C658D040C957DF4F38839F
:1090A000C758D040C4DEF50180819181CA57DF4F97
:1090B0002881C658D040C957DF4F3881C758D040A3
:1090C0000097F1F4F6018191882339F09091C00066
:1090D00095FFFCCF8093C600F6CFF90181918823DC
:1090E00039F09091C00095FFFCCF8093C600F6CF79
:1090F0008091C00085FFFCCF8AE08093C600E2CE5D
:109100008130910539F4F401808191810196918338
:109110008083D8CE029709F0D5CE232D30E0F4011C
:10912000808191812817390711F03394CBCEC9572C
:10913000DF4F0FB6F894DEBF0FBECDBFDF91CF91EA
:109140001F910F91FF90EF90DF90CF90BF90AF9065
:109150009F908F907F906F905F904F903F90089579
:10916000EF92FF920F931F93CF93DF93CDB7DEB7AC
:109170006F970FB6F894DEBF0FBECDBF8C01FC0118
:10918000E450FF4F118210827C0183E3E80EF11C52
:1091900040E050E0BA01C7010E94BA3C8BE1F70100
:1091A000DE01159601900D928A95E1F7F80181A9EB
:1091B00092A99C838B8381ED93E09A838983AE018E
:1091C0004F5F5F4F6CEB74E0C80147DECE01019644
:1091D0000E9413376F960FB6F894DEBF0FBECDBF57
:1091E000DF91CF911F910F91FF90EF9008952BE1A8
:1091F000FB013496DC01149601900D922A95E1F75B
:10920000FB0122813381FC01338322830895EF9295
:10921000FF920F931F93CF93DF93EC011B828EA9D4
:10922000882321F0CE01C3960E949D3D7E018DEAE8
:10923000E80EF11C45E360E0C7010E941E38811171
:109240001FC0EBE8F7E08491882341F09091C000C3
:1092500095FFFCCF8093C6003196F5CFEEE7F7E09F
:109260008491882341F09091C00095FFFCCF8093BA
:10927000C6003196F5CF8091C00085FFFCCF74C049
:109280008E010E541F4F41E0B701C80140DC81112F
:1092900025C040E0B701C8013ADC81111FC0E1E9F7
:1092A000F7E08491882341F09091C00095FFFCCFB6
:1092B0008093C6003196F5CFEBE6F7E084918823E2
:1092C00041F09091C00095FFFCCF8093C60031968D
:1092D000F5CF8091C00085FFFCCF46C0B801CE011C
:1092E000C3960E94AB3A81111FC0E1E9F7E0849177
:1092F000882341F09091C00095FFFCCF8093C60079
:109300003196F5CFEBE5F7E08491882341F0909119
:10931000C00095FFFCCF8093C6003196F5CF8091B9
:10932000C00085FFFCCF20C081E08B83EBE8F7E035
:109330008491882341F09091C00095FFFCCF8093E9
:10934000C6003196F5CFE0E5F7E08491882341F03F
:109350009091C00095FFFCCF8093C6003196F5CF69
:109360008091C00085FFFCCF8AE08093C6008E010B
:10937000015D1F4FB801CE01805B9F4F38DFC25B9C
:10938000DF4F19830883DF91CF911F910F91FF90D9
:10939000EF900895FC01128213820895FC0123814D
:1093A000222311F021E022830895FC012281211162
:1093B000128208952F923F924F925F926F927F9206
:1093C0008F929F92AF92BF92CF92DF92EF92FF92D5
:1093D0000F931F93CF93DF93CDB7DEB7AD970FB643
:1093E000F894DEBF0FBECDBF7C016B014DA7FC0121
:1093F0008381882309F4A8C14701F4ED8F0E911CE5
:10940000C4010E949D3DF7011282CE0101965C01CC
:10941000B8DC17019EE4290E311CC7018F96F101BB
:1094200091838083F60180818F3209F07FC06FE2E3
:1094300070E0C6010E94D3BC8C010F5F1F4F09F47E
:109440007BC06FE270E0C8010E94D3BC2C01009782
:1094500009F473C00817190708F06FC03C01601ABF
:10946000710AA301B801CE0180960E94F3BCE0E22C
:10947000F0E0EC0FFD1FE60DF71D1082FE01B09627
:109480008191882339F09091C00095FFFCCF8093A3
:10949000C600F6CF8091C00085FFFCCFFAE0F093C4
:1094A000C600F101608171816115710519F06C5F71
:1094B0007F4F02C060E070E021E0AE01405E5F4F90
:1094C000CE0105960E94943F81112BC0ECE3F7E09A
:1094D0008491882341F09091C00095FFFCCF809348
:1094E000C6003196F5CFFE01B0968191882339F000
:1094F0009091C00095FFFCCF8093C600F6CFEAE3C1
:10950000F7E08491882341F09091C00095FFFCCF53
:109510008093C6003196F5CF8091C00085FFFCCFC7
:10952000E7C0F101B182A082820187CFC701805BD1
:109530009F4FF101918380838601FDA5FF2309F4EC
:109540009CC0F101608171816115710519F06C5F3A
:109550007F4F02C060E070E021E0A801C4010E94DA
:10956000943F882309F45FC0F40181899289A3891B
:10957000B489F701E151FF4F80839183A283B383C4
:10958000ECE2F7E08491D701A151BF4F882349F065
:109590009091C00095FFFCCF8093C60031968491D6
:1095A000F5CFF8018191882339F09091C00095FFA3
:1095B000FCCF8093C600F6CFE4E2F7E084918823E5
:1095C00041F09091C00095FFFCCF8093C60031968A
:1095D000F5CF4D915D916D917C912AE030E080E76F
:1095E00095E00E94DB168091C00085FFFCCF8AE0E9
:1095F0008093C600F701E950FF4F1082118212825A
:109600001382E6E1F7E08491882341F09091C00055
:1096100095FFFCCF8093C6003196F5CF8091C000B6
:1096200085FFFCCF88C0E2E0F7E08491882341F019
:109630009091C00095FFFCCF8093C6003196F5CF86
:10964000F8018191882339F09091C00095FFFCCFFB
:109650008093C600F6CFE0E0F7E08491882341F0E4
:109660009091C00095FFFCCF8093C6003196F5CF56
:109670008091C00085FFFCCF3BC0F101608171810A
:109680006115710519F06C5F7F4F02C060E070E0FA
:1096900026E5A801C4010E94943F81112DC0ECEE83
:1096A000F6E08491882341F09091C00095FFFCCFB3
:1096B0008093C6003196F5CFF8018191882339F067
:1096C0009091C00095FFFCCF8093C600F6CFEAEEE4
:1096D000F6E08491882341F09091C00095FFFCCF83
:1096E0008093C6003196F5CF8091C00085FFFCCFF6
:1096F0008AE08093C60025C081E0F7018083E8ED11
:10970000F6E08491882341F09091C00095FFFCCF52
:109710008093C6003196F5CFF6018191882339F008
:109720009091C00095FFFCCF8093C600F6CF80914A
:10973000C00085FFFCCF8AE08093C600C8010E946C
:109740000086C5010E941337AD960FB6F894DEBFB0
:109750000FBECDBFDF91CF911F910F91FF90EF9082
:10976000DF90CF90BF90AF909F908F907F906F9041
:109770005F904F903F902F90089521E0FC0121834E
:1097800040E018CE3F924F925F926F927F928F92FD
:109790009F92AF92BF92CF92DF92EF92FF920F9380
:1097A0001F93CF93DF93CDB7DEB7AC970FB6F89486
:1097B000DEBF0FBECDBF7C015B01FC01838188232E
:1097C00009F401C1C7018C529F4F0E949D3DF701D2
:1097D0001282CE0101966C01D4DA27019EE4490E73
:1097E000511CC7018F96F20191838083F50180811E
:1097F0008F3209F084C06FE270E0C5010E94D3BCD3
:109800008C010F5F1F4F9AE0392E0115110509F4E5
:109810007CC06FE270E0C8010E94D3BC4C0100978D
:1098200009F474C00817190708F070C03C01601AE9
:10983000710AA301B801CE0180960E94F3BCE0E258
:10984000F0E0EC0FFD1FE60DF71D1082FE01B09653
:109850008191882339F09091C00095FFFCCF8093CF
:10986000C600F6CF8091C00085FFFCCF3092C600C5
:10987000F201608171816115710519F06C5F7F4F94
:1098800002C060E070E021E0AE01405E5F4FCE01BB
:1098900005960E94943F81112BC0E4ECF6E0849180
:1098A000882341F09091C00095FFFCCF8093C600C3
:1098B0003196F5CFFE01B0968191882339F09091D1
:1098C000C00095FFFCCF8093C600F6CFE2ECF6E037
:1098D0008491882341F09091C00095FFFCCF809344
:1098E000C6003196F5CF8091C00085FFFCCF65C0E2
:1098F000F201D182C08284010F5F1F4F86CFC70162
:10990000805B9F4FF201918380838501F20180810A
:109910009181009711F0049602C080E090E0B801B8
:109920000E946A40882301F1E4EBF6E084918823E9
:1099300041F09091C00095FFFCCF8093C600319616
:10994000F5CFF8018191882339F09091C00095FFFF
:10995000FCCF8093C600F6CFF701E950FF4F10828D
:109960001182128213822CC0ECE9F6E084918823E4
:1099700041F09091C00095FFFCCF8093C6003196D6
:10998000F5CFF8018191882339F09091C00095FFBF
:10999000FCCF8093C600F6CFEAE9F6E084918823F5
:1099A00041F09091C00095FFFCCF8093C6003196A6
:1099B000F5CF8091C00085FFFCCF8AE08093C60080
:1099C000C6010E941337AC960FB6F894DEBF0FBEE7
:1099D000CDBFDF91CF911F910F91FF90EF90DF905E
:1099E000CF90BF90AF909F908F907F906F905F903F
:1099F0004F903F900895CF93DF93EC018B818823A4
:109A0000C1F1E8E8F6E08491882341F09091C0002C
:109A100095FFFCCF8093C6003196F5CFFE01E9504B
:109A2000FF4F40815181628173812AE030E080E7FD
:109A300095E00E94DB16E6E8F6E08491882341F089
:109A40009091C00095FFFCCF8093C6003196F5CF72
:109A5000C151DF4F488159816A817B812AE030E022
:109A600080E795E00E94DB168091C00085FFFCCF67
:109A700011C0E6E7F6E08491882341F09091C000A0
:109A800095FFFCCF8093C6003196F5CF8091C00042
:109A900085FFFCCF8AE08093C600DF91CF910895C7
:109AA000AF92BF92CF92DF92EF92FF920F931F93EC
:109AB000CF93DF935C01EB01FB0101900020E9F7FC
:109AC0008F0101501109061B170B6C01F4EDCF0E2D
:109AD000D11CF60110826EE470E0CE010E94D3BC6E
:109AE0007C01009729F4F8013197EC0FFD1F0DC0A0
:109AF00060E270E00E94D3BCEC0121966AE270E063
:109B0000C7010E94D3BCFC0131978DE081838AE0BC
:109B100082831382BE01C50180539F4F0E94304251
:109B2000F6018081882309F1E1E9F7E08491882337
:109B300041F09091C00095FFFCCF8093C600319614
:109B4000F5CFE0E6F6E08491882341F09091C000E3
:109B500095FFFCCF8093C6003196F5CF8091C00071
:109B600085FFFCCF8AE08093C600DF91CF911F91E3
:109B70000F91FF90EF90DF90CF90BF90AF9008953E
:109B80002F923F924F925F926F927F928F929F920D
:109B9000AF92BF92CF92DF92EF92FF920F931F93FB
:109BA000CF93DF93CDB7DEB7CC55D1090FB6F8947C
:109BB000DEBF0FBECDBF8C0185509F4F5C01662379
:109BC00039F0F5011082F801838181111DC015C0A3
:109BD000FC018081882309F4ADC0F801ED50FF4FEE
:109BE000C080D180E280F3800E9470AEC616D70696
:109BF000E806F90608F49EC0E4CFC80108DBF801C6
:109C00008381882309F496C0F80186A58F9385A5E2
:109C10008F9387E596E09F938F937E01FFE3EF0E8E
:109C2000F11CFF92EF920E947ABD0F900F900F905F
:109C30000F900F900F90B12CF70101900020E9F7E1
:109C40003197EE19FF09BE1684F46701CB0CD11CC5
:109C5000B7FCDA94F6018081992787FD90950E94E0
:109C600059BCF6018083B394E7CF4801F3E38F0E2C
:109C7000911C40E050E0BA01C4010E94BA3C512C52
:109C8000CE0101966C0120E5622E26E0722E5E0167
:109C900091E2A90EB11C40E050E0B601C4010E945F
:109CA000073C1816DCF5412CF60101900020E9F77D
:109CB0003197EC19FD094E1674F41601240C311C71
:109CC00047FC3A94F101808190E00E9459BCF10177
:109CD00080834394E9CF8A858E37E9F245E050E0EE
:109CE000B701C6010E94E5BC892BA9F6FF92EF924D
:109CF0007F926F92BF92AF920E947ABDC5010E947F
:109D000040198CE496E00E94B3190F900F900F90C9
:109D10000F900F900F9055245394BDCF511004C055
:109D20008FEF9FEFF80104C0F80185A596A5019675
:109D300096A785A7C45ADF4F0FB6F894DEBF0FBEB3
:109D4000CDBFDF91CF911F910F91FF90EF90DF90EA
:109D5000CF90BF90AF909F908F907F906F905F90CB
:109D60004F903F902F9008950F931F93CF93DF93C1
:109D7000EC018C010C521F4FC8010E94533DC801D9
:109D80000E949D3D18821982DF91CF911F910F9102
:109D90000895EF92FF920F931F93CF93DF93CDB768
:109DA000DEB76F970FB6F894DEBF0FBECDBF8C0144
:109DB0007C018EE4E80EF11CC801805B9F4FF70127
:109DC00091838083E255FF4F22E030E0318320838E
:109DD000329670E07183608340E050E0BA010496EF
:109DE0000E94BA3CF701808191812BE1FC013496FD
:109DF000DE01159601900D922A95E1F7FC01828112
:109E000093819C838B8381ED93E09A838983AE0158
:109E10004F5F5F4F6CEB74E0C8011FD8CE01019615
:109E20000E9413376F960FB6F894DEBF0FBECDBFFA
:109E3000DF91CF911F910F91FF90EF900895CF92F6
:109E4000DF92EF92FF920F931F93CF93DF93CDB7E3
:109E5000DEB76F970FB6F894DEBF0FBECDBF8C0193
:109E60006C012EE4C20ED11C805B9F4FF6019183E2
:109E70008083E255FF4F21E030E031832083780179
:109E8000FEEFEF0EF11CF7011182108240E050E06E
:109E9000BA0104960E94BA3CF601808191812BE1BF
:109EA000FC013496DE01159601900D922A95E1F79A
:109EB000FC01828193819C838B8381ED93E09A8363
:109EC0008983AE014F5F5F4F6CEB74E0C8010E9465
:109ED0002D47CE0101960E941337F70180819181B1
:109EE0006F960FB6F894DEBF0FBECDBFDF91CF9156
:109EF0001F910F91FF90EF90DF90CF900895CF9337
:109F0000DF93EC010E94616A0E94D76ACE018C52F5
:109F10009F4F0E949D3D1A8280E496E00E94B319F3
:109F20008091F4108823F9F01092F410C0919D08EC
:109F3000D0E0CC0FDD1FC45CDD4E688179818827BD
:109F400077FD8095982F0E9422B62091470230918C
:109F500048024091490250914A020E9483B7181664
:109F600014F419821882DF91CF9108952F923F92B5
:109F70004F925F926F927F928F929F92AF92BF9219
:109F8000CF92DF92EF92FF920F931F93CF93DF93C5
:109F9000CDB7DEB7C454D1090FB6F894DEBF0FBEFB
:109FA000CDBF3C011B014A012FA309A7EBA62196B7
:109FB000ACAEBDAECEAEDFAE219734E0239F200124
:109FC0001124440D551D5AAB49ABDA01CD90DD90FB
:109FD000ED90FC90FC01E40DF51D20813181428162
:109FE0005381C701B6010E94A7B46BAB7CAB8DABAC
:109FF0009EABB4E00B9F80011124F401E00FF11F30
:10A00000F8AFEFAB80809180A280B380F301E00FC6
:10A01000F11F2081318142815381C501B4010E9429
:10A02000A7B469AF7AAF8BAF9CAF2BA5F4E02F9F9D
:10A03000C0011124F301E80FF91F20813181428111
:10A040005381298F3A8F4B8F5C8FF101E80FF91FF5
:10A0500060817181828193810E94A6B46F8F78A301
:10A0600089A39AA3D1011C968D919D910D90BC91CD
:10A07000A02D8DA79EA7AFA7B8ABD3011C962D919D
:10A080003D914D915C911F972BA33CA34DA35EA3E3
:10A09000A701960150582D8B3E8B4F8B588FD501C1
:10A0A000C401B058898B9A8BAB8BBC8BF101E40D4A
:10A0B000F51D2BA93CA94DA95EA960817181828102
:10A0C00093810E94A6B46B017C01F101E00FF11FA6
:10A0D00029AD3AAD4BAD5CAD6081718182819381D8
:10A0E0000E94A6B44B015C01A70196016D897E898F
:10A0F0008F89988D0E9455B82B013C01A5019401D0
:10A1000069897A898B899C890E9455B89B01AC0129
:10A11000C301B2010E94A7B42B013C01A501940127
:10A120006D897E898F89988D0E9455B84B015C019D
:10A13000A701960169897A898B899C890E9455B803
:10A140009B01AC01C501B4010E94A6B4A301920118
:10A150000E941AB56B017C0120E030E0A9010E9449
:10A1600080B587FF0AC02BED3FE049EC50E4C70102
:10A17000B6010E94A7B46B017C016F968FAD6F97FB
:10A18000882351F02BED3FE049EC50E4C701B601C4
:10A190000E94A6B46B017C016E962CAD3DAD4EAD18
:10A1A0005FAD6E97C701B6010E9455B82F8D38A1DB
:10A1B00049A15AA15F770E9490B74B015C012FE63D
:10A1C00032E143E85AE30E9480B587FDC4C1C5016E
:10A1D000B4010E945DB60E94F4B57E8F6D8FDB01E5
:10A1E000AB2B21F4E1E0F0E0FE8FED8F2D8D3E8D65
:10A1F000B90180E090E00E9420B64B015C019B0118
:10A20000AC01C701B6010E9487B52B013C01A50135
:10A2100094016F8D78A189A19AA10E9487B5259696
:10A220006CAF7DAF8EAF9FAF25972BA13CA14DA109
:10A230005EA16DA57EA58FA598A90E94A6B4A501D3
:10A2400094010E9487B56DA77EA78FA798AB20E0E9
:10A2500030E040E05FE3C301B2010E9455B8A301C2
:10A2600092010E9455B89B01AC0160E070E080E86B
:10A270009FE30E94A6B46F8F78A389A39AA3CE010F
:10A280000196FC014BA534E0439FE00DF11D112424
:10A29000298D3A8D4B8D5C8D20833183428353838E
:10A2A0002BA13CA14DA15EA12D873E874F87588BE6
:10A2B000B12C41E050E05A8F498F81E090E08C0F43
:10A2C0009D1FBFA1A4E0BA9F800D911D11249CA7E2
:10A2D0008BA721E030E02C0F3D1F59A544E0549F8F
:10A2E000200D311D11243AA729A7F8A7EFA3498D06
:10A2F0005A8D8D8D9E8D4817590708F017C188E13A
:10A300008B150CF444C02F8D38A149A15AA169893D
:10A310007A898B899C890E9455B86B017C01A301C5
:10A3200092016D897E898F89988D0E9455B8A70109
:10A3300096010E94A7B4A62E172F982E892E2F8D36
:10A3400038A149A15AA16D897E898F89988D0E9473
:10A3500055B86B017C01A301920169897A898B89C7
:10A360009C890E9455B89B01AC01C701B6010E94AF
:10A37000A6B46D8B7E8B8F8B988FB3948A2D912F83
:10A38000A92DB82D898B9A8BAB8BBC8B6AC0A98DFC
:10A39000BA8DBD0180E090E00E9420B6A301920139
:10A3A0000E9455B86B017C010E9484B5698B7A8B41
:10A3B0008B8B9C8BC701B6010E94B8B84B015C0126
:10A3C000E9A9FAA9C080D180E280F380F7FAF0947D
:10A3D000F7F8F094AFA9B8AD2D913D914D915C91F6
:10A3E0002BA33CA34DA35EA329893A894B895C89A1
:10A3F000C701B6010E9455B86D8B7E8B8F8B988FED
:10A40000A50194016BA17CA18DA19EA10E9455B8CC
:10A410009B01AC016D897E898F89988D0E94A7B4BC
:10A420006D8B7E8B8F8B988FA5019401C701B60130
:10A430000E9455B86B017C0129893A894B895C8956
:10A440006BA17CA18DA19EA10E9455B89B01AC017E
:10A45000C701B6010E94A6B4698B7A8B8B8B9C8B4B
:10A46000B12C2D893E894F89588D6BA97CA98DA966
:10A470009EA90E94A7B4EBA5FCA56083718382838B
:10A48000938329893A894B895C8969AD7AAD8BAD13
:10A490009CAD0E94A7B4A9A5BAA56D937D938D9399
:10A4A0009C93139725962CAD3DAD4EAD5FAD259792
:10A4B000EFA1F8A560817181828193810E94A7B488
:10A4C000AFA1B8A56D937D938D939C9313972DA504
:10A4D0003EA54FA558A96D857E858F8598890E94D8
:10A4E000A7B46D877E878F87988BCE0101960E94D7
:10A4F000D720FE01E15AFF4F6F012196ECACFDAC75
:10A500000EAD1FAD21979E01235F3F4FAE01475F08
:10A510005F4FBE016B5F7F4FCE01019656D5298DEF
:10A520003A8D2F5F3F4F3A8F298FE1CE9101245F03
:10A530003F4FA101485F5F4FB1016C5F7F4FDE016C
:10A54000A15ABF4F6D012196ECACFDAC0EAD1FAD15
:10A550002197C1013AD5CC5BDF4F0FB6F894DEBF2F
:10A560000FBECDBFDF91CF911F910F91FF90EF9064
:10A57000DF90CF90BF90AF909F908F907F906F9023
:10A580005F904F903F902F9008952F923F924F925F
:10A590005F926F927F928F929F92AF92BF92CF9273
:10A5A000DF92EF92FF920F931F93CF93DF93CDB77C
:10A5B000DEB768970FB6F894DEBF0FBECDBF1C01A3
:10A5C0002A013B0148015901DC01D8966D917D912A
:10A5D0008D919C91DB970E9420B66B017C01A301B9
:10A5E00092010E9455B80E946DB50E94F4B56D8726
:10A5F0007E878F87988BA5019401C701B6010E94C1
:10A6000055B80E946DB50E94F4B5698B7A8B8B8B1F
:10A610009C8B2D853E854F8558892837310541050E
:10A62000510540F488E790E0A0E0B0E08D879E8778
:10A63000AF87B88B29893A894B895C8928373105DE
:10A640004105510540F488E790E0A0E0B0E0898B37
:10A650009A8BAB8BBC8B91012C5B3F4FD9018D91B9
:10A660009D910D90BC91A02D8D839E83AF83B88763
:10A67000BC01CD010E9422B669837A838B839C83BF
:10A68000F10164AD75AD86AD97AD0E9420B66987C6
:10A690007A878B879C8720E030E0A90169817A81E5
:10A6A0008B819C810E9480B5882339F1A701960196
:10A6B000C701B6010E9455B84B015C0129853A8556
:10A6C0004B855C85CA01B9010E9455B89B01AC015C
:10A6D000C501B4010E94A6B44B015C0129813A81F5
:10A6E0004B815C81CA01B9010E94A7B49B01AC01F6
:10A6F000C501B4010E9487B503C060E070E0CB01E2
:10A700000E946DB50E94EFB52B013C016D817E81E9
:10A710008F81988590958095709561957F4F8F4F2B
:10A720009F4F0E9422B64B015C01F101E05CFF4F9C
:10A7300060817181828193810E9420B66D837E83C6
:10A740008F83988720E030E0A901C501B4010E9401
:10A7500080B5882349F12D813E814F815885CA01FA
:10A76000B9010E9455B86D8B7E8B8F8B988FA70196
:10A770009601C701B6010E9455B89B01AC016D89D5
:10A780007E898F89988D0E94A6B46B017C01A501FA
:10A790009401C501B4010E94A7B49B01AC01C7019B
:10A7A000B6010E9487B503C060E070E0CB010E9453
:10A7B0005DB6D10150968D909D90AD90BC90539711
:10A7C00075016401C418D508E608F7080E94EFB5C2
:10A7D000C61AD70AE80AF90AF7FE6BC020E030E093
:10A7E000A90169817A818B819C810E9480B588232F
:10A7F00009F447C029813A814B815C81CA01B901C2
:10A800000E94A7B46B017C01C501B4010E9420B66F
:10A810009B01AC01C701B6010E9455B86B017C01D8
:10A8200029853A854B855C85CA01B9010E9455B8D6
:10A830009B01AC01C701B6010E94A6B46B017C016B
:10A840002D813E814F815885CA01B9010E9455B8BA
:10A850009B01AC01C701B6010E94A7B46B017C014A
:10A8600020E030E040E850E469817A818B819C816E
:10A870000E9455B89B01AC01C701B6010E9487B583
:10A8800003C060E070E0CB010E946DB50E94EFB59F
:10A890002B013C0197FF03C0412C512C320148147D
:10A8A00059046A047B0410F024013501C12CD12C19
:10A8B00076018FB7F894F101E45BFF4F908191111D
:10A8C00021C0F101448A558A668A778AC40CD51C56
:10A8D000E61CF71CD101C08ED18EE28EF38E2D8541
:10A8E0003E854F85588924AF35AF46AF57AFA05C42
:10A8F000BF4F29893A894B895C892D933D934D93AC
:10A900005C9313978FBF68960FB6F894DEBF0FBEA7
:10A91000CDBFDF91CF911F910F91FF90EF90DF900E
:10A92000CF90BF90AF909F908F907F906F905F90EF
:10A930004F903F902F9008954F925F926F927F9229
:10A94000AF92BF92CF92DF92EF92FF920F931F933D
:10A95000CF93DF93EB017A01209709F458C041159A
:10A96000510509F454C0AAA4BBA40CA51DA59501CA
:10A97000A8016EA17FA188A599A50E9480B5882312
:10A9800009F445C08FA981113AC0F70146A057A02C
:10A9900060A471A4A3019201B501C8010E9483B70C
:10A9A00018166CF5A3019201C301B2010E9455B8BB
:10A9B0006B017C018AA99BA9ACA9BDA9BC01CD01F1
:10A9C00090589B01AC010E94A7B42EA53FA548A9B1
:10A9D00059A90E9455B89B01AC01C701B6010E945C
:10A9E000A6B40E94C2B86B017C019B01AC01B50109
:10A9F000C8010E9480B587FD02C056018701A501EC
:10AA0000B8014EA35FA368A779A781E08EABDF9161
:10AA1000CF911F910F91FF90EF90DF90CF90BF905B
:10AA2000AF907F906F905F904F900895DF92EF927C
:10AA3000FF920F931F93CF93DF938091230C8FB7D7
:10AA4000F894E090220C8FBF8091230C90E08E1937
:10AA500091098F7099270497F4F01091230C1350EB
:10AA60001F7040E050E000E0F12C8DE4D82E1E1560
:10AA700091F0111101C010E11150D19EE00111249B
:10AA8000CC5DD34F602F7F2DCE0156DF402F5F2D41
:10AA90000C2FFD2EECCFDF91CF911F910F91FF90E6
:10AAA000EF90DF9008954F925F926F927F92AF92F6
:10AAB000BF92CF92DF92EF92FF920F931F93CF93AB
:10AAC000DF938C01EB01009709F453C0FC0187A9C7
:10AAD00081114FC046A057A060A471A4AEA0BFA032
:10AAE000C8A4D9A49501A601C301B2010E9480B5F2
:10AAF00087FF3FC0A3019201C301B2010E9455B874
:10AB00002B013C01F80182A993A9A4A9B5A9BC0114
:10AB1000CD0190589B01AC010E94A7B4F80126A575
:10AB200037A540A951A90E9455B89B01AC01C301AA
:10AB3000B2010E94A6B40E94C2B87B018C019B01A5
:10AB4000AC01B501C6010E9480B587FF02C0750146
:10AB500086019701A801B501C6010E9480B588232E
:10AB600041F0A701B8014EA35FA368A779A781E0D0
:10AB70008EABDF91CF911F910F91FF90EF90DF90FF
:10AB8000CF90BF90AF907F906F905F904F9008955F
:10AB9000EF92FF920F931F93CF93DF93F090220CCD
:10ABA00000E010E080E090E02DE4E22E2091230C04
:10ABB000F21689F0EF9CE0011124CC5DD34FAE0179
:10ABC000B80171DF81E08F0D803109F480E0F82E4B
:10ABD000C8018E01EBCF40E050E0B801DF91CF918A
:10ABE0001F910F91FF90EF905ECF4F925F926F9207
:10ABF0007F928F929F92AF92BF92CF92DF92EF920D
:10AC0000FF920F931F93CF93DF939090220CC0E09D
:10AC1000D0E03DE4832E892D992787FD90952091E2
:10AC2000230C30E082179307B9F1889E5001899E6A
:10AC3000B00C1124C5018C5D934F5C01209729F164
:10AC40008EA9811104C0F50186A98823F1F0CAA05C
:10AC5000DBA0ECA0FDA0A7019601F50166A177A1FC
:10AC600080A591A50E9487B52B013C01A701960103
:10AC70006EA17FA188A599A50E9487B5AB01BC01F3
:10AC800093018201CE0181DC1EAA9394F0E19F1210
:10AC900001C0912CE501BFCF2097E9F0CAA0DBA04D
:10ACA000ECA0FDA0A70196016DEC7CEC8CE49DE38B
:10ACB0000E9487B54B015C01A70196016EA17FA19F
:10ACC00088A599A50E9487B5AB01BC0195018401B7
:10ACD000CE015BDC1EAADF91CF911F910F91FF90F7
:10ACE000EF90DF90CF90BF90AF909F908F907F902C
:10ACF0006F905F904F90089599DE4ADF76CF109263
:10AD0000230C1092220C80E1E9E0F1E1DF011D92B9
:10AD10008A95E9F71092F9101092FA101092FB1030
:10AD20001092FC101092FD101092FE101092FF1065
:10AD30001092001110920111109202111092031141
:10AD40001092041110920511109206111092071121
:10AD5000109208111092F5101092F6101092F71040
:10AD60001092F81008954F925F926F927F928F9297
:10AD70009F92AF92BF92CF92DF92EF92FF920F938A
:10AD80001F93CF93DF938091F410882309F4EFC0D1
:10AD9000C0904702D0904802E0904902F0904A02E9
:10ADA00060913C1270913D12882777FD8095982F15
:10ADB0000E9422B620E030E040E050E40E94A7B4B8
:10ADC0009601A7010E9480B587FDD1C05090220C4A
:10ADD000612C712C00E010E04DE4442E8091230C96
:10ADE000581609F453C0852D90E0489EF001499E05
:10ADF000F00D1124EC5DF34F40815181628173812C
:10AE0000452B462B472B81F4448155816681778100
:10AE1000452B462B472B41F4408551856285738530
:10AE2000452B462B472B69F1489EE001499ED00DEA
:10AE30001124CC5DD34F6C857D858E859F850E94C6
:10AE400022B64B015C01688979898A899B890E94B5
:10AE500020B69B01AC01C501B4010E9487B52AA1AF
:10AE60003BA14CA15DA10E9455B85B01D82FC92F11
:10AE70009301A8010E9483B718161CF435010D2F09
:10AE80001C2F5394852D8F70582EA8CF20914302EC
:10AE9000309144024091450250914602B301C801ED
:10AEA0000E9455B89B01AC01B601C7010E94A7B42E
:10AEB0008B01D82FC92F9601A7010E9480B587FD6D
:10AEC00003C06801ED2EFC2E00914B0210914C0244
:10AED000D0914D02C0914E0298014D2F5C2FB601CA
:10AEE000C7010E9483B718161CF08601DE2DCF2DF6
:10AEF00080901E0C90901F0CA090200CB090210C04
:10AF000098014D2F5C2FC501B4010E9483B718161C
:10AF1000D4F420E037ED43EA5CE3B8018D2F9C2F99
:10AF20000E9455B86B017C0128E431EE4AE75FE3EB
:10AF3000C501B4010E9455B8A70196010E94A7B4AB
:10AF40008B01D82FC92FC801AD2FBC2F80931E0CA9
:10AF500090931F0CA093200CB093210CB8018D2F5F
:10AF60009C2F0E94EFB570933D1260933C12DF91CD
:10AF7000CF911F910F91FF90EF90DF90CF90BF90F6
:10AF8000AF909F908F907F906F905F904F900895BB
:10AF900060919B089091220C8091230C981781F06E
:10AFA0008091220C9DE4899FF0011124E459F34F14
:10AFB00060819091230C891719F08F5F8F70F9CF02
:10AFC00070E089E00E9438AFCECE2F923F924F9230
:10AFD0005F926F927F928F929F92AF92BF92CF9229
:10AFE000DF92EF92FF920F931F93CF93DF93CDB732
:10AFF000DEB7CC56D1090FB6F894DEBF0FBECDBF79
:10B000002C015B014A013901EBAAFFAAD9AEC8AEF7
:10B010002091230C2F5F21962FAF2197203119F417
:10B0200021961FAE219721963FAD2197E32EFF2455
:10B03000E7FCF0948091220C90E08E159F0539F486
:10B040000E949D6C0E9471230E941C87F3CF209167
:10B050005511309156114091571150915811D2010C
:10B060006D917D918D919C910E9455B80E9425B85B
:10B0700069966CAF7DAF8EAF9FAF699720915911E4
:10B0800030915A1140915B1150915C11F501608132
:10B090007181828193810E9455B80E9425B86D9676
:10B0A0006CAF7DAF8EAF9FAF6D9720915D113091EA
:10B0B0005E1140915F1150916011D4016D917D91AD
:10B0C0008D919C910E9455B80E9425B8A1966CAFB5
:10B0D0007DAF8EAF9FAFA19720916111309162112A
:10B0E0004091631150916411F301608171818281FB
:10B0F00093810E9455B80E9425B86CAF7DAF8EAF8A
:10B100009FAF8091151190911611A0911711B091D8
:10B1100018112CAD3DAD4EAD5FAD281739074A076C
:10B120005B0709F4B3C0E0919D0834E0E39FF001B0
:10B130001124E25DFD4E20913F023091400240918A
:10B1400041025091420260817181828193810E940B
:10B1500080B587FF2DC08CAD9DADAEADBFAD8093EA
:10B16000151190931611A0931711B0931811E0EDDB
:10B17000F7E08491882341F09091C00095FFFCCFC7
:10B180008093C6003196F5CFE6EBF7E084918823F3
:10B1900041F09091C00095FFFCCF8093C60031969E
:10B1A000F5CF8091C00085FFFCCF8AE08093C60078
:10B1B0008091151190911611A0911711B09118114D
:10B1C0002CAD3DAD4EAD5FAD281B390B4A0B5B0B73
:10B1D000CA01B90157FF07C0909580957095619598
:10B1E0007F4F8F4F9F4F0E9422B66B017C01609171
:10B1F000FC087091FD088091FE089091FF08680F8F
:10B20000791F882777FD8095982F0E9422B620917C
:10B2100061113091621140916311509164110E944B
:10B2200055B89B01AC01C701B6010E9483B718163F
:10B230006CF58CAD9DADAEADBFAD80931511909307
:10B240001611A0931711B0931811E0EDF7E0849157
:10B25000882341F09091C00095FFFCCF8093C600F9
:10B260003196F5CFE8E9F7E08491882341F0909199
:10B27000C00095FFFCCF8093C6003196F5CF80913A
:10B28000C00085FFFCCF8AE08093C6008091230C2C
:10B290009DE4899F10011124D101AC5DB34F1D01C4
:10B2A000FD01E45BFF4F10822091091130910A11DA
:10B2B00040910B1150910C112BA33CA34DA35EA305
:10B2C00069964CAC5DAC6EAC7FAC6997421A530A80
:10B2D000640A750A77FE08C0709460945094409494
:10B2E000411C511C611C711CD1014D925D926D92EB
:10B2F0007C92139720910D1130910E1140910F11F6
:10B30000509110112FA338A749A75AA76D968CAC5E
:10B310009DACAEACBFAC6D97821A930AA40AB50A75
:10B32000B7FE08C0B094A09490948094811C911CA6
:10B33000A11CB11CD10114968D929D92AD92BC922C
:10B3400017972091111130911211409113115091C2
:10B3500014112FA738AB49AB5AABA196CCACDDACDE
:10B36000EEACFFACA197C21AD30AE40AF50AF7FEC5
:10B3700008C0F094E094D094C094C11CD11CE11C8E
:10B38000F11CD1011896CD92DD92ED92FC921B97A3
:10B3900020911511309116114091171150911811EB
:10B3A0002BA73CA74DA75EA72CAD3DAD4EAD5FAD25
:10B3B0008BA59CA5ADA5BEA5281B390B4A0B5B0B25
:10B3C00057FF07C050954095309521953F4F4F4FFF
:10B3D0005F4FA0912B02B0912C020E949FB924E6EE
:10B3E00030E040E050E00E9473B9D1011C962D93EB
:10B3F0003D934D935C931F97C814D904EA04FB0452
:10B4000014F475016401C216D306E406F50614F4BB
:10B4100069017A01D301C2014C145D046E047F04FA
:10B4200014F4D701C601F101808B918BA28BB38BF1
:10B430000697A105B10508F445C7E85BFF4F809169
:10B440009B0890919C08AA2797FDA095BA2F80830E
:10B450009183A283B38369962CAD3DAD4EAD5FADB4
:10B4600069978BA19CA1ADA1BEA1281739074A07F6
:10B470005B0724F0D10190961C9203C081E0F1019A
:10B4800080A36D962CAD3DAD4EAD5FAD6D978FA198
:10B4900098A5A9A5BAA5281739074A075B073CF460
:10B4A000D10190968C919097826090968C93A19602
:10B4B0002CAD3DAD4EAD5FADA1978FA598A9A9A9C3
:10B4C000BAA9281739074A075B073CF4D1019096BF
:10B4D0008C919097846090968C932CAD3DAD4EAD41
:10B4E0005FAD8BA59CA5ADA5BEA5281739074A075A
:10B4F0005B073CF4D10190968C9190978860909670
:10B500008C93E8ADF9AD8081D10191968C9345285B
:10B510004628472809F05F98F10184819581A6812A
:10B52000B781892B8A2B8B2B09F08A98F1018085B2
:10B530009185A285B385892B8A2B8B2B41F09FB7F0
:10B54000F894809108018E7F809308019FBFF101DC
:10B5500084859585A685B785892B8A2B8B2B11F041
:10B5600012984798D1011C962D913D914D915C9177
:10B570001F9725962CAF3DAF4EAF5FAF2597232B7E
:10B58000242B252BF1F4B0912911BBA3E0912A11B2
:10B59000EFA3F0912B11FFA720912C112BA72B2F9C
:10B5A0003E2F4F2F5BA56BA97FA9C8010E9480B5D4
:10B5B00087FD18C03BA93BA34FA94FA30FA71BA70B
:10B5C00011C0509141115BA3809142118FA39091C2
:10B5D00043119FA7A0914411ABA7252F382F492FC6
:10B5E0005A2FE1CF8091091190910A11A0910B116E
:10B5F000B0910C1169962CAD3DAD4EAD5FAD699724
:10B60000281B390B4A0B5B0BCA01B9010E9422B6F9
:10B610002091551130915611409157115091581168
:10B620000E9487B52B013C01698B7A8B8B8B9C8B9D
:10B6300080910D1190910E11A0910F11B0911011E8
:10B640006D962CAD3DAD4EAD5FAD6D97281B390BA2
:10B650004A0B5B0BCA01B9010E9422B62091591115
:10B6600030915A1140915B1150915C110E9487B545
:10B670004B015C016D8B7E8B8F8B988F80911111AC
:10B6800090911211A0911311B0911411A1962CADAB
:10B690003DAD4EAD5FADA197281B390B4A0B5B0B3F
:10B6A000CA01B9010E9422B620915D1130915E114C
:10B6B00040915F11509160110E9487B56B017C0130
:10B6C000698F7A8F8B8F9C8F8091151190911611B5
:10B6D000A0911711B09118112CAD3DAD4EAD5FADDD
:10B6E000281B390B4A0B5B0BCA01B9010E9422B619
:10B6F0002091611130916211409163115091641158
:10B700000E9487B56BAB7CAB8DAB9EAB60912B027F
:10B7100070912C02882777FD8095982F0E9422B681
:10B720009B01AC016BA97CA98DA99EA90E9455B86B
:10B7300020E030E048EC52E40E9487B56D8F7E8FA8
:10B740008F8F98A3D1012D913D914D915C911397CD
:10B7500028AF39AF4AAF5BAF2630310541055105FF
:10B76000FCF414960D911D912D913C911797063084
:10B77000110521053105A4F418960D911D912D9107
:10B780003C911B9706301105210531054CF4DC0175
:10B79000CB01BF77F10186A797A7A0ABB1AB25C0BE
:10B7A000C301B2010E9400B92B013C01C501B401E3
:10B7B0000E9400B99B01AC01C301B2010E94A7B471
:10B7C0004B015C01C701B6010E9400B99B01AC01AD
:10B7D000C501B4010E94A7B40E94C2B8D1019E96CF
:10B7E0006D937D938D939C93D197D1019E962D91CE
:10B7F0003D914D915C91D19765962CAF3DAF4EAF89
:10B800005FAF659760E070E080E89FE30E9487B5D6
:10B810009B01AC016BA17FA18FA59BA50E9455B890
:10B820002B013C019091230C8091220CE92FF0E038
:10B83000E81BF109EF70FF27F8ABEFA7A301920116
:10B8400060E074E284E799E40E9487B50E9425B81D
:10B850006B017C012FA538A9223031050CF442C0C0
:10B860004901AA2497FCA094BA2CC501B4010E94F6
:10B8700022B620E030E040E051E40E9480B587FF2E
:10B8800031C08091751190917611A0917711B0918E
:10B890007811C816D906EA06FB0620F5BC01CD01D1
:10B8A0006C197D098E099F09660F771F881F991FE4
:10B8B000A50194010E9451B9CA01B9010E9420B6A4
:10B8C0000E9425B86C0D7D1D8E1D9F1D0E9420B607
:10B8D0009B01AC0160E074E284E799E40E9487B5C3
:10B8E0002B013C01A301920165966CAD7DAD8EAD3F
:10B8F0009FAD65970E9455B829966CAF7DAF8EAF0E
:10B900009FAF2997D10192966D937D938D939C93D0
:10B91000959750966D917D918D919C9153970E9432
:10B9200020B66BA37CA38DA39EA3A30192010E94CA
:10B9300055B80E946DB50E94F4B56B017C01F10110
:10B9400060AF71AF82AF93AF8E010F5E1F4F25E6E0
:10B9500031E161963FAF2EAF6197AE014F5D5F4F12
:10B960005AA349A3CE0101962F969FAF8EAF2F9772
:10B970001FA21BA690E89BABAFE3AFABF8016191B0
:10B980007191819191918F01A30192010E9455B80B
:10B990002F96AEADBFAD2F976D937D938D939D93F5
:10B9A0002F96BFAFAEAF2F979B01AC015F772D965F
:10B9B0002CAF3DAF4EAF5FAF2D976196AEADBFAD33
:10B9C00061978D909D90AD90BD906196BFAFAEAFE9
:10B9D0006197A50194012D966CAD7DAD8EAD9FADA7
:10B9E0002D970E9483B71816F4F42D962CAD3DAD1B
:10B9F0004EAD5FAD2D97C501B4010E9487B5B62E3F
:10BA0000A72E982E892E262F372F482F592F6FA11A
:10BA10007BA58BA99FA90E9480B587FD04C0BFA20A
:10BA2000ABA69BAA8FAAE9A1FAA10E171F0709F0DE
:10BA3000A5CF20E030E040E85FE36FA17BA58BA9B4
:10BA40009FA90E9480B587FF3FC05E01F1E1AF0E64
:10BA5000B11C8E010F5F1F4F2FA13BA54BA95FA902
:10BA6000D8016D917D918D919C910E9455B8F801FE
:10BA700061937193819391938F01EA15FB0561F7AF
:10BA80002FA13BA54BA95FA929966CAD7DAD8EADCD
:10BA90009FAD29970E9455B8D10192966D937D93E1
:10BAA0008D939C939597C701B6010E9420B62FA154
:10BAB0003BA54BA95FA90E9455B80E94F4B5F101BE
:10BAC00060AF71AF82AF93AF65962CAD3DAD4EAD1B
:10BAD0005FAD65976BA17CA18DA19EA10E9487B5EA
:10BAE0006B017C0128AD39AD4AAD5BAD232B242B16
:10BAF000252B59F5F10184819581A681B781892B88
:10BB00008A2B8B2B11F580859185A285B385892B96
:10BB10008A2B8B2BD1F42091391130913A1140911D
:10BB20003B1150913C11C701B6010E9455B80E94CB
:10BB30006DB581010C5B1F4F0E94F4B5D8016D9368
:10BB40007D938D939C931397F6C020913D11309176
:10BB50003E1140913F1150914011C701B6010E9422
:10BB600055B80E946DB50E94F4B581010C5B1F4F62
:10BB7000F801608371838283938340901911509000
:10BB80001A1160901B1170901C110E9420B64B017D
:10BB90005C0168AD79AD8AAD9BAD0E9422B69B0178
:10BBA000AC01C501B4010E9455B82BA13CA14DA127
:10BBB0005EA10E9487B54B015C01C301B2010E94E6
:10BBC00020B69B01AC01C501B4010E9483B71816D1
:10BBD00034F4D8014D925D926D927C92139740900F
:10BBE0001D1150901E1160901F1170902011F801CE
:10BBF00060817181828193810E9420B64B015C013A
:10BC0000D10114966D917D918D919C9117970E9411
:10BC100022B69B01AC01C501B4010E9455B82BA10D
:10BC20003CA14DA15EA10E9487B54B015C01C301FF
:10BC3000B2010E9420B69B01AC01C501B4010E9473
:10BC400083B718162CF4F801408251826282738205
:10BC50004090251150902611609027117090281166
:10BC600081010C5B1F4FD8016D917D918D919C914D
:10BC70000E9420B64B015C0125966CAD7DAD8EAD6A
:10BC80009FAD25970E9422B69B01AC01C501B4016E
:10BC90000E9455B82BA13CA14DA15EA10E9487B581
:10BCA0004B015C01C301B2010E9420B69B01AC01B3
:10BCB000C501B4010E9483B718162CF4F801408224
:10BCC00051826282738240902111509022116090C3
:10BCD000231170902411D8016D917D918D919C91CB
:10BCE0000E9420B64B015C01F1016085718582855F
:10BCF00093850E9422B69B01AC01C501B4010E944C
:10BD000055B82BA13CA14DA15EA10E9487B54B0166
:10BD10005C01C301B2010E9420B69B01AC01C501C8
:10BD2000B4010E9483B7181634F4D8014D925D9285
:10BD30006D927C921397F101EC5BFF4F60817181F2
:10BD4000828193810E9420B64B015C01A70196017C
:10BD50000E9487B5A5966CAF7DAF8EAF9FAFA597BC
:10BD6000F10162AB73AB84AB95AB2DEB37E346E0EF
:10BD700051E4C501B4010E9455B80E94EFB5D1014C
:10BD80005C966D937D938D939C935F97C0903511D6
:10BD9000D0903611E0903711F090381120E030E06B
:10BDA00040E05FE3C701B6010E9455B86BA37FA3D3
:10BDB0008C0129853A854B855C85A9962CAF3DAFD2
:10BDC0004EAF5FAFA9978091311190913211A09140
:10BDD0003311B091341125968CAF9DAFAEAFBFAF8C
:10BDE000259720E030E040E05FE3BC01CD010E94F8
:10BDF00055B8B62EA72E982E892EA9966CAD7DAD7E
:10BE00008EAD9FADA9979F772B2D3A2D492D582D9B
:10BE10000E9483B718167CF42B2D3A2D492D582DEE
:10BE20006BA17FA1C8010E9480B587FD04C0BBA2A1
:10BE3000AFA2092D182D2D853E854F855889AD96C9
:10BE40002CAF3DAF4EAF5FAFAD9780912D1190916C
:10BE50002E11A0912F11B091301129968CAF9DAF6A
:10BE6000AEAFBFAF299720E030E040E05FE3BC0118
:10BE7000CD010E9455B8B62EA72E982E892EAD96CC
:10BE80006CAD7DAD8EAD9FADAD979F772B2D3A2DCF
:10BE9000492D582D0E9483B718167CF42B2D3A2D6E
:10BEA000492D582D6BA17FA1C8010E9480B587FD47
:10BEB00004C0BBA2AFA2092D182DD1019296BC914E
:10BEC000BBA7F101F3A1FBABD1019496BC91BFAB31
:10BED000F101F5A1F8AF2BA53BA94B2F5F2F6BA16B
:10BEE0007FA1C8010E9480B587FD06C02BA52BA3AA
:10BEF0003BA93FA30FA918AD4FA558A94230510542
:10BF00000CF409C15091F5105FA78091F6102A96A4
:10BF10008FAF2A979091F7102E969FAF2E97A091F2
:10BF2000F8106096AFAF609727E137EB41ED58E32B
:10BF30006FA5782F892F9A2F0E9483B718160CF0BF
:10BF4000EAC02091F9103091FA104091FB10509105
:10BF5000FC1069817A818B819C810E94A6B42B019F
:10BF60003C012091FD103091FE104091FF10509146
:10BF700000116D817E818F8198850E94A6B44B014E
:10BF80005C01A3019201C301B2010E9455B82B01CB
:10BF90003C01A5019401C501B4010E9455B89B0163
:10BFA000AC01C301B2010E94A7B40E94C2B84B0108
:10BFB0005C01A70196010E9483B718164CF4A501F5
:10BFC0009401C701B6010E9487B55B014C0106C010
:10BFD000A12CB12C50E8852E6FE3962E20910111F3
:10BFE000309102114091031150910411A9966CAD4A
:10BFF0007DAD8EAD9FADA9970E94A6B46B017C016B
:10C00000E894F7F825962CAD3DAD4EAD5FAD259784
:10C01000C701B6010E9483B71816E4F4A701960180
:10C0200025966CAD7DAD8EAD9FAD25970E9487B5F1
:10C03000F62EE72ED82EC92E262F372F482F592F10
:10C04000B501C4010E9480B587FD04C0AF2CBE2C91
:10C050008D2C9C2C209105113091061140910711D7
:10C0600050910811AD966CAD7DAD8EAD9FADAD9785
:10C070000E94A6B46B017C01E894F7F829962CADD8
:10C080003DAD4EAD5FAD2997C701B6010E9483B7A4
:10C090001816E4F4A701960129966CAD7DAD8EAD1E
:10C0A0009FAD29970E9487B5F62EE72ED82EC92E70
:10C0B000262F372F482F592FB501C4010E9480B574
:10C0C00087FD04C0AF2CBE2C8D2C9C2C9501A401A7
:10C0D0006BA57BA98FA998AD0E9455B84B015C0157
:10C0E0009B01AC016FA52A967FAD2A972E968FAD46
:10C0F0002E9760969FAD60970E9480B587FF0EC017
:10C100008FA42A969FAC2A972E96AFAC2E97609656
:10C11000BFAC609703C08BA09FA05801C401D5019C
:10C12000F10182A793A7A4A7B5A7A5966CAD7DAD95
:10C130008EAD9FADA59790589B01AC010E94A7B40E
:10C1400065962CAD3DAD4EAD5FAD65970E9455B87F
:10C150009B01AC016BE077ED83E29BE30E94A6B408
:10C160000E94C2B87B01D82EC92E9B01482F592F9F
:10C17000B401C5010E9480B587FD03C04701AD2C05
:10C18000BC2CC401D501F10186A397A3A0A7B1A738
:10C1900097014D2D5C2D6BA57BA98FA998AD0E94B1
:10C1A00080B518162CF081E0D101D7968C9302C08F
:10C1B000F10117AA81E0D101D6968C9380E1FE01AE
:10C1C0003196A9EFB0E101900D928A95E1F78BA528
:10C1D0009BA9AFA9B8AD8093F5109093F610A093EA
:10C1E000F710B093F8109C01AD016BA17FA1C801BD
:10C1F0000E9487B56B017C012BA53BA94FA958ADC7
:10C20000B401C5010E9487B5AB01BC01970186014D
:10C21000C1010E94C5522196BFAD2197B093230C56
:10C2200069962CAD3DAD4EAD5FAD69972093091178
:10C2300030930A1140930B1150930C116D968CADF5
:10C240009DADAEADBFAD6D9780930D1190930E1166
:10C25000A0930F11B0931011A1962CAD3DAD4EAD32
:10C260005FADA197209311113093121140931311D8
:10C27000509314118CAD9DADAEADBFAD8093151133
:10C2800090931611A0931711B09318110E947C5629
:10C29000C459DF4F0FB6F894DEBF0FBECDBFDF919C
:10C2A000CF911F910F91FF90EF90DF90CF90BF90B3
:10C2B000AF909F908F907F906F905F904F903F9046
:10C2C0002F90D2C1C459DF4F0FB6F894DEBF0FBE16
:10C2D000CDBFDF91CF911F910F91FF90EF90DF9035
:10C2E000CF90BF90AF909F908F907F906F905F9016
:10C2F0004F903F902F900895EF92FF920F931F93CE
:10C30000CF93DF937B018A01E90120915511309190
:10C3100056114091571150915811FC016081718163
:10C32000828193810E9455B80E9425B860930911BB
:10C3300070930A1180930B1190930C112091591155
:10C3400030915A1140915B1150915C11F70160815D
:10C350007181828193810E9455B80E9425B86093B3
:10C360000D1170930E1180930F1190931011209165
:10C370005D1130915E1140915F1150916011F80193
:10C3800060817181828193810E9455B80E9425B895
:10C3900060931111709312118093131190931411E3
:10C3A000209161113091621140916311509164119B
:10C3B000688179818A819B810E9455B80E9425B845
:10C3C00060931511709316118093171190931811A3
:10C3D00025E131E141E151E16DE071E189E091E177
:10C3E0000E946E6A1092F5101092F6101092F710DB
:10C3F0001092F8101092F9101092FA101092FB108F
:10C400001092FC101092FD101092FE101092FF106E
:10C41000109200111092011110920211109203114A
:10C42000109204111092051110920611109207112A
:10C4300010920811DF91CF911F910F91FF90EF9013
:10C4400008952091611130916211409163115091D2
:10C450006411FC0160817181828193810E9455B8D1
:10C460000E9425B8609315117093161180931711CF
:10C470009093181185E191E10C94AA6A60933F02B0
:10C480007093400280934102909342020895CF92AC
:10C49000DF92EF92FF920F931F93CF93DF9300D021
:10C4A0001F92CDB7DEB7F5E4CF2EF1E1DF2EA5E583
:10C4B000EA2EA1E1FA2E09E111E1F60161917191F3
:10C4C000819191916F01F7012191319141915191A8
:10C4D0007F0129833A834B835C830E9420B62981A4
:10C4E0003A814B815C810E9455B80E94F4B5F801F5
:10C4F00061937193819391938F01F5E5CF16F1E1EB
:10C50000DF06D9F60F900F900F900F90DF91CF912B
:10C510001F910F91FF90EF90DF90CF900895809141
:10C520008E11811109C080918D11811105C08091FA
:10C530008C11811101C00895E1E2F0E1849188231A
:10C5400041F09091C00095FFFCCF8093C6003196DA
:10C55000F5CFE2E1F8E08491882341F09091C000AA
:10C5600095FFFCCF8093C6003196F5CF80918E1158
:10C570008823F1F060918F11709190118091911149
:10C58000909192110E9422B620915511309156112E
:10C5900040915711509158110E9487B5AB01BC01D1
:10C5A0008EE098E00E9412198EEF97E00E940F86AD
:10C5B00080918D118823F1F0609193117091941105
:10C5C00080919511909196110E9422B62091591157
:10C5D00030915A1140915B1150915C110E9487B5C6
:10C5E000AB01BC018AEF97E00E9412198AEE97E036
:10C5F0000E940F8680918C118823F1F06091971131
:10C60000709198118091991190919A110E9422B67F
:10C6100020915D1130915E1140915F115091601138
:10C620000E9487B5AB01BC0186EE97E00E9412190B
:10C6300086ED97E00E940F868091C00085FFFCCFB9
:10C640008AE08093C60010928E1110928D11109284
:10C650008C11089510928E1110928D1110928C11E0
:10C660000895809353020895EFE6F0E080818260A0
:10C67000808308951F920F920FB60F9211240BB66C
:10C680000F920F931F932F933F934F935F936F934B
:10C690007F938F939F93AF93BF93EF93FF9380917B
:10C6A000BF119091C011892B09F086C19091230C84
:10C6B0008091220C981771F0E091220C8DE4E89F94
:10C6C000F0011124EC5DF34FDF01A45BBF4F81E06B
:10C6D0008C9302C0E0E0F0E0F093C011E093BF1152
:10C6E000309709F463C1DF01A45BBF4F81E08C93F5
:10C6F0001092A2111092A3111092A4111092A511E0
:10C7000060AD71AD61349CE9790728F461329EE433
:10C71000790748F002C060E47CE9769567957695E4
:10C72000679584E007C0613197E2790730F076952C
:10C73000679582E080939F1107C080939F116032BC
:10C74000710510F460E270E060527109611588E0D3
:10C750007807D0F0872F9927880F991F880F991F86
:10C760008F5D934FFC01329645915491AA27659FA6
:10C770009001649F210D3A1F06942A1F3A1F11242D
:10C78000FC01859194911DC0CB01969587958C7F76
:10C790008F5D974FFC01459154910296FC01859164
:10C7A0009491FB01E770FF278E9F90018F9F300DC2
:10C7B0009E9F300D1124E3E036952795EA95E1F729
:10C7C000CA01821B930B84369105A0F4EAEEF3E0D4
:10C7D0008191882339F09091C00095FFFCCF809320
:10C7E000C600F6CF4AE050E080E795E00E94EC16E4
:10C7F00084E690E090939E1180939D1180919F110B
:10C80000992787FD909590939C1180939B11E091BF
:10C81000BF11F091C01164AD75AD7093A11160931B
:10C82000A01161349CE9790728F461328EE478071D
:10C8300048F002C060E47CE9769567957695679547
:10C8400084E007C0613197E2790730F0769567950B
:10C8500082E080939F1108C081E080939F11603235
:10C86000710510F460E270E060527109611588E0B2
:10C870007807E0F0872F9927880F991F880F991F55
:10C880008F5D934FFC01329625913491AA27639FC7
:10C89000A001629F410D5A1F06944A1F5A1F11247E
:10C8A000FC0125913491241B350B1EC0CB019695BC
:10C8B00087958C7F8F5D974FFC012591349102966F
:10C8C000FC0145915491FB01E770FF274E9FC00189
:10C8D0004F9F900D5E9F900D1124F3E096958795E4
:10C8E000FA95E1F7281B390B24363105A0F4EAEE5E
:10C8F000F3E08191882339F09091C00095FFFCCF3F
:10C900008093C600F6CF4AE050E080E795E00E94B1
:10C91000EC1624E630E0C901A0E0B0E08093A61157
:10C920009093A711A093A811B093A91130938900F7
:10C9300020938800E091BF11F091C0118089918906
:10C94000A289B389B695A79597958795B095A09537
:10C95000909581959F4FAF4FBF4F8093BA119093A1
:10C96000BB11A093BC11B093BD118093B6119093ED
:10C97000B711A093B811B093B9118093B2119093ED
:10C98000B311A093B411B093B5118093AE119093ED
:10C99000AF11A093B011B093B1111092AA111092DF
:10C9A000AB111092AC111092AD1106C080ED97E062
:10C9B0009093890080938800E091BF11F091C0119D
:10C9C000309709F4DCC480A18093BE1180FF41C080
:10C9D000899A8FEF80934F02809153028823E9F167
:10C9E0002CB131E025FB222720F9232779F1809112
:10C9F0008B11882359F1E091BF11F091C011808112
:10CA00009181A281B381181619061A061B06F4F447
:10CA10008091791190917A11A0917B11B0917C1144
:10CA200080938F1190939011A0939111B0939211D4
:10CA300030938E1180899189A289B3898093AA113C
:10CA40009093AB11A093AC11B093AD1120938B11C7
:10CA500004C0899881E080934F028091BE1181FFCC
:10CA600041C08F9A8FEF80935002809153028823A8
:10CA7000E9F12091030131E026952170232779F116
:10CA800080918A11882359F1E091BF11F091C01172
:10CA900084819581A681B781181619061A061B068E
:10CAA000F4F480917D1190917E11A0917F11B0914D
:10CAB00080118093931190939411A0939511B0934A
:10CAC000961130938D1180899189A289B3898093C1
:10CAD000AA119093AB11A093AC11B093AD11209318
:10CAE0008A1104C08F9881E0809350028091BE111A
:10CAF0009FB782FF48C0F89480910B018D7F80938F
:10CB00000B019FBF8FEF80935102809153028823C6
:10CB100009F443C029B131E023FB222720F9232760
:10CB200079F180918911882359F1E091BF11F09139
:10CB3000C01180859185A285B385181619061A063D
:10CB40001B06F4F48091811190918211A0918311C0
:10CB5000B09184118093971190939811A09399119B
:10CB6000B0939A1130938C1180899189A289B389ED
:10CB70008093AA119093AB11A093AC11B093AD1117
:10CB8000209389110AC0F89480910B0182608093F0
:10CB90000B019FBF81E0809351028091BE11E09113
:10CBA000BF11F091C01183FF08C081A1813011F441
:10CBB000439801C0169A8FEF07C081A1813011F40C
:10CBC000439A01C0169881E08093520220E0809140
:10CBD0009F1128170CF0C7C18091C00087FF19C0B2
:10CBE0003091C6004091F1055091F205CA010196BD
:10CBF0008F7799276091F3057091F4058617970751
:10CC000041F0FA01EF58FA4F30839093F205809388
:10CC1000F105E091BF11F091C0118091BA1190918E
:10CC2000BB11A091BC11B091BD11408151816281B5
:10CC30007381840F951FA61FB71F8093BA1190931D
:10CC4000BB11A093BC11B093BD11181619061A069A
:10CC50001B06CCF5889AE091BF11F091C01180912C
:10CC6000BA119091BB11A091BC11B091BD11408936
:10CC7000518962897389841B950BA60BB70B80932E
:10CC8000BA119093BB11A093BC11B093BD11409108
:10CC90004F028091791190917A11A0917B11B091FE
:10CCA0007C11552747FD5095652F752F840F951FD3
:10CCB000A61FB71F8093791190937A11A0937B11CF
:10CCC000B0937C118898E091BF11F091C0118091D0
:10CCD000B6119091B711A091B811B091B9114481DA
:10CCE000558166817781840F951FA61FB71F80939A
:10CCF000B6119093B711A093B811B093B91118164B
:10CD000019061A061B06CCF58E9AE091BF11F09118
:10CD1000C0118091B6119091B711A091B811B09146
:10CD2000B9114089518962897389841B950BA60BBF
:10CD3000B70B8093B6119093B711A093B811B0932D
:10CD4000B9114091500280917D1190917E11A09176
:10CD50007F11B0918011552747FD5095652F752F94
:10CD6000840F951FA61FB71F80937D1190937E118E
:10CD7000A0937F11B09380118E98E091BF11F09134
:10CD8000C0118091B2119091B311A091B411B091E2
:10CD9000B5114085518562857385840F951FA61F47
:10CDA000B71F8093B2119093B311A093B411B093B5
:10CDB000B511181619061A061B060CF047C09FB7C6
:10CDC000F89480910B01886080930B019FBFE091E4
:10CDD000BF11F091C0118091B2119091B311A09147
:10CDE000B411B091B5114089518962897389841B4E
:10CDF000950BA60BB70B8093B2119093B311A09330
:10CE0000B411B093B511409151028091811190916C
:10CE10008211A0918311B0918411552747FD50953F
:10CE2000652F752F840F951FA61FB71F8093811143
:10CE300090938211A0938311B09384119FB7F894BB
:10CE400080910B01877F80930B019FBFE091BF1101
:10CE5000F091C0118091AE119091AF11A091B011DD
:10CE6000B091B1114485558566857785840F951FEE
:10CE7000A61FB71F8093AE119093AF11A093B0116E
:10CE8000B093B111181619061A061B060CF043C010
:10CE900081A1813011F4419A01C0149AE091BF112F
:10CEA000F091C0118091AE119091AF11A091B0118D
:10CEB000B091B1114089518962897389841B950BA6
:10CEC000A60BB70B8093AE119093AF11A093B01146
:10CED000B093B111409152028091851190918611C9
:10CEE000A0918711B0918811552747FD5095652F66
:10CEF000752F840F951FA61FB71F809385119093E0
:10CF00008611A0938711B093881181A1813011F40B
:10CF1000419801C014988091AA119091AB11A091F1
:10CF2000AC11B091AD110196A11DB11D8093AA1154
:10CF30009093AB11A093AC11B093AD114091AA1195
:10CF40005091AB116091AC117091AD11E091BF1196
:10CF5000F091C01180899189A289B3894817590736
:10CF60006A077B07B0F04091AA115091AB11609114
:10CF7000AC117091AD11E091BF11F091C011848995
:10CF80009589A689B78984179507A607B70718F466
:10CF9000DAC02F5F1CCE4091A6115091A71160916D
:10CFA000A8117091A911048D158D268D378DAA2792
:10CFB000419FB12D529FC001629F900D619F800DD6
:10CFC000911D429FB00D811D9A1F519FB00D811D73
:10CFD0009A1F609FB00D811D9A1F509FB10D8A1F2F
:10CFE0009A1FB6958A1F9A1F112444AD55AD480F5C
:10CFF000591F5093A1114093A01180AD91ADA2ADE6
:10D00000B3AD60E070E084179507A607B70720F47A
:10D010009093A1118093A0116091A0117091A11122
:10D0200061349CE9790728F461328EE4780748F08E
:10D0300002C060E47CE9769567957695679584E013
:10D0400007C0613197E2790730F07695679582E005
:10D0500080939F1108C081E080939F116032710519
:10D0600010F460E270E060527109611588E07807A1
:10D07000E0F0872F9927880F991F880F991F8F5DE0
:10D08000934FFC01329625913491AA27639FA0010A
:10D09000629F410D5A1F06944A1F5A1F1124FC011A
:10D0A00025913491241B350B1EC0CB019695879595
:10D0B0008C7F8F5D974FFC01259134910296FC0186
:10D0C00045915491FB01E770FF274E9FC0014F9F90
:10D0D000900D5E9F900D112413E0969587951A95FB
:10D0E000E1F7281B390B24363105A0F4EAEEF3E012
:10D0F0008191882339F09091C00095FFFCCF8093F7
:10D10000C600F6CF4AE050E080E795E00E94EC16BA
:10D1100024E630E030938900209388008091A611A6
:10D120009091A711A091A811B091A911820F931FFE
:10D13000A11DB11D8093A6119093A711A093A811D2
:10D14000B093A911F7C04091AA115091AB11609111
:10D15000AC117091AD11808D918DA28DB38D84171E
:10D160009507A607B70708F0D9C04091A2115091C2
:10D17000A3116091A4117091A511048D158D268DB8
:10D18000378DAA27419FB12D529FC001629F900DFC
:10D19000619F800D911D429FB00D811D9A1F519F6F
:10D1A000B00D811D9A1F609FB00D811D9A1F509F69
:10D1B000B10D8A1F9A1FB6958A1F9A1F11242091BC
:10D1C000A0113091A111E05CFF4F2817390718F426
:10D1D0002081318102C0281B390B80819181A2817D
:10D1E000B381A90160E070E0481759076A077B071F
:10D1F00008F49C0121349CE9390728F421328EE49B
:10D20000380748F002C020E43CE93695279536956A
:10D21000279584E007C0213197E2390730F0369531
:10D22000279582E080939F1108C081E080939F1131
:10D230002032310510F420E230E0B901605271096A
:10D24000611588E07807E0F0872F9927880F991FEC
:10D25000880F991F8F5D934FFC0132962591349171
:10D26000AA27639FA001629F410D5A1F06944A1F7F
:10D270005A1F1124FC0125913491241B350B1EC02B
:10D28000CB01969587958C7F8F5D974FFC012591FB
:10D2900034910296FC0145915491FB01E770FF2700
:10D2A0004E9FC0014F9F900D5E9F900D112443E053
:10D2B000969587954A95E1F7281B390B2436310559
:10D2C000A0F4EAEEF3E08191882339F09091C00058
:10D2D00095FFFCCF8093C600F6CF4AE050E080E790
:10D2E00095E00E94EC1624E630E03093890020930C
:10D2F00088008091A2119091A311A091A411B091E6
:10D30000A511820F931FA11DB11D8093A2119093AF
:10D31000A311A093A411B093A5110CC080919D11ED
:10D3200090919E11909389008093880080919B1129
:10D3300080939F114091AA115091AB116091AC1153
:10D340007091AD11E091BF11F091C0118089918968
:10D35000A289B389481759076A077B0780F01092A2
:10D36000C0111092BF119091230C8091220C98173C
:10D3700031F08091220C8F5F8F708093220CFF918F
:10D38000EF91BF91AF919F918F917F916F915F913D
:10D390004F913F912F911F910F910F900BBE0F90C6
:10D3A0000FBE0F901F901895819A879AEAE0F1E0DE
:10D3B0008081826080830E9A3B9A579A5F9A829A04
:10D3C0008A9AE7E0F1E08081816080839FB7F894DA
:10D3D000E8E0F1E08081816080839FBF0A9A129A21
:10D3E0003F9A479A6C98749AE4E0F1E080818E7FCE
:10D3F00080839FB7F894E5E0F1E0808181608083CD
:10D400009FBF6D98759AE4E0F1E080818D7F808305
:10D410009FB7F894E5E0F1E08081826080839FBF50
:10D4200053985B9A809A88985F9A869A8E988A9A7F
:10D43000EAE0F1E08081886080839FB7F894EBE0B8
:10D44000F1E08081877F80839FBF9FB7F894E8E0F9
:10D45000F1E08081816080839FBF0C9A1498129ABA
:10D46000399A4198479AA1E8B0E08C918F7E8C93CD
:10D470008C9188608C93E0E8F0E080818D7F8083E0
:10D4800080818E7F808380818F73808380818F7C79
:10D4900080838C91887F82608C9380E090E490936D
:10D4A0008900809388001092850010928400EFE636
:10D4B000F0E080818260808381E0809353027894E1
:10D4C00008959091230C8091220C981731F035D259
:10D4D0000E9471230E941C87F4CF0895CF93DF939D
:10D4E000EFB7F894EC0188819981AA81BB81809380
:10D4F000791190937A11A0937B11B0937C11EB0179
:10D5000088819981AA81BB8180937D1190937E113E
:10D51000A0937F11B0938011EA0188819981AA813B
:10D52000BB818093811190938211A0938311B0935A
:10D530008411E90188819981AA81BB818093851139
:10D5400090938611A0938711B0938811EFBFDF915C
:10D55000CF9108952FB7F894FC0180819181A28129
:10D56000B3818093851190938611A0938711B09316
:10D5700088112FBF08952FB7F89494E0899FF00188
:10D580001124E758FE4E60817181828193812FBF03
:10D59000089597DF5F9A8A9A9FB7F894E8E0F1E0E0
:10D5A0008081816080839FBF129A479A08958091FD
:10D5B0006F008D7F80936F009091230C8091220CDF
:10D5C00098130CC01092C0111092BF1180916F007F
:10D5D000826080936F001092F00808959091230C60
:10D5E0008091220C981741F38091220C8F5F8F70ED
:10D5F0008093220CE1CF2F923F924F925F926F92D5
:10D600007F928F929F92AF92BF92CF92DF92EF92D2
:10D61000FF920F931F93CF93DF9300D000D0CDB72D
:10D62000DEB78C01F62E21E0261760F5E1E3F1E18B
:10D630008491882341F09091C00095FFFCCF8093A6
:10D64000C6003196F5CF8F2D90E04AE050E0BC0146
:10D6500080E795E00E94AF16E7E2F0E1849188232D
:10D6600041F09091C00095FFFCCF8093C6003196A9
:10D67000F5CF8091C00085FFFCCF8AE08093C60083
:10D680000E9438236F2D70E0FB01EE0FFF1FE45C5A
:10D69000FB4F408151815E834D83452B09F4A6C029
:10D6A000FB01E65CFB4F50815A832D813E812C5F4C
:10D6B0003F4F81E090E089836A81861708F07BC044
:10D6C000DC01F901459154910196B9016C5F7F4FDE
:10D6D000041715070CF06DC00297AC01440F551FDD
:10D6E000440F551F4E5F5F4F6D817E81460F571F60
:10D6F000FA0165917491880F991F880F991FED8128
:10D70000FE818E0F9F1FFC01A590B490FD01EE0FCE
:10D71000FF1FEE0FFF1F3296AD81BE81EA0FFB1F88
:10D72000C590D490FA01E590F490F90125903490D9
:10D73000FC01259134913C832B83882777FD8095CC
:10D74000982F0E9422B62B013C01B8016A197B096F
:10D75000882777FD8095982F0E9422B64B015C01A7
:10D76000B6016E197F09882777FD8095982F0E9452
:10D7700022B69B01AC01C501B4010E9455B86B01F2
:10D780007C01B1014B815C81641B750B882777FD9F
:10D790008095982F0E9422B69B01AC01C701B6016B
:10D7A0000E9487B59B01AC01C301B2010E94A7B4DE
:10D7B00006C09B0180CF60E070E080E090E0A9812E
:10D7C000BA81AB132BC02D813E81E4E0AE9F200DCA
:10D7D000311D112422503109F90165917491882776
:10D7E00077FD8095982F0E9422B618C0B80188272F
:10D7F00077FD8095982F0E9422B620E030E04AEF16
:10D800005EE30E9455B820E030E040E85DE30E940E
:10D8100055B820E030E0A9010E94A7B426960FB6C3
:10D82000F894DEBF0FBECDBFDF91CF911F910F9156
:10D83000FF90EF90DF90CF90BF90AF909F908F9030
:10D840007F906F905F904F903F902F9008958091C0
:10D850003612909137129093030980930209209118
:10D86000F50820FD09C010922E1210922F1210926E
:10D870003012109231120AC060E0BDDE60932E12A9
:10D8800070932F128093301290933112809138123E
:10D890009091391290930509809304092091F5081D
:10D8A00021FF0BC061E0A7DE609332127093331248
:10D8B000809334129093351208C010923212109255
:10D8C00033121092341210923512109228121092C4
:10D8D000291210922A1210922B128FB7F8941092DC
:10D8E00027128FBF08952091650230916602409102
:10D8F00067025091680260E070E08FE793E40E9455
:10D9000087B56093E7117093E8118093E9119093C4
:10D91000EA116093EB117093EC118093ED119093E9
:10D92000EE11089597FF03C08091DE1104C0FC0141
:10D93000E152FE4E808190E008952F923F924F92E7
:10D940005F926F927F928F929F92AF92BF92CF928F
:10D95000DF92EF92FF920F931F93CF93DF93CDB798
:10D96000DEB7A2970FB6F894DEBF0FBECDBF809191
:10D970002712882309F4D2C16ADF8091690290914D
:10D980006A02A0916B02B0916C028D8B9E8BAF8B63
:10D99000B88F8091650290916602A0916702B09164
:10D9A0006802898F9A8FAB8FBC8F809161029091B2
:10D9B0006202A0916302B09164028D8F9E8FAF8F3F
:10D9C000B8A3AEE2B2E1BA8BA98BECE3F2E1F88B3B
:10D9D000EF8787EF91E19A878987AFEDB1E1BA834D
:10D9E000A983E5E5F2E0F887EF8386ED91E19C8B72
:10D9F0008B8B05EE11E14FE1242E42E1342EA7E19D
:10DA0000B2E1BC83AB83EFEFF1E1FE83ED831AA2B9
:10DA100019A2A989BA898D909D90AD90BD90BA8BBD
:10DA2000A98BEF85F88961907190F88BEF87B3012E
:10DA3000882777FD8095982F0E9422B6A501940132
:10DA40000E94A6B46B017C01A985BA856D937D9374
:10DA50008D939D93BA87A98720E030E040E251E49E
:10DA60000E9483B7181624F421E0F8012083D6C061
:10DA700020E030E040E251ECC701B6010E9480B5E1
:10DA800087FD02C0672821F4E1E0D801EC93CDC006
:10DA9000D8018C91882331F0F10110821182128219
:10DAA00013821C92A70196016D897E898F89988DBA
:10DAB0000E9455B86B877C878D879E87E9A1FAA164
:10DAC000E15FFD4E6083718382839383D1012D9149
:10DAD0003D914D915C91C701B6010E94A7B46B01C5
:10DAE0007C01E9A1FAA1E151FE4E50806180728073
:10DAF0004380252D362D472D542D0E9480B587FD5E
:10DB000016C0E9A1FAA1E951FE4E508061807280F1
:10DB10004380252D362D472D542DB601C7010E9477
:10DB200083B7181624F05C2C6D2C7E2C4F2C852D81
:10DB3000962DA72DB42DF10180839183A283B38309
:10DB4000252D362D472D542D698D7A8D8B8D9C8DED
:10DB50000E9455B82B013C01E9A1FAA1E95FFD4EF5
:10DB60006083718382839383AB81BC812D913D91CE
:10DB70004D915C91C501B4010E94A6B49B01AC011A
:10DB80006D8D7E8D8F8D98A10E9455B820ED3CEC57
:10DB90004CE45DE30E9455B86B017C0123E333E361
:10DBA00043E75FE3ED81FE81608171818281938132
:10DBB0000E9455B89B01AC01C701B6010E94A7B4F1
:10DBC0006B017C01AD81BE816D937D938D939C93A0
:10DBD0001397EB81FC8180829182A282B382A301A0
:10DBE00092016B857C858D859E850E94A7B4A701D7
:10DBF00096010E94A6B46B017C0120E030E0A901EF
:10DC00000E9480B587FD11C020E030E040E853E479
:10DC1000C701B6010E9483B7181654F4C12CD12C49
:10DC200030E8E32E33E4F32E03C0C12CD12C76016F
:10DC3000AB89BC898D919D91BC8BAB8BBC01882736
:10DC400077FD8095982F0E9422B69B01AC01C501FB
:10DC5000B4010E9483B71816F4F4EF81F88580812F
:10DC60009181BC01882777FD8095982F0E9422B66C
:10DC70009B01AC01C501B4010E9480B587FF0BC0B8
:10DC8000C701B6010E94EFB5CB0195958795A98193
:10DC9000BA818C9303C0E981FA81108289A19AA18B
:10DCA00004969AA389A3A981BA811196BA83A983FC
:10DCB000EF81F8853296F887EF830F5F1F4FF4E00E
:10DCC0002F0E311C8B819C8104969C838B83AD81AC
:10DCD000BE811496BE83AD83E9A1FAA1389709F0FD
:10DCE00098CE0E9470AE0091E1111091E211209146
:10DCF000E3113091E411601B710B820B930B6838B8
:10DD000073418105910550F00E9470AE6093E1115E
:10DD10007093E2118093E3119093E411A2960FB6F1
:10DD2000F894DEBF0FBECDBFDF91CF911F910F9151
:10DD3000FF90EF90DF90CF90BF90AF909F908F902B
:10DD40007F906F905F904F903F902F900895CF936A
:10DD5000DF93C0915502D09156021092EF111092AC
:10DD6000F0111092F1111092F21120916502309190
:10DD70006602409167025091680260E070E08FE7B0
:10DD800093E40E9487B56093E7117093E811809344
:10DD9000E9119093EA11D0935802C0935702109260
:10DDA000F3111092F4111092F5111092F611609384
:10DDB000EB117093EC118093ED119093EE11249A76
:10DDC0008091010180618093010180910101806255
:10DDD000809301018091010180648093010187EDAE
:10DDE00080937A0010927E0010927D0080917D00D9
:10DDF000806280937D0080917D00806880937D00AB
:10DE000080917D00806480937D0080E888BD809152
:10DE10006E00846080936E006AEF70E080E090E0B6
:10DE20000E949FAE85E090E09093D7118093D61129
:10DE300060E08091590290915A02DDDB20E030E0F1
:10DE400040EA50E40E9480B587FF0AC080915902E1
:10DE500090915A02409790935A0280935902E8CFCA
:10DE600084E591E0909356028093550260E08091A2
:10DE7000DA119091DB11BFDB20E030E04AEA53E495
:10DE80000E9483B7181654F48091DA119091DB1137
:10DE900040969093DB118093DA11E8CF85E090E013
:10DEA0009093D9118093D81161E080915B02909199
:10DEB0005C02A1DB20E030E040EA50E40E9480B543
:10DEC00087FF0AC080915B0290915C02409790931B
:10DED0005C0280935B02E8CF84E591E09093580266
:10DEE0008093570261E08091DC119091DD1183DB1A
:10DEF00020E030E04AEA53E40E9483B7181654F455
:10DF00008091DC119091DD1140969093DD1180930A
:10DF1000DC11E8CFDF91CF910895089510923D1262
:10DF200010923C12EEE3F2E11182108210923B1249
:10DF300010923A121092DF112C981092E0119FB7B4
:10DF4000F894E2E0F1E080818F7E80839FBF1092A1
:10DF50003B1210923A121092DE119FB7F894808112
:10DF60008F7D80839FBF08952F923F924F925F9243
:10DF70006F927F928F929F92AF92BF92CF92DF92D9
:10DF8000EF92FF920F931F93CF93DF93CDB7DEB73E
:10DF9000AE970FB6F894DEBF0FBECDBF6C8F7D8FEE
:10DFA0008E8F9F8F5EA74DA73CA72BA70E9470AEB8
:10DFB00069A37AA38BA39CA32DA53EA5233031058D
:10DFC0001CF4EDEFF3E017C0E0E1F4E08191882369
:10DFD00039F09091C00095FFFCCF8093C600F6CF3A
:10DFE0008091C00085FFFCCF15C29091C00095FFC5
:10DFF000FCCF8093C60081918111F7CF8091C00042
:10E0000085FFFCCF8AE08093C60088DF4DA55EA522
:10E0100080E857FF43C08093DE1189A19AA1ABA18C
:10E02000BCA1898B9A8BAB8BBC8B8D879E87AF876E
:10E03000B88B1D8290E4998FACE1AA8FB6E4BB8FB8
:10E040001D8A1E8A1F8A188E20E830E040E050E0CA
:10E0500029833A834B835C83F0E84F2E512C612C4B
:10E06000712C1DA21EA21FA218A631E038A31C8687
:10E070001B86312C00E010E0212C4DA55EA54152FD
:10E080005E4E5AA749A78DA59EA5880F991F880F98
:10E09000991F825D9D4E9A87898708C0EDA5FEA5D0
:10E0A000E152FE4E8083B9CF0E941C8780912712D7
:10E0B000882309F4DCC0CBDBADA5BEA5B7FF09C042
:10E0C000309028120091291210912A1220902B12C0
:10E0D00006C0E985FA853080018112812380232DD5
:10E0E000302F412F522D6D897E898F89988D0E9406
:10E0F00083B7181624F03D8A0E8B1F8B288E232D94
:10E10000302F412F522D6D81798D8A8D9B8D0E94EC
:10E1100080B587FD04C03D82098F1A8F2B8EF8A130
:10E12000FF2309F451C02C8D3D8D4E8D5F8D632DE5
:10E13000702F812F922D0E9483B718160CF097C074
:10E140000E9470AE29893A894B895C89621B730BE6
:10E15000840B950B693873418105910508F487C0DC
:10E16000D301C20129813A814B815C81821B930BCF
:10E17000A40BB50B4DA55EA5B595A795979587956D
:10E1800057FF03C08093DE1103C0E9A5FAA5808381
:10E190000E9470AE6D877E878F87988B9B01AC0144
:10E1A00089899A89AB89BC89281B390B4A0B5B0B7F
:10E1B0002DA33EA34FA358A79C8D9D8BAD8DAE8BF9
:10E1C000BE8DBF8BEF8DE88F2C8D3D8D4E8D5F8D7D
:10E1D000632D702F812F922D0E9480B587FFF0C292
:10E1E0000E9470AE2D853E854F855889621B730B4A
:10E1F000840B950B693873418105910508F4E0C2E1
:10E200000E9470AE698B7A8B8B8B9C8BDC01CB016F
:10E210002D853E854F855889821B930BA40BB50B2A
:10E220004B855C85452B09F011C189819A81AB81B1
:10E23000BC81840D951DA61DB71D2DA53EA5B595C8
:10E24000A7959795879537FFB7C28093DE112B85E9
:10E250003C852F5F3F4F3C872B873C8D3D834D8D09
:10E26000498F5E8D5A8F8F8D8B8F91E098A320E020
:10E2700030E040EA51E46C8D7D8D8E8D9F8D0E9443
:10E28000A7B49B01AC01632D702F812F922D0E94AA
:10E2900083B7181694F4E2ECF0E18491882341F0FE
:10E2A0009091C00095FFFCCF8093C6003196F5CFCA
:10E2B0008091C00085FFFCCFADC00E9470AE29A147
:10E2C0003AA14BA15CA1621B730B840B950B613DC2
:10E2D00077408105910508F450C04DA55EA557FF14
:10E2E00010C0E090DE11F12CECEBF0E1849188237A
:10E2F000C9F09091C00095FFFCCF8093C600319685
:10E30000F5CFA9A5BAA5EC90F12CE6EBF0E184914C
:10E31000882341F09091C00095FFFCCF8093C60008
:10E320003196F5CF22E030E0432D502F612F722D32
:10E3300080E795E00E948517E2EBF0E18491882365
:10E3400041F09091C00095FFFCCF8093C6003196BC
:10E35000F5CF4AE050E0B70180E795E00E94AF16A4
:10E360008091C00085FFFCCF8AE08093C6000E94A8
:10E3700070AE69A37AA38BA39CA30E9470AE6B01BD
:10E380007C010E9470AE89889A88AB88BC882D85F4
:10E390003E854F855889820E931EA41EB51EC8184F
:10E3A000D908EA08FB08C60ED71EE81EF91E31E898
:10E3B000C3163FE4D30632E1E306F10490F0E5E949
:10E3C000F0E18491882341F09091C00095FFFCCF4B
:10E3D0008093C6003196F5CF8091C00085FFFCCFB9
:10E3E00019C04B855C858BA59CA5841795070CF0FF
:10E3F0005BCEE4E4F0E18491882341F09091C00089
:10E4000095FFFCCF8093C6003196F5CF8091C00078
:10E4100085FFFCCF8AE08093C600AE960FB6F894D5
:10E42000DEBF0FBECDBFDF91CF911F910F91FF9047
:10E43000EF90DF90CF90BF90AF909F908F907F90A4
:10E440006F905F904F903F902F9008958DA09EA069
:10E45000AFA0B8A4880E991EAA1EBB1E2DA13EA176
:10E460004FA158A5281B390B4A0B5B0BCA01B901F8
:10E4700029813A814B815C810E941BB9A5019401DD
:10E480000E9473B9240D351D461D571D24313105D9
:10E490004105510504F129013A013DEE43165104AD
:10E4A000610471042CF07CEE472E512C612C712CF0
:10E4B00041E84416510461047104DCF08FEF90E0F0
:10E4C000A0E0B0E084199509A609B70989839A8369
:10E4D000AB83BC8312C064E1462E512C612C712C9D
:10E4E00024E130E040E050E029833A834B835C83B1
:10E4F00004C049825A826B827C82E9E2F1E1849114
:10E50000882341F09091C00095FFFCCF8093C60016
:10E510003196F5CF2AE030E0B301A20180E795E023
:10E520000E948C16E4E2F1E18491882341F09091FD
:10E53000C00095FFFCCF8093C6003196F5CF2AE04E
:10E5400030E049815A816B817C8180E795E00E94AF
:10E550008C16EDE1F1E18491882341F09091C000A7
:10E5600095FFFCCF8093C6003196F5CF22E030E0D6
:10E570004D81598D6A8D7B8D80E795E00E948517CE
:10E58000E6E1F1E18491882341F09091C00095FF8C
:10E59000FCCF8093C6003196F5CF22E030E04D8964
:10E5A0005E896F89788D80E795E00E94851780915C
:10E5B000C00085FFFCCF8AE08093C6002B853C8598
:10E5C000233031050CF431CE69817A818B819C81B5
:10E5D0000E9422B620E030E040E850E40E9455B8A6
:10E5E0006B017C012D81398D4A8D5B8D6D897E8912
:10E5F0008F89988D0E94A6B420ED3FE049E450E455
:10E600000E9455B820E030E040E05FE30E9455B83A
:10E610009B01AC01C701B6010E9487B56B017C016B
:10E62000C501B4010E9422B620E030E04AE754E47C
:10E630000E9487B54B015C01E0E1F1E18491882300
:10E6400041F09091C00095FFFCCF8093C6003196B9
:10E65000F5CF22E030E0B701A60180E795E00E9407
:10E660008517EAE0F1E18491882341F09091C000A0
:10E6700095FFFCCF8093C6003196F5CF22E030E0C5
:10E68000B501A40180E795E00E9485178091C00044
:10E6900085FFFCCF8AE08093C6002AE939E949E189
:10E6A0005FE3C701B6010E9455B86B017C019B0175
:10E6B000AC010E94A7B4A50194010E9487B56D83A7
:10E6C0007E838F839887A5019401C701B6010E94BC
:10E6D00055B820E030E040E05EE30E9455B84B01C1
:10E6E0005C01EDEFF0E18491882341F09091C0004E
:10E6F00095FFFCCF8093C6003196F5CF8091C00086
:10E7000085FFFCCF8AE08093C600E7EFF0E18491BB
:10E71000882341F09091C00095FFFCCF8093C60004
:10E720003196F5CF22E030E0B701A60180E795E011
:10E730000E9485178091C00085FFFCCF8AE08093FE
:10E74000C600E1EFF0E18491882341F09091C00090
:10E7500095FFFCCF8093C6003196F5CF22E030E0E4
:10E760004D815E816F81788580E795E00E948517F5
:10E770008091C00085FFFCCF8AE08093C600EBEE5D
:10E78000F0E18491882341F09091C00095FFFCCF87
:10E790008093C6003196F5CF22E030E0B501A401A8
:10E7A00080E795E00E9485178091C00085FFFCCF2F
:10E7B0008AE08093C60039CDE9A5FAA5808347CDCC
:10E7C00018A255CD1F920F920FB60F9211240BB6BF
:10E7D0000F922F933F934F935F936F937F938F93FA
:10E7E0009F93AF93BF93EF93FF9380915402811156
:10E7F00027C08091DF118093D511882329F0809163
:10E80000F408813109F42C9A8091E0118093D4119D
:10E81000882341F09FB7F894809102018061809332
:10E8200002019FBF8091DE118093D311882341F0B4
:10E830009FB7F894809102018062809302019FBF8C
:10E840009091D51180915402891728F08091F40895
:10E85000813109F42C989091D41180915402891738
:10E8600040F09FB7F894809102018F7E809302015F
:10E870009FBF9091D31180915402891740F09FB7A8
:10E88000F894809102018F7D809302019FBF809157
:10E8900054028F5F8F77809354028091D21190E061
:10E8A0008830910508F08DC0FC01EE58FF4F0C94A4
:10E8B0008FB988E080937B0085E480937C00809111
:10E8C0007A00806480937A000E949D8681E019C05E
:10E8D00020917800309179008091CE119091CF11E4
:10E8E000A091D011B091D111820F931FA11DB11D24
:10E8F0008093CE119093CF11A093D011B093D111EA
:10E9000082E08093D2115DC088E080937B0086E432
:10E9100080937C0080917A00806480937A000E94CA
:10E920009D8683E0EECF2091780030917900809130
:10E93000CA119091CB11A091CC11B091CD11820F41
:10E94000931FA11DB11D8093CA119093CB11A09369
:10E95000CC11B093CD1184E0D4CF88E080937B00BC
:10E9600087E480937C0080917A00806480937A00B1
:10E970000E949D8685E0C5CF209178003091790076
:10E980008091C6119091C711A091C811B091C91181
:10E99000820F931FA11DB11D8093C6119093C711C3
:10E9A000A093C811B093C91186E0ABCF0E949D8699
:10E9B00087E0A7CF1092D2118091C5118F5F80930D
:10E9C000C5118091C511803108F484C0809127124F
:10E9D000811118C08091CE119091CF119093371270
:10E9E000809336128091C6119091C711909339127D
:10E9F000809338128091CA119091CB1190932D126F
:10EA000080932C1281E0809327121092C5111092EE
:10EA1000CE111092CF111092D0111092D1111092EC
:10EA2000C6111092C7111092C8111092C9111092FC
:10EA3000C1111092C2111092C3111092C411109200
:10EA4000CA111092CB111092CC111092CD1180915D
:10EA50003612909137122091DA113091DB114091EA
:10EA6000F5082817390714F0427001C0416040933F
:10EA7000F5082091590230915A024091F508821709
:10EA8000930714F0427001C041604093F5088091F3
:10EA90003812909139122091DC113091DD114091A2
:10EAA000F5082817390714F0417001C042604093FF
:10EAB000F50820915B0230915C024091F5088217C5
:10EAC000930714F0417001C042604093F50881E063
:10EAD0008093F908FF91EF91BF91AF919F918F9132
:10EAE0007F916F915F914F913F912F910F900BBE4E
:10EAF0000F900FBE0F901F9018952DEB37E346E057
:10EB00005EE30C9455B82DEB37E346E05EE30C94DE
:10EB100087B52DEB37E346E05EE30C9487B52DEB2C
:10EB200037E346E05EE30C9455B810928E121092D3
:10EB30008F12109290121092911285E790EA9093A2
:10EB40006F0280936E02089510923D1210923C1253
:10EB500010923F1210923E1210923B1210923A12F3
:10EB6000E4CF10928E1210928F1210929012109287
:10EB7000911281EC9FE790936F0280936E0282E086
:10EB800080936D020895FB0160916E0270916F0297
:10EB9000709387126093861260918E1270918F121B
:10EBA000709385126093841262E060936D0265EA4F
:10EBB0007FE970936F0260936E029093831280934B
:10EBC0008212F0938112E0938012662757FD6095C0
:10EBD000762F40937C1250937D1260937E12709337
:10EBE0007F12C901AA2797FDA095BA2F80937812AA
:10EBF00090937912A0937A12B0937B1280819181C5
:10EC0000AA2797FDA095BA2F80938E1290938F120A
:10EC1000A0939012B09391120895CF93DF93262F73
:10EC2000FC01EB5BFF4F40815181EC01CD5BDF4F7D
:10EC30006881798104960E94C3A928813981280FAF
:10EC4000311D87FD3A953983288381E090E0DF917B
:10EC5000CF91089581E090E09093DE128093DD12D1
:10EC600084E190E09093E0128093DF128091F008AD
:10EC7000853019F460E474E004C0873031F46BE44B
:10EC800074E08AE992E10E94FCB081E090E0909308
:10EC9000DE128093DD128BE290E09093E01280937D
:10ECA000DF1266E574E08AE992E10C94FCB0CF9340
:10ECB000DF93FC016491EC012196662331F08AE92F
:10ECC00092E10E94FDB0CE01F4CFDF91CF91089583
:10ECD000CF92DF92EF92FF920F931F93CF93DF9328
:10ECE0001F92CDB7DEB7E62E8901F9010190002011
:10ECF000E9F7F22EFE1A92E1F90E1092DE1210924E
:10ED0000DD1290E001965CE0589F9001599F300D14
:10ED100011243093E0122093DF12642F8AE992E1EC
:10ED200079830E94FDB0CE2C7981D72EFE0CEF2C7A
:10ED3000EC18F6016491662341F08AE992E10E94A1
:10ED4000FDB0EFEFCE1ADE0AF2CF6AE38AE992E174
:10ED50000E94FDB0EE2039F060E28AE992E10E9463
:10ED6000FDB0EA94F7CFB8018AE992E10F90DF9104
:10ED7000CF911F910F91FF90EF90DF90CF900C9467
:10ED8000FCB08091090991E08927809309098823C3
:10ED900019F083E695E102C08FE595E10C94B31973
:10EDA000CF92DF92EF92FF9285E08093F00810926D
:10EDB000F1081092F2081092501210925112109213
:10EDC0005212109253121092541210925512109225
:10EDD000561210925712C12CD12C88E4E82E82E4EE
:10EDE000F82EC0925812D0925912E0925A12F09214
:10EDF0005B12C0925C12D0925D12E0925E12F092B1
:10EE00005F126091FC087091FD08625371098827B8
:10EE100077FD8095982F0E9422B6609360127093C0
:10EE200061128093621290936312C0926412D09226
:10EE30006512E0926612F092671260936812709306
:10EE4000691280936A1290936B126091FE08709120
:10EE5000FF0862537109882777FD8095982F0E94DB
:10EE600022B660936C1270936D1280936E12909321
:10EE70006F12C0927012D0927112E0927212F092E0
:10EE8000731260937412709375128093761290933C
:10EE900077124BDE8CEB94E1FF90EF90DF90CF90F8
:10EEA0000C94B319AF92BF92CF92DF92EF92FF9280
:10EEB0000F931F93CF93DF931F92CDB7DEB790EFE1
:10EEC000A92E98E0B92E87E0F501808380E090E0DC
:10EED000A0E0B0E48093E2089093E308A093E408F4
:10EEE000B093E508198220E030E040EA50E46091F8
:10EEF0003702709138028091390290913A020E9453
:10EF000087B59E012F5F3F4F69017B018C0126EE83
:10EF100038E042EE58E06EED78E08AED98E00E942D
:10EF2000E557F501108281E69CE890936F0280938B
:10EF30006E0282E080936D0210928E1210928F12F8
:10EF4000109290121092911285ED92E10E94B319E5
:10EF50000F90DF91CF911F910F91FF90EF90DF9075
:10EF6000CF90BF90AF9008950E94261A0C94EF1195
:10EF7000DF92EF92FF920F931F93CF93DF93D82FDF
:10EF8000F62ED72EC42FE22E61E08EE992E14E33A9
:10EF900011F04632A9F40E94A9AB8CE0D89FA001E1
:10EFA00011244D5F5F4F0CE010E020E830E060E09E
:10EFB00070E08EE992E10E9400AE60E08EE992E19D
:10EFC0000E94A9AB1092DE121092DD128D2F90E0FC
:10EFD00001962CE0289FF001299FF00D1124F09359
:10EFE000E012E093DF12CE3311F06C2F01C060E22B
:10EFF0008AE992E10E94FDB0CF2DDD2D11E11F0DB8
:10F00000912F9C1BFE016491662331F08AE992E105
:10F010000E94FDB02196F4CFC92FCC2339F060E2D5
:10F020008AE992E10E94FDB0C150F7CF6E2D8AE9C6
:10F0300092E10E94FDB060E28AE992E10E94FDB097
:10F0400061E08EE992E1DF91CF911F910F91FF90E6
:10F05000EF90DF900C94A9ABCF92DF92EF92FF92EA
:10F060000F931F93CF93DF931F92CDB7DEB7E0913D
:10F07000F10828E0E29FF0011124E05BFD4E808161
:10F080009181A281B3818093DA089093DB08A093E9
:10F09000DC08B093DD0884819581A681B7818093D7
:10F0A000DE089093DF08A093E008B093E10819828E
:10F0B00020E030E040E752E460912F02709130028E
:10F0C00080913102909132020E9487B59E012F5F9C
:10F0D0003F4F69017B018C0126EE38E042EE58E09B
:10F0E0006EED78E08AED98E00E94E5570E94616A33
:10F0F0001092E2081092E3081092E4081092E508DA
:10F10000198220E030E040E251E4609137027091D2
:10F1100038028091390290913A020E9487B57B01B2
:10F120008C0126EE38E042EE58E06EED78E08AED94
:10F1300098E00E94E5570E94616A0F90DF91CF919D
:10F140001F910F91FF90EF90DF90CF900895CF9295
:10F15000DF92EF92FF920F931F93CF93DF931F9253
:10F16000CDB7DEB787E08093F00880E090E0A0E0C4
:10F17000B0E48093E2089093E308A093E408B0938E
:10F18000E508198220E030E040EA50E4609137025F
:10F19000709138028091390290913A020E9487B5AD
:10F1A0009E012F5F3F4F69017B018C0126EE38E005
:10F1B00042EE58E06EED78E08AED98E00E94E55767
:10F1C000B4DC8091F10881508093F108813039F4EA
:10F1D0008091F208823040F41092F20805C081114B
:10F1E00003C084E08093F10837DF0F90DF91CF9167
:10F1F0001F910F91FF90EF90DF90CF900895CF92E5
:10F20000DF92EF92FF920F931F93CF93DF931F92A2
:10F21000CDB7DEB787E08093F00880E090E0A0E013
:10F22000B0E48093E2089093E308A093E408B093DD
:10F23000E508198220E030E040EA50E460913702AE
:10F24000709138028091390290913A020E9487B5FC
:10F250009E012F5F3F4F69017B018C0126EE38E054
:10F2600042EE58E06EED78E08AED98E00E94E557B6
:10F270005CDC8091F1088F5F8093F108853031F478
:10F2800084E08093F20881E08093F108E5DE0F903E
:10F29000DF91CF911F910F91FF90EF90DF90CF9072
:10F2A0000895CF9382E080936D020E9470AE6C50FF
:10F2B0007E4F8F4F9F4F609394127093951280935F
:10F2C000961290939712389ACAE0409A63E070E0E1
:10F2D00080E090E00E949FAE409863E070E080E0A4
:10F2E00090E00E949FAEC15081F7CF910895109297
:10F2F0008E1210928F12109290121092911280E53D
:10F300009FE790936F0280936E02CBCFCF92DF92F4
:10F31000EF92FF920F931F93CF93DF9380918E1202
:10F3200090918F12A0919012B091911281309048DB
:10F33000A105B10540F010928E1210928F1210921A
:10F3400090121092911260918E1270918F12809192
:10F3500090129091911225E030E040E050E00E9440
:10F3600051B98091981290E0A0E0B0E028173907D9
:10F370004A075B0710F420939812D0919812C0E0CE
:10F3800025E0C22ED12CE12CF12C11E060918E12DF
:10F3900070918F128091901290919112D11137C07B
:10F3A00020916D02222369F026E265307105810506
:10F3B000910510F446E201C040E263E575E18C2F4F
:10F3C000D7DD8091991282FD12C020E030E040E24A
:10F3D00051E460914C1270914D1280914E129091B7
:10F3E0004F120E9480B587FD77C003E036C180913F
:10F3F0008E1290918F12A0919012B0919112059758
:10F40000A105B10510F74DDF83EB9BE770C1D1304B
:10F4100081F520916D02222391F0A70196010E94AF
:10F4200051B9213031054105510519F42AEF4EE358
:10F4300002C02AEF40E26CE475E18C2F99DD8091E7
:10F44000991282FFC2CF60918E1270918F128091BB
:10F45000901290919112A70196010E9451B921300A
:10F4600031054105510509F0B0CF1BDF88E09BE86D
:10F470003EC1D23009F0A9CF20916D02222391F034
:10F48000A70196010E9451B922303105410551056D
:10F4900019F42AEF4EE302C02AEF40E265E475E179
:10F4A0008C2F66DD8091991282FF8FCF60918E1232
:10F4B00070918F128091901290919112A7019601F4
:10F4C0000E9451B9223031054105510509F07DCF27
:10F4D000E8DE8BE59AE80BC1D33031F08091F50876
:10F4E00080FD39C004E072C080916D028823D1F0A4
:10F4F00060918E1270918F12809190129091911262
:10F50000A70196010E9451B92330310541055105EB
:10F5100019F42AEF4EE302C02AEF40E26EE375E1F0
:10F520008C2F26DD8091991282FFD8CF60918E12A8
:10F5300070918F128091901290919112A701960173
:10F540000E9451B9233031054105510539F6A9DE34
:10F550008CE898E8CCC0D43011F005E037C0809139
:10F560006D028823D1F060918E1270918F1280917C
:10F57000901290919112A70196010E9451B92430E6
:10F5800031054105510519F42AEF4EE302C02AEF77
:10F5900040E263E375E18C2FEBDC8091991282FFEE
:10F5A000DCCF60918E1270918F12809190129091A9
:10F5B0009112A70196010E9451B9243031054105ED
:10F5C000510559F66EDE88ED99E891C08091F508F5
:10F5D00081FF43C00D1711F00F5F3FC080916D0296
:10F5E0008823F1F060918E1270918F1280919012A9
:10F5F00090919112A70196010E9451B9802F90E03D
:10F60000A0E0B0E0281739074A075B0719F42AEF92
:10F610004EE302C02AEF40E268E275E18C2FA8DCDD
:10F620008091991282FFD8CF60918E1270918F12C3
:10F630008091901290919112A70196010E9451B968
:10F64000802F90E0A0E0B0E0281739074A075B0759
:10F6500019F627DE82E599E84AC060918E12709112
:10F660008F128091901290919112A70196010E94A1
:10F6700051B9802F90E0A0E0B0E0281739074A0781
:10F680005B0788F025E0029FC00111240197AA279B
:10F6900097FDA095BA2F80938E1290938F12A0930E
:10F6A0009012B093911260918E1270918F1280918E
:10F6B000901290919112A70196010E9451B98091E8
:10F6C000981290E00496422F50E0841795074CF46E
:10F6D0008CEF820F8093981210936D02DBEFD20FA4
:10F6E000CFEFCF5FDF5FC53008F450CE0CC09093F2
:10F6F0006F0280936E0210928E1210928F121092EF
:10F70000901210929112DF91CF911F910F91FF9063
:10F71000EF90DF90CF9008958DEC9CECACECBDE3C6
:10F7200080934C1290934D12A0934E12B0934F12AF
:10F73000EDCD80E090E0A0E8BFE380934C12909381
:10F740004D12A0934E12B0934F12E0CD80E090E0A6
:10F75000A0E2B1E480934C1290934D12A0934E120C
:10F76000B0934F12D3CD8F929F92AF92BF92CF9210
:10F77000DF92EF92FF921F93CF93DF9380918E12CF
:10F7800090918F12A0919012B09191128130904877
:10F79000A105B10540F010928E1210928F121092B6
:10F7A00090121092911260918E1270918F1280912E
:10F7B00090129091911225E030E040E050E00E94DC
:10F7C00051B98091981290E0A0E0B0E02817390775
:10F7D0004A075B0710F420939812D0919812C0E06A
:10F7E00035E0C32ED12CE12CF12C43E1842E912C59
:10F7F000A12CB12C11E060918E1270918F1280912A
:10F80000901290919112D11122C020916D02222369
:10F8100069F026E2653071058105910510F446E234
:10F8200001C040E26AE075E18C2FA2DB8091991261
:10F8300082FF2AC080918E1290918F12A091901217
:10F84000B09191120597A105B105F0F4D1C0D13066
:10F8500009F045C020916D02222391F0A701960185
:10F860000E9451B9213031054105510519F42AEFA3
:10F870004EE302C02AEF40E260E075E18C2F78DBB6
:10F880008091991282FD16C080918E1290918F12F4
:10F89000A0919012B09191124497A105B10508F47E
:10F8A00083C080928E1290928F12A0929012B0928A
:10F8B00091127AC060918E1270918F128091901285
:10F8C00090919112A70196010E9451B92130310502
:10F8D00041055105C9F6E5DC86EA9BE78CC0D230CC
:10F8E00081F520916D02222391F0A70196010E94DB
:10F8F00051B9223031054105510519F42AEF4EE383
:10F9000002C02AEF40E267EF74E18C2F31DB809177
:10F91000991282FFB9CF60918E1270918F128091EF
:10F92000901290919112A70196010E9451B9223034
:10F9300031054105510509F0A7CFB3DC89E99BE703
:10F940005AC0D33009F0A0CF20916D02222391F04C
:10F95000A70196010E9451B9233031054105510597
:10F9600019F42AEF4EE302C02AEF40E26CEE74E194
:10F970008C2FFEDA8091991282FF86CF60918E12D1
:10F9800070918F128091901290919112A70196011F
:10F990000E9451B9233031054105510509F074CF5A
:10F9A00080DC8CE89BE727C060918E1270918F12EB
:10F9B0008091901290919112A70196010E9451B9E5
:10F9C0008091981290E00496422F50E0841795079A
:10F9D0004CF48CEF820F8093981210936D02DBEF42
:10F9E000D20FCFEFCF5FDF5FC53008F404CF0FC079
:10F9F00058DC88E094E990936F0280936E02109235
:10FA00008E1210928F121092901210929112DF911A
:10FA1000CF911F91FF90EF90DF90CF90BF90AF906C
:10FA20009F908F9008952091F50820FF08C0809145
:10FA3000ED129091EE1290933D1280933C1221FFB3
:10FA400008C08091ED129091EE1290933F12809336
:10FA50003E128091F908811108C08091EB129091BB
:10FA6000EC1290933B1280933A128091E91290919C
:10FA7000EA1290939C0880939B0857D80C948D6F42
:10FA80002091F50820FF08C08091E7129091E812BC
:10FA900090933D1280933C1221FF08C08091E712A1
:10FAA0009091E81290933F1280933E128091F90852
:10FAB000811108C08091E5129091E61290933B125B
:10FAC00080933A128091E3129091E41290939C08F3
:10FAD00080939B082AD80C948D6F9F92AF92BF920F
:10FAE000CF92DF92EF92FF920F931F93CF93DF930A
:10FAF0002091BF062F5F2093BF068AE0289FE00178
:10FB0000112430E08091C4069091C506281739076A
:10FB100020F48E01065F1F4F06C00091C6061091AB
:10FB2000C7060C0F1D1F50E2E52E59E0F52E61E9C6
:10FB3000C62E62E1D62E74E1972EEAE0AE2EB12CED
:10FB4000C017D10778F56091C0067091C106615069
:10FB500071096C1B7D0B7093C3066093C2068FE026
:10FB600099E00E94C94EFF92EF92DF92CF921F92CE
:10FB70009F92CE01B5010E942AB9989E9001999E4C
:10FB8000300D112429503A4F3F932F930E943EBDD0
:10FB900021968DB79EB708960FB6F8949EBF0FBEFC
:10FBA0008DBFCECF87EF91E890936F0280936E0266
:10FBB00010928E1210928F12109290121092911237
:10FBC000DF91CF911F910F91FF90EF90DF90CF9039
:10FBD000BF90AF909F9008959F92AF92BF92CF92A7
:10FBE000DF92EF92FF920F931F93CF93DF932091B9
:10FBF000BF0621502093BF068AE0289FE001112410
:10FC000030E08091C4069091C5062817390720F48A
:10FC10008E01065F1F4F06C00091C6061091C706F1
:10FC20000C0F1D1FF0E2EF2EF9E0FF2EAEE8CA2EFA
:10FC3000A2E1DA2EB4E19B2E8AE0A82EB12CC017E7
:10FC4000D10778F56091C0067091C10661507109C5
:10FC50006C1B7D0B7093C3066093C2068FE099E026
:10FC60000E94C94EFF92EF92DF92CF921F929F9215
:10FC7000CE01B5010E942AB9989E9001999E300D3F
:10FC8000112429503A4F3F932F930E943EBD219655
:10FC90008DB79EB708960FB6F8949EBF0FBE8DBF66
:10FCA000CECF87EF91E890936F0280936E0210920F
:10FCB0008E1210928F121092901210929112DF9168
:10FCC000CF911F910F91FF90EF90DF90CF90BF9059
:10FCD000AF909F9008957F928F929F92AF92BF9224
:10FCE000CF92DF92EF92FF920F931F93CF93DF9308
:10FCF00080911209882309F4C5C080916D02811199
:10FD000004C08091991282FFBDC08FE099E00E94EB
:10FD10001F4F9093C1068093C0069093C3068093B3
:10FD2000C2062AE030E0B9010E942AB97093C506E4
:10FD30006093C406009719F46115710529F4909336
:10FD4000C7068093C6060AC03093C7062093C6062E
:10FD5000615071097093C5066093C4068091C40612
:10FD60009091C506892B29F4E090C606F090C7064D
:10FD700003C05AE0E52EF12C1092BF0663E179E052
:10FD800083E699E00E94523A809113098F32A1F4E0
:10FD90001092C806C0E0D0E090E2C92E99E0D92EBA
:10FDA00006E614E024E1722E3AE0A32EB12C43E1E2
:10FDB000842E49E0942E36C081E08093C806EACFB5
:10FDC0006091C0067091C106615071096C1B7D0B7A
:10FDD0007093C3066093C2068FE099E00E94C94EFB
:10FDE00080912009811122C09F928F921F930F93BF
:10FDF0001F927F92CE01B5010E942AB9789E900190
:10FE0000799E300D112429503A4F3F932F930E9431
:10FE100002BD8DB79EB708960FB6F8949EBF0FBE71
:10FE20008DBF2196CE15DF0559F61EC0DF92CF9209
:10FE30001F930F931F927F92CE01B5010E942AB9A2
:10FE4000789E9001799E300D112429503A4F3F93AE
:10FE50002F930E9402BD8DB79EB708960FB6F894F7
:10FE60009EBF0FBE8DBFDDCF87EF91E890936F02ED
:10FE700080936E0210928E1210928F121092901236
:10FE800010929112DF91CF911F910F91FF90EF90FF
:10FE9000DF90CF90BF90AF909F908F907F9008950C
:10FEA000CF93DF93C1E0D0E0D093DE12C093DD1298
:10FEB00089E090E09093E0128093DF1269E674E0AD
:10FEC0008AE992E10E94FCB0D093DE12C093DD1269
:10FED00086E190E09093E0128093DF126AE774E08D
:10FEE0008AE992E10E94FCB065E874E08AE992E157
:10FEF0000E94FCB0D093DE12C093DD1283E290E04A
:10FF00009093E0128093DF126AE874E08AE992E14C
:10FF10000E94FCB0D093DE12C093DD1280E390E02B
:10FF20009093E0128093DF126CE974E08AE992E129
:10FF30000E94FCB0D093DE12C093DD128DE390E0FE
:10FF40009093E0128093DF1261EB74E08AE992E112
:10FF50000E94FCB08091991282FF10C08091F40839
:10FF6000823119F488E991E902C088E094E990931C
:10FF70006F0280936E02DF91CF9193C9DF91CF9191
:10FF80000895EF92FF920F931F93CF93DF93C1E0F9
:10FF9000D0E0D093DE12C093DD1289E090E0909320
:10FFA000E0128093DF126DEB74E08AE992E10E9427
:10FFB000FCB0D093DE12C093DD1283E190E0909309
:10FFC000E0128093DF1269EC74E08AE992E10E940A
:10FFD000FCB0D093DE12C093DD128DE190E09093DF
:10FFE000E0128093DF126EED74E08AE992E10E94E4
:10FFF000FCB06DEEE62E60E2F62E00E210E024E0AA
:020000021000EC
:1000000030E04EE150E060E370E08EE992E10E9462
:1000100052A68091991282FF17C082E18093F40862
:10002000109209098BE08093F00881E69CE8909398
:100030006F0280936E0235D910928E1210928F1239
:100040001092901210929112DF91CF911F910F9107
:10005000FF90EF900895CF92DF92EF92FF920F936F
:100060001F93CF93DF931F92CDB7DEB7E82E8A019F
:10007000CA0169830E9468BC71E1F72EF81A1092D8
:10008000DE121092DD122E2D30E02F5F3F4F4CE03C
:10009000429FC001439F900D11249093E0128093E2
:1000A000DF1269818AE992E10E94FDB0E1EECE2E75
:1000B000E6E1DE2EFC0CEF2CEC18F60164916623D1
:1000C00041F08AE992E10E94FDB08FEFC81AD80A88
:1000D000F2CF6AE38AE992E10E94FDB0EE2039F0A6
:1000E00060E28AE992E10E94FDB0EA94F7CFC8018C
:1000F0000F90DF91CF911F910F91FF90EF90DF90C4
:10010000CF900C945776CF92DF92EF92FF920F939D
:100110001F93CF93DF9388E090E09093DE1280935B
:10012000DD128DE090E09093E0128093DF1261EF9A
:1001300074E08AE992E10E94FCB08091F10882307B
:1001400038F08091F208823018F481E08093F20850
:1001500080918E1290918F12A0919012B091911275
:1001600081309048A105B10540F010928E12109296
:100170008F12109290121092911260918E127091C3
:100180008F12809190129091911225E030E040E022
:1001900050E00E9451B98091981290E0A0E0B0E048
:1001A000281739074A075B0710F420939812D0915B
:1001B0009812C2E0F5E0CF2ED12CE12CF12C11E009
:1001C000DD2371F02091F20860918E1270918F12F0
:1001D0008091901290919112211136C001E064C07B
:1001E00080916D028823A9F080918E1290918F12D8
:1001F000A0919012B091911220E20597A105B1054E
:1002000010F44EE301C040E265EE72E18C2F0E94D3
:10021000B8778091991282FFD5CF80918E129091FC
:100220008F12A0919012B09191120597A105B1057E
:1002300048F637D8DF91CF911F910F91FF90EF9043
:10024000DF90CF900C94FF78D13069F520916D024A
:10025000222399F0A70196010E9451B9213031055E
:100260004105510519F420E24EE302C020E240E2CC
:1002700060EE72E18C2F0E94B8778091991282FF14
:100280004AC060918E1270918F128091901290915D
:100290009112A70196010E9451B921303105410503
:1002A0005105C9F58CC002E00D1336C020916D02D6
:1002B0002223B9F0A70196010E9451B9802F90E046
:1002C000A0E0B0E0281739074A075B0719F420E2DD
:1002D0004EE302C020E240E269ED72E18C2F0E9401
:1002E000B8778091991282FF17C060918E12709139
:1002F0008F128091901290919112A70196010E9405
:1003000051B9802F90E0A0E0B0E0281739074A07E4
:100310005B0711F460C002E00F5F60918E12709174
:100320008F128091901290919112A70196010E94D4
:1003300051B9802F90E0A0E0B0E0281739074A07B4
:100340005B0788F025E0029FC00111240197AA27CE
:1003500097FDA095BA2F80938E1290938F12A09341
:100360009012B093911260918E1270918F128091C1
:10037000901290919112A70196010E9451B980911B
:10038000981290E00496422F50E0841795074CF4A1
:100390008CEF820F8093981210936D02DBEFD20FD7
:1003A000CFEFCF5FDF5FC53008F40ACFDF91CF9189
:1003B0001F910F91FF90EF90DF90CF9008950E94D2
:1003C0005179DF91CF911F910F91FF90EF90DF90C6
:1003D000CF900C94A7780E945179DF91CF911F9113
:1003E0000F91FF90EF90DF90CF900C9452772F9267
:1003F0003F924F925F926F927F928F929F92AF92B5
:10040000BF92CF92DF92EF92FF920F931F93CF9301
:10041000DF93CDB7DEB7A9970FB6F894DEBF0FBE56
:10042000CDBF80916D02811104C08091991282FF2D
:100430000FC32091BF063AE0239FF0011124FAA3D5
:10044000E9A330E08091C4069091C50628173907CA
:1004500038F429A13AA1265F3F4F38A32F8F0AC055
:100460008091C6069091C706E9A1FAA1E80FF91F8D
:10047000F8A3EF8F80918E1290918F12A09190121D
:10048000B091911281309048A105B10540F01092D1
:100490008E1210928F1210929012109291126091FF
:1004A0008E1270918F12809190129091911225E08E
:1004B00030E040E050E00E9451B98091981290E005
:1004C000A0E0B0E0281739074A075B0710F4209333
:1004D000981220909812312CB5E0CB2ED12CE12C23
:1004E000F12C8091BF06811150C0222019F12CE01F
:1004F000329EC0011124FC013396FCA3EBA39C01A6
:10050000245F3F4F3EA32DA3832D90E001962CE066
:10051000289FF001299FF00D1124F8A7EFA389A0CF
:100520009AA011E031E0320D39A7422C512C612CF8
:10053000712C6CC080916D028823A9F080918E127D
:1005400090918F12A0919012B091911226E205978E
:10055000A105B10510F446E201C040E261EB72E191
:10056000832D0E94B8778091991282FFC0CF80912D
:100570008E1290918F12A0919012B09191120597C6
:10058000A105B10508F0B3CF53C22110B0CF8091BF
:100590006D028823A9F080918E1290918F12A09104
:1005A0009012B091911220E20597A105B10510F4C7
:1005B0004EE301C040E268EA72E1832D0E94B87701
:1005C0008091991282FF93CF80918E1290918F1219
:1005D000A0919012B09191120597A105B10508F074
:1005E00086CF0E945179F8DA33C28091C00690918B
:1005F000C1060197881999099093C3068093C20692
:10060000121551F01F5FFFEF8F1A9F0A2F8D38A12F
:100610008216930650F3B9C080916D02882309F4C5
:100620009DC060918E1270918F1280919012909166
:100630009112A70196010E9451B9C4016AE070E0CD
:10064000241535054605570509F054C00E942AB9FE
:1006500044E1489F5001499FB00C1124C5018950C5
:100660009A4F5C01FC0180818111138A61E08EE95F
:1006700092E10E94A9AB0CE010E020E830E04BA131
:100680005CA160E070E08EE992E10E9400AE60E063
:100690008EE992E10E94A9AB1092DE121092DD1257
:1006A0002DA13EA13093E0122093DF1260E28AE98F
:1006B00092E10E94FDB0850133E1A30E8A2D801BDB
:1006C000F80161918F01662329F08AE992E10E9485
:1006D000FDB0F4CF182F112339F060E28AE992E1DE
:1006E0000E94FDB01150F7CF61E08EE992E10E94C7
:1006F000A9AB34C00E942AB9F4E1F89F8001F99FA8
:10070000100D112409501A4FF80180818111138AAC
:100710001092DE121092DD122FA138A53093E01254
:100720002093DF1260E28AE992E10E94FDB0580155
:100730000D5E102F1A19F50161915F01662329F0F2
:100740008AE992E10E94FDB0F4CF112339F060E212
:100750008AE992E10E94FDB01150F7CF8091991281
:1007600082FF0DC160918E1270918F128091901254
:1007700090919112A70196010E9451B92415350557
:100780004605570509F0FBC0FCC04091C4065091D6
:10079000C50660918E1270918F1280919012909187
:1007A00091124115510509F463C02091C60630919C
:1007B000C706232B09F45CC02091BF0630E0241744
:1007C0003507B8F5121156C020916D022223B9F0F9
:1007D000A70196010E9451B9812F90E0A0E0B0E0FE
:1007E000281739074A075B0719F420E24EE302C0D5
:1007F00020E240E26EE972E1832D0E94B877809199
:10080000991282FF37C060918E1270918F12809181
:10081000901290919112A70196010E9451B9812FD7
:1008200090E0A0E0B0E0281739074A075B0711F510
:10083000FBC02417350709F054C012111BC02091CA
:100840006D022223A1F1A70196010E9451B9812FC7
:1008500090E0A0E0B0E0281739074A075B0719F4D9
:1008600026E246E202C026E240E269E972E11CC0EB
:10087000121511F01F5F35C020916D022223B9F0CF
:10088000A70196010E9451B9812F90E0A0E0B0E04D
:10089000281739074A075B0719F426E246E202C027
:1008A00026E240E264E972E1832D0E94B8778091EC
:1008B000991282FFDFCF60918E1270918F1280911A
:1008C000901290919112A70196010E9451B9812F27
:1008D00090E0A0E0B0E0281739074A075B0751F61F
:1008E000A7C060918E1270918F128091901290919A
:1008F0009112A70196010E9451B9812F90E0A0E0CA
:10090000B0E0281739074A075B0788F035E0139FE6
:10091000C00111240197AA2797FDA095BA2F8093B3
:100920008E1290938F12A0939012B09391126091B7
:100930008E1270918F128091901290919112A70156
:1009400096010E9451B98091981290E00496422F2E
:1009500050E08417950764F48CEF820F809398120F
:1009600041E040936D02ABEF2A2E220E33243A94DD
:100970003394239484E0831508F0B3CD69C019A59E
:1009800042CE0E9451798091F408823121F48AE8A4
:1009900092E10E94B3196091C2068FE099E00E9433
:1009A000C94E83E199E09F938F9383E892E19F93EF
:1009B0008F938E010F5F1F4F1F930F930E947ABD7D
:1009C000E0E2F9E00F900F900F900F900F900F90D2
:1009D0008191882339F09091C00095FFFCCF8093DE
:1009E000C600F6CF8091C00085FFFCCF8AE08093DF
:1009F000C6007E01F5E0EF0EF11CF701808188232F
:100A000049F0992787FD90950E9459BCF701819381
:100A10007F01F3CFC8010E9440198FE792E10E9445
:100A2000B3190E94957514C00E94517956D810C010
:100A30000E94517981E69CE890936F0280936E0248
:100A400010928E1210928F12109290121092911298
:100A5000A9960FB6F894DEBF0FBECDBFDF91CF9140
:100A60001F910F91FF90EF90DF90CF90BF90AF90CC
:100A70009F908F907F906F905F904F903F902F90BE
:100A80000895CF93DF93FC01E95BFF4F2081EC01D8
:100A90002496211105C081E08083CE010E9449ABDC
:100AA000CE01DF91CF910C947CABEF92FF920F932C
:100AB0001F9361E081E40E9450B061E081E40E94F4
:100AC00089B08AE992E1DDDF62E478E18EE992E1C2
:100AD0000E9436AA61E08EE992E10E94A9AB0091E2
:100AE000A0121091A11220919E1230919F1240E00D
:100AF00050E060E070E08EE992E10E9400AE61E0BB
:100B00008EE992E10E94A9AB8EE992E10E9480AB4E
:100B10008111DACF8AE992E1B4DF1DEAE12E1CE10E
:100B2000F12E00E410E020E130E040E050E060E031
:100B300070E08EE992E10E9452A68EE992E10E9455
:100B400080AB8111EACF1F910F91FF90EF90089534
:100B5000AF92BF92CF92DF92EF92FF920F931F93CB
:100B6000CF93DF935C01EB019AE9C92E92E1D92E74
:100B7000F60126813781255231094DEDE42E42E1FF
:100B8000F42EF701118210820FED12E1F80131838A
:100B9000208362E478E18EE992E10E9436AAC501E1
:100BA0000E9457766AE3C6010E94FDB0F601868175
:100BB00097818597FE0101900020E9F79F01215060
:100BC00031092C1B3D0B67EF6203A001639F500DA1
:100BD00011249A0122583F4FF70131832083F801F5
:100BE00091838083BE01C601DF91CF911F910F9148
:100BF000FF90EF90DF90CF90BF90AF900C94FCB03F
:100C00002091E21221110AC044E150E0BC0180E7CA
:100C100092E00E94F3BC82E080936D0208952091DF
:100C2000E21221110AC044E150E0BC0180E792E0E9
:100C30000E9489BC82E080936D020895CF93DF9378
:100C4000109211098FE099E00E94B44E0E94D76A79
:100C500080EE94E10E94B3198091F4108823F9F09A
:100C60001092F410C0919D08D0E0CC0FDD1FC45C41
:100C7000DD4E68817981882777FD8095982F0E94C5
:100C800022B620914702309148024091490250918A
:100C90004A020E9483B7181614F4198218828CED48
:100CA00094E10E94B3190E94957582ED94E1B7DF3B
:100CB0000E9470AE6093CA067093CB068093CC06F8
:100CC0009093CD0681E08093F008DF91CF91089555
:100CD0008091F70880FD16C092E09093F008909103
:100CE000F608992341F087FF06C01092F7088DECB3
:100CF00094E10E94B3198FE099E00E94CE4980EC04
:100D000094E18DCF08958FE099E00E94D54983E06A
:100D10008093F0088091F70880FF03C08EEB92E18A
:100D200002C086EB92E17BCF7ADF81E08093E21212
:100D30000C9495751092E2120895CF92DF92EF9283
:100D4000FF92CF93C6B1C6FBCC27C0F981E0C8277C
:100D5000349BC260C0909412D0909512E09096128D
:100D6000F09097120E9470AEC616D706E806F906F4
:100D700010F4329B39C0C0939912809199128170FE
:100D80009091991291FD826090919312891721F1AF
:100D90008130F1F028F0823089F08330A1F01CC05E
:100DA000913021F4909192129F5F05C09230A1F48E
:100DB000909192129150909392120EC0992391F3B8
:100DC000933051F4F5CF923069F3913029F4F0CF9C
:100DD000933041F3992361F380939312CF91FF9065
:100DE000EF90DF90CF900895C460C5CF5EDE60E0E5
:100DF0008FE10E9450B060E081E20E9450B060E05C
:100E000081E30E9450B0469A449A60E083E20E94D7
:100E100050B0429A9FB7F894EBE0F1E08081816096
:100E200080839FBF809109018095817080938D128E
:100E300084DF109292120895CF92DF92EF92FF9288
:100E4000CF93DF937ADF80910901817091E0892748
:100E500020918D128217E1F082E080936D028091E3
:100E600009018170892780938D121FDE80918D1278
:100E7000882339F08FE099E00E94074981E792E1E9
:100E800006C08FE099E00E94CA4984E692E1C7DE7D
:100E9000C0908912D0908A12E0908B12F0908C1240
:100EA0000E9470AEC616D706E806F90608F0C3C061
:100EB00040919212442361F181E080936D025527A5
:100EC00047FD5095652F752F80918E1290918F124E
:100ED000A0919012B0919112840F951FA61FB71F79
:100EE00080938E1290938F12A0939012B0939112D0
:100EF000109292120E9470AE6856754C8F4F9F4FA1
:100F00006093401270934112809342129093431267
:100F10008091991282FF0EC00E9470AE6856754C87
:100F20008F4F9F4F609340127093411280934212F3
:100F3000909343128091EF128F5F8093EF128AE9B2
:100F400092E19FDDCDE7D0E062E478E18EE992E1C5
:100F50000E9436AAD093DE12C093DD121092E012E6
:100F60001092DF128091EF1280FF02C061E001C099
:100F700060E08EE992E10E94A9AB4FE350E06FE799
:100F800070E08EE992E10E948EAB61E08EE992E121
:100F90000E94A9ABE0916E02F0916F0219958091C9
:100FA0006D02811107C08091F0089BEF980F94307B
:100FB00068F007C08EE992E10E9480AB8111C4CF36
:100FC000F2CFC1E08C3018F4C0E001C0C1E0C090A5
:100FD0004012D0904112E0904212F09043120E94D1
:100FE00070AEC616D706E806F90648F480916E0280
:100FF00090916F028557904A11F0CC23B1F0809107
:101000006D02882319F0815080936D020E9470AEAA
:101010006C597F4F8F4F9F4F6093891270938A1244
:1010200080938B1290938C1206C00E94957582E07B
:1010300080936D02E4CFDF91CF91FF90EF90DF902E
:10104000CF9008958091991282FB882780F90895A6
:10105000FC01808190E02AE030E0B9010E943EB9B5
:10106000482FCB01B9010E943EB9805D80934412A4
:10107000405D409345121092461284E492E1089537
:1010800020E030E040E251E4FC0160817181828126
:1010900093810E9455B80E94EFB577FD02C02BE204
:1010A00001C02DE2209344129B0177FF04C0222748
:1010B0003327261B370BC90168EE73E00E943EB947
:1010C000CB01EAE0F0E0BF010E943EB9805D809371
:1010D0004512C90164E670E00E943EB9CB01BF0130
:1010E0000E943EB9805D80934612C901BF010E94F3
:1010F0003EB9282FCB01BF010E943EB9805D80938D
:1011000047128EE280934812205D2093491210927C
:101110004A1284E492E10895CF92DF92EF92FF9217
:101120000F931F9380918E1290918F12A091901225
:10113000B09191120097A105B10509F486C02091E4
:10114000F408BC01882777FD8095982F223139F467
:101150000E9422B62DEC3CEC4CEC5DE30AC00E94F0
:1011600022B620914C1230914D1240914E12509166
:101170004F120E9455B89B01AC016091E20870913A
:10118000E3088091E4089091E5080E94A7B4609379
:10119000E2087093E3088093E4089093E50820E068
:1011A00030E0A9016091E2087091E3088091E408C1
:1011B0009091E5080E9480B587FF08C01092E20870
:1011C0001092E3081092E4081092E508609100097B
:1011D00070910109882777FD8095982F0E9422B68B
:1011E0006B017C019B01AC016091E2087091E30806
:1011F0008091E4089091E5080E9483B7181644F4A2
:10120000C092E208D092E308E092E408F092E50888
:1012100010928E1210928F121092901210929112C0
:101220006DE9C62E68E0D62EE12CF12C00E712E421
:1012300026EE38E042EE58E06EED78E08AED98E078
:101240000E94E55781E080936D0280916D028823B2
:1012500039F082EE98E014DFBC018DE595E178DC91
:101260008091991282FF17C00E9451798091F408F1
:10127000823119F488E991E902C086E899E79093F0
:101280006F0280936E0210928E1210928F12109243
:101290009012109291121F910F91FF90EF90DF909A
:1012A000CF900895BF92CF92DF92EF92FF920F936B
:1012B0001F93CF93DF931F92CDB7DEB780918E122D
:1012C00090918F12A0919012B09191120097A10568
:1012D000B10509F443C0BC01882777FD8095982F9C
:1012E0000E9422B620914C1230914D1240914E1224
:1012F00050914F120E9455B89B01AC016091E608D5
:101300007091E7088091E8089091E9080E94A7B4DD
:101310006093E6087093E7088093E8089093E908E3
:1013200010928E1210928F121092901210929112AF
:10133000BB24B394B982CE0101966C01E12CF12C4F
:1013400000EA11E426EE38E042EE58E06EED78E077
:101350008AED98E00E94E557B0926D0280916D028F
:10136000882339F086EE98E08BDEBC018FE195E1B1
:10137000EFDB8091991282FF10C00E94517986E8BC
:1013800099E790936F0280936E0210928E121092E2
:101390008F1210929012109291120F90DF91CF91B4
:1013A0001F910F91FF90EF90DF90CF90BF90089525
:1013B000CF92DF92EF92FF920F931F93CF93DF9321
:1013C0001F92CDB7DEB780918E1290918F12A091AF
:1013D0009012B09191120097A105B10509F442C095
:1013E000BC01882777FD8095982F0E9422B6209116
:1013F0004C1230914D1240914E1250914F120E945A
:1014000055B89B01AC016091E6087091E7088091A6
:10141000E8089091E9080E94A7B46093E6087093E9
:10142000E7088093E8089093E90810928E121092D2
:101430008F1210929012109291121982CE01019681
:101440006C01E12CF12C00EA11E426EE38E042EECA
:1014500058E06EED78E08AED98E00E94E55781E073
:1014600080936D0280916D02882339F086EE98E0BA
:1014700007DEBC0186E195E16BDB8091991282FF6A
:1014800010C00E94517986E899E790936F0280938B
:101490006E0210928E1210928F1210929012109271
:1014A00091120F90DF91CF911F910F91FF90EF90CC
:1014B000DF90CF900895CF92DF92EF92FF920F933B
:1014C0001F9380918E1290918F12A0919012B091E3
:1014D00091120097A105B10509F474C0BC018827D9
:1014E00077FD8095982F0E9422B620914C12309162
:1014F0004D1240914E1250914F120E9455B82091BA
:10150000DE083091DF084091E0085091E1080E9428
:10151000A7B46B017C0120E030E0A9010E9480B5F6
:1015200087FD09C0C092DE08D092DF08E092E00893
:10153000F092E10808C01092DE081092DF081092C5
:10154000E0081092E1086091FE087091FF0888277A
:1015500077FD8095982F0E9422B66B017C019B013C
:10156000AC016091DE087091DF088091E0089091F5
:10157000E1080E9483B7181644F4C092DE08D092A6
:10158000DF08E092E008F092E10810928E121092CB
:101590008F121092901210929112ADE9CA2EA8E00B
:1015A000DA2EE12CF12C06E114E426EE38E042EECE
:1015B00058E06EED78E08AED98E00E94E55781E012
:1015C00080936D0280916D02882339F08EED98E052
:1015D00057DDBC0184E195E1BBDA8091991282FF6D
:1015E00010C00E94517986E899E790936F0280932A
:1015F0006E0210928E1210928F1210929012109210
:1016000091121F910F91FF90EF90DF90CF9008956E
:10161000CF92DF92EF92FF920F931F9380918E12E1
:1016200090918F12A0919012B09191120097A10504
:10163000B10509F474C0BC01882777FD8095982F07
:101640000E9422B620914C1230914D1240914E12C0
:1016500050914F120E9455B82091DA083091DB0862
:101660004091DC085091DD080E94A7B46B017C0119
:1016700020E030E0A9010E9480B587FD09C0C0923A
:10168000DA08D092DB08E092DC08F092DD0808C0AE
:101690001092DA081092DB081092DC081092DD0834
:1016A0006091FC087091FD08882777FD8095982F40
:1016B0000E9422B66B017C019B01AC016091DA08AB
:1016C0007091DB088091DC089091DD080E9483B75F
:1016D000181644F4C092DA08D092DB08E092DC08D5
:1016E000F092DD0810928E1210928F1210929012CA
:1016F000109291121DE9C12E18E0D12EE12CF12C8F
:1017000006E114E426EE38E042EE58E06EED78E0B3
:101710008AED98E00E94E55781E080936D02809108
:101720006D02882339F08AED98E0AADCBC0182E1E1
:1017300095E10EDA8091991282FF10C00E945179D2
:1017400086E899E790936F0280936E0210928E1252
:1017500010928F1210929012109291121F910F916D
:10176000FF90EF90DF90CF90089520E030E040E2CE
:1017700051E4FC0160817181828193810E9455B89E
:101780000E94EFB5FB0177FD2FC0CB0168EE73E03F
:101790000E943EB9CB012AE030E0B9010E943EB977
:1017A000805D80934412CF0164E670E00E943EB9F0
:1017B000CB01B9010E943EB9805D80934512CF01F3
:1017C000B9010E943EB9482FCB01B9010E943EB930
:1017D000805D809346128EE280934712405D409375
:1017E00048121092491235C02DE220934412EE2780
:1017F000FF27E61BF70BCF0168EE73E00E943EB9AE
:10180000CB012AE030E0B9010E943EB9805D8093AF
:101810004512CF0164E670E00E943EB9CB01B901E8
:101820000E943EB9805D80934612CF01B9010E94AB
:101830003EB9482FCB01B9010E943EB9805D80932B
:1018400047128EE280934812405D409349121092F5
:101850004A1284E492E10895FC01808191818436EA
:1018600091055CF064E670E00E943EB9CB016AE04D
:1018700070E00E943EB9805D01C080E28093441216
:10188000808191818A3091055CF02AE030E0B901D5
:101890000E943EB9CB01B9010E943EB9805D01C0F2
:1018A00080E280934512808191816AE070E00E941D
:1018B0003EB9805D809346121092471284E492E113
:1018C0000895CF92DF92EF92FF920F931F93CF93E1
:1018D000DF938091F008813011F41092F00880912C
:1018E0008E1290918F12A0919012B091911281302E
:1018F0009048A105B10540F010928E1210928F12FF
:10190000109290121092911260918E1270918F121B
:10191000809190129091911225E030E040E050E0EB
:101920000E9451B98091981290E0A0E0B0E0281791
:1019300039074A075B0710F420939812D091981248
:10194000C0E011E025E0C22ED12CE12CF12CDD23EA
:1019500071F02091F40860918E1270918F12809135
:10196000901290919112213109F035C22EC08091D0
:101970006D028823A9F080918E1290918F12A09110
:101980009012B091911226E20597A105B10510F4CD
:1019900046E201C040E260EF76E18C2F0E94B8770A
:1019A0008091991282FFD5CF80918E1290918F12E3
:1019B000A0919012B09191120597A105B10548F63A
:1019C0000E94517985E790EA89C42091F00822505D
:1019D000223008F079C0D13099F520916D02222390
:1019E00099F0A70196010E9451B9213031054105B6
:1019F000510519F42AEF4EE302C02AEF40E26BEEE4
:101A000076E18C2F0E94B8778091991282FD02C0F6
:101A100003E0FFC060918E1270918F12809190123E
:101A200090919112A70196010E9451B92130310580
:101A30004105510569F70E94517985E59DE94EC43C
:101A4000D23031F720916D022223F9F0A7019601DF
:101A50000E9451B98091F6082230310541055105A7
:101A600049F4882319F04DED56E102C049ED56E1E5
:101A70006EE308C0882319F045ED56E102C041ED40
:101A800056E160E28C2F0E942B808091991282FF98
:101A9000BFCF60918E1270918F12809190129091B1
:101AA0009112A70196010E9451B9223031054105DA
:101AB000510509F0ADCF0E9451798091F60891E06F
:101AC00089278093F6082BC4D13099F520916D02B7
:101AD000222399F0A70196010E9451B921303105C6
:101AE0004105510519F42AEF4EE302C02AEF40E206
:101AF00069EC76E18C2F0E94B8778091991282FD73
:101B000002C004E086C060918E1270918F128091A5
:101B1000901290919112A70196010E9451B9213023
:101B200031054105510569F70E94517988E094E932
:101B3000D5C3D23091F520916D02222399F0A701EF
:101B400096010E9451B9223031054105510519F421
:101B500020E24EE302C020E240E260EC76E18C2F0E
:101B60000E94B8778091991282FFCBCF60918E123C
:101B700070918F128091901290919112A70196010D
:101B80000E9451B9223031054105510509F0B9CF04
:101B90000E9451798CEB96E1B8C3D33009F0B1CFF4
:101BA00020916D02222399F0A70196010E9451B95C
:101BB000233031054105510519F420E24EE302C0FE
:101BC00020E240E26DEA76E18C2F0E94B8778091A6
:101BD000991282FF96CF60918E1270918F12809130
:101BE000901290919112A70196010E9451B9233051
:101BF00031054105510509F084CF0E945179DF91EB
:101C0000CF911F910F91FF90EF90DF90CF900C94A8
